:100000000C94CE310C94C8340C94F3340C941E35FB
:100010000C9449350C9474350C949F350C94CA3566
:100020000C94F5350C94FF310C94FF310C94FF3196
:100030000C94FF310C94FF310C94FF310C94FF3180
:100040000C94FF310C945EEE0C94FF310C94FF3154
:100050000C94FF310C94FF310C9437DD0C94013279
:100060000C94FF310C9435B50C94E1B50C94FF3130
:100070000C94FF310C94FF310C94FF310C94FF3140
:100080000C94FF310C94FF310C94FF310C94FF3130
:100090000C94FF310C94FF310C94FF310C94FF3120
:1000A0000C94FF310C94FF310C94FF310C94FF3110
:1000B0000C94FF310C94FF310C94FF310C94FF3100
:1000C0000C94FF310C94FF310C94FF310C94FF31F0
:1000D0000C94FF310C94FF310C94FF310C94FF31E0
:1000E0000C94FF313E334333483352335C33D533C2
:1000F00066336E33763380338A339433A333AD3330
:10010000D533B733C133CB33F933FC33EB33EF3370
:10011000F5333334003404340A340E3412341834D2
:100120001C342034333426342A342E34C56DA56D66
:10013000AB6DA86DAE6DB16DB46DC06DB76DD26DA8
:10014000BA6DBD6D70B26EB292B28FB28DB2C4B2E2
:10015000C1B2BFB21DB3EBB2E8B2E6B268B56EB5DC
:100160007FB58AB592B5A7B596B5A7B59AB59EB530
:10017000A7B5A4B54AC44FC454C45CC461C466C422
:100180006BC470C48DC48DC475C48DC47AC47FC45F
:1001900088C4A8C4ADC4B2C4BAC4BFC4C4C4C9C4AA
:1001A000CEC4EBC4EBC4D3C4EBC4D8C4DDC4E6C432
:1001B00006C50BC510C518C51DC522C527C52CC54C
:1001C00049C549C531C549C536C53BC544C564C5E2
:1001D00069C56EC576C57BC580C585C58AC5A7C5F9
:1001E000A7C58FC5A7C594C599C5A2C56EC673C658
:1001F0007EC689C694C69FC6AAC6B5C6EAC6EAC662
:10020000EAC6EAC6C0C609C715C726C737C748C762
:1002100059C76AC77BC7B3C7B3C7B3C7B3C789C713
:10022000D2C7DEC7EFC700C811C822C833C844C848
:100230007CC87CC87CC87CC852C89BC8A4C8B3C84A
:10024000BEC8C9C8D4C8DFC8E9C818C918C918C900
:1002500018C9F1C85AC960C96AC976C982C999C999
:10026000A9C97ECAB9C97ECAC9C97ECADAC9E6C9DE
:10027000FBC907CA39CA43CA4BCA57CA63CA72CA3A
:10028000A5CAAECABBCACACAD9CAF3CA06CB0DCC64
:1002900019CB0DCC2CCB0DCC40CB52CB6ACB84CB25
:1002A000B9CBC6CBD1CBE0CBEFCB01CC34CC3DCC62
:1002B0004ACC59CC68CC82CC95CC9CCDA8CC9CCDDA
:1002C000BBCC9CCDCFCCE1CCF9CC13CD48CD55CD1A
:1002D00060CD6FCD7ECD90CDC3CDC9CDD1CDDBCDA1
:1002E000E3CDF8CD06CED7CE14CED7CE22CED7CE04
:1002F00031CE40CE53CE6ACE9FCEA7CEAFCEB7CEB4
:10030000BFCECECE084AD73B3BCE016E84BCBFFDEC
:10031000C12F3D6C74319ABD56833DDA3D00C77FD5
:1003200011BED9E4BB4C3E916BAAAABE000000806E
:100330003F05A84CCDB2D44EB93836A9020C50B9FD
:10034000918688083CA6AAAA2ABE000000803F0029
:100350000D94B2730D94FD510D94A7780D94542C07
:100360004E414E494E495459494E46CDCCCC3D0A9A
:10037000D7233C17B7D13877CC2B329595E6241F7D
:10038000B14F0A000020410000C84200401C462036
:10039000BCBE4CCA1B0E5AAEC59D7400000A0B02AF
:1003A000090C0D0E08070304010000000000000006
:1003B000000000000000000000000000000000003D
:1003C00000000000000000121110000000000000FA
:1003D000000000000000000000000000000000001D
:1003E0000001021020200808102040102040800248
:1003F000010201080402010102040810204080806B
:1004000040201008040201800402018040201008EE
:1004100004020108040201010204081020408001C6
:100420000204081020408005050505070508080896
:1004300008020202020A0A08080404040401010175
:10044000010101010103030303030303030407077D
:10045000070C0C0C0C0C0C0C0C020202020606061B
:1004600006060606060B0B0B0B0B0B0B0B000020F6
:10047000002300260029002C002F0032000001007C
:100480000003010601090100002200250028002BBD
:10049000002E003100340002010000050108010BAC
:1004A0000100002100240027002A002D0030003325
:1004B0000001010000040107010A0101060D00FE10
:1004C00009016602D620FFFE0BFE0AFE0D00602227
:1004D0001969808080808080800080183363A0A0AC
:1004E000A00357675050F850F850500259692078CF
:1004F000A0A0702828F02002596948A85010204078
:1005000050A89002586840A0A040A0989068281376
:1005100063808080113B6B204040808080808040E1
:100520004020113B6B804040202020202040408014
:1005300006556520A870A8200455652020F82020C5
:10054000113363604080065161F811336340E0402D
:100550000259690808101020404080800259692023
:1005600050888888888850200259692060A02020FF
:10057000202020F80259697088880810204080F8EF
:10058000025969F80810207008088870025969102B
:100590001030505090F81010025969F88080B0C89F
:1005A0000808887002596970888080F0888888708F
:1005B000025969F808101020204040400259697023
:1005C00088888870888888700259697088888878D7
:1005D0000808887011386840E040000040E0401191
:1005E000386840E0400000604080025969081020EF
:1005F000408040201008045464F80000F802596953
:1006000080402010081020408002596970888808B6
:10061000102020002002596970888898A8A8B0800E
:10062000780259692050888888F888888802596932
:10063000F048484870484848F002596970888080FE
:100640008080808870025969F04848484848484886
:10065000F0025969F8808080F0808080F802596942
:10066000F8808080F0808080800259697088808066
:10067000809888887002596988888888F88888886E
:1006800088123969E040404040404040E0025969EA
:10069000381010101010109060025969888890A0CE
:1006A000C0A0908888025969808080808080808086
:1006B000F80259698888D8A8A88888888802596962
:1006C00088C8C8A8A89898888802596970888888B6
:1006D0008888888870025969F0888888F0808080CE
:1006E00080015A6A70888888888888A870080259AA
:1006F00069F0888888F0A09088880259697088809D
:10070000807008088870025969F820202020202075
:1007100020200259698888888888888888700259CA
:1007200069888888885050502020025969888888B4
:1007300088A8A8A8A850025969888850502050500D
:10074000888802596988885050202020202002592A
:1007500069F808101020404080F8113B6BE0808061
:1007600080808080808080E00259698080404020C5
:1007700010100808113B6BE02020202020202020B2
:1007800020E0085363205088015161F82A226280DA
:10079000400256667008788898680259698080809F
:1007A000F088888888F00256667088808088700299
:1007B0005969080808788888888878025666708899
:1007C000F880887002596930484040F0404040400D
:1007D0000058687088888878088870025969808015
:1007E00080B0C8888888881238684000C04040407F
:1007F00040E0004A6A100030101010109090600223
:10080000596980808090A0C0A09088123969C0404A
:10081000404040404040E0025666D0A8A8A8A888C2
:10082000025666B0C88888888802566670888888AC
:100830008870005868F0888888F080808000586848
:100840007888888878080808025666B0C880808052
:10085000800256667088601088700258684040F0C8
:10086000404040483002566688888888986802561A
:10087000668888885050200256668888A8A8A850A4
:1008800002566688502020508800586888888898CA
:1008900068088870025666F810204080F8015B6B8B
:1008A0001820202020C020202020182219698080B4
:1008B00080808080808080015B6BC0202020201899
:1008C00020202020C008536348A890FFFFFFFFFFAF
:1008D000FFFFFFFFFFFFFFFFFFFFFFFFFFFFFFFF28
:1008E000FFFFFFFFFFFFFFFFFFFFFFFF0D00602285
:1008F0001969800080808080808080035868207023
:10090000A8A0A0A8702002596930484040E04040AB
:1009100048B00356668870505070880259698888BC
:100920005050F820F82020221969808080800080B3
:10093000808080124A6A6090806090906010906021
:100940001A3262A0A00359697088A8D8C8D8A888AC
:1009500070045767700878887800F8035666285046
:10096000A0A05028045363F80808163161E0035929
:10097000697088E8D8D8E8D888700A5161F81744B7
:1009800064609090600357672020F8202000F807EB
:10099000356540A02040E007356540A04020C02AD2
:1009A000226240800058688888888898E8808002A1
:1009B000596978E8E8E8E868282828262161C020F5
:1009C0002262408007356540C04040E004576770B0
:1009D0008888887000F8035666A050282850A00226
:1009E0005A6A40C04040E00818283808025A6A4055
:1009F000C04040E01028081038025A6A40A0402049
:100A0000A048182838080259692000202040808812
:100A10008870025A6A40200020508888F88888022E
:100A20005A6A10200020508888F88888025A6A3054
:100A3000480020508888F88888025A6A2850002088
:100A4000508888F88888025A6A5050002050888858
:100A5000F88888025A6A20502020508888F88888B0
:100A600002596958A0A0A0B0E0A0A0B8005B6B70CC
:100A700088808080808088702040025A6A402000F0
:100A8000F88080F08080F8025A6A102000F8808098
:100A9000F08080F8025A6A304800F88080F0808048
:100AA000F8025A6A505000F88080F08080F8123ABC
:100AB0006A804000E04040404040E0123A6A2040F6
:100AC00000E04040404040E0124A6A609000E04050
:100AD00040404040E0123A6AA0A000E04040404060
:100AE00040E0025969F0484848E8484848F0025A4E
:100AF0006A2850008888C8A8988888025A6A4020C6
:100B00000070888888888870025A6A10200070886F
:100B10008888888870025A6A304800708888888877
:100B20008870025A6A285000708888888888700205
:100B30005A6A505000708888888888700355658884
:100B400050205088015B6B08709898A8A8A8C8C866
:100B50007080025A6A4020008888888888887002DD
:100B60005A6A10200088888888888870025A6A30FB
:100B7000480088888888888870025A6A505000889F
:100B8000888888888870025A6A10200088885020D7
:100B900020202002596980F0888888F080808002B7
:100BA0005969609090A0A0908888B002596940204F
:100BB00000700878889868025969102000700878D9
:100BC00088986802596930480070087888986802E7
:100BD00059692850007008788898680259695050FF
:100BE00000700878889868025A6A304830007008A7
:100BF00078889868025666702870A0A850005868D7
:100C00007088808088702040025969402000708878
:100C1000F88088700259691020007088F880887008
:100C20000259693048007088F8808870025969500C
:100C300050007088F8808870123969804000C04088
:100C4000404040E0123969204000C040404040E050
:100C5000124969609000C040404040E0123969A0EC
:100C6000A000C040404040E0025A6A50206010702E
:100C70008888888870025969285000B0C888888898
:100C800088025969402000708888888870025969F4
:100C90001020007088888888700259693048007078
:100CA00088888888700259692850007088888888E8
:100CB000700259695050007088888888700357679F
:100CC000202000F8002020015868087098A8A8C8C3
:100CD0007080025969402000888888889868025985
:100CE000691020008888888898680259693048000F
:100CF0008888888898680259695050008888888850
:100D00009868005B6B102000888888986808887055
:100D1000005A6A8080B0C88888C8B08080005B6B49
:100D2000505000888888986808887001050700FE80
:100D30000500FB01F220FFFE05FE05FE0200400259
:100D400015258080800080053242A0A002556550A4
:100D5000F850F8500146562070C030E0200255652A
:100D60009010204048025565608068906805122206
:100D700080800225354080808040022535804040BB
:100D80004080043343A040A003334340E0400122AD
:100D9000324080043141E002112180025565081083
:100DA0002040800245556090909060022535C040FB
:100DB000404040024555E0106080F0024555E0108B
:100DC0006010E00245552060A0F020024555F080FB
:100DD000E010E00245556080E09060024555F0105B
:100DE00020404002455560906090600245556090FB
:100DF0007010600313238000800214248000808020
:100E00000235452040804020033343E000E00235B6
:100E1000458040204080024555E01060004002556A
:100E2000657088B8A870024555609090F0900245B2
:100E300055E090E090E0023545608080806002459A
:100E400055E0909090E0023545E080E080E002358A
:100E500045E080E080800245557080B0907002458A
:100E6000559090F09090023545E0404040E00245BA
:100E700055301010906002455590A0C0A0900235EA
:100E80004580808080E002556588D8A88888024522
:100E90005590D0B09090024555609090906002457A
:100EA00055E09090E080014656609090906010026E
:100EB0004555E09090E09002455570806010E0024A
:100EC0003545E0404040400245559090909060028A
:100ED00045559090A0A04002556588A8A8A850024A
:100EE000455590906090900245559090701060022A
:100EF0003545E0204080E0022535C0808080C0027A
:100F000055658040201008022535C0404040C0058E
:100F1000324240A0024151F0052232804002445446
:100F20007090907002455580E09090E002344460EB
:100F3000808060024555107090907002445460B0FB
:100F4000C0600235452040E0404000465670909019
:100F500070106002455580E0909090021525800049
:100F60008080800027374000404040408002455547
:100F70008090A0E0900215258080808080025464DB
:100F8000F0A8A8A8024454E09090900244546090C5
:100F90009060004656E09090E08080004656709049
:100FA00090701010023444A0C0808002445470C07D
:100FB00030E002354540E04040200244549090909B
:100FC000700244549090A040025464A8A85050026B
:100FD0003444A04040A000465690909070106002AB
:100FE0004454F02040F002354560408040600215D6
:100FF000258080808080023545C0402040C0054269
:101000005250A0FFFFFFFFFFFFFFFFFFFFFFFFFFAB
:10101000FFFFFFFFFFFFFFFFFFFFFFFFFFFFFFFFE0
:10102000FFFFFFFF020040FFFFFFFFFFFFFFFFFF8B
:10103000FFFFFFFFFFFFFFFFFFFFFFFFFFFFFFFFC0
:10104000FFFFFFFFFFFFFFFFFFFFFFFFFFFFFFFFB0
:10105000FFFFFFFFFFFFFFFFFFFFFFFFFFFFFFFFA0
:10106000FFFFFFFFFFFFFFFFFFFFFFFFFFFFFFFF90
:10107000FFFFFFFFFFFFFFFFFFFFFFFFFFFFFFFF80
:10108000FFFFFFFFFFFF01050800FF0601210235FA
:1010900020FFFF07FF06FF090050221656808080C0
:1010A000800080153353A0A0A00257575050F8502D
:1010B000F850500257572070A070287020133555F3
:1010C00080A040A02002475740A0A040A0A05025EB
:1010D00013538080801226564080808080401226E4
:1010E000568040404040800245559060F06090023C
:1010F00055552020F8202011335360408004415181
:10110000F011335340E040024656101020408080DA
:1011100012365640A0A0A0A04012365640C0404013
:1011200040E00246566090106080F0024656F02083
:10113000601090600246562060A0F02020024656C3
:10114000F080E01090600246566080E0909060026F
:101150004656F01020204040024656609060909025
:1011600060024656609090701060122555C0C00015
:10117000C0C0113656606000604080123656204074
:1011800080804020034353F000F012365680402008
:1011900020408012365640A0204000400158583070
:1011A0004898A8A8904030024656609090F09090E1
:1011B000024656E090E09090E002465660908080B3
:1011C0009060024656E090909090E0024656F08083
:1011D000E08080F0024656F080E080808002465633
:1011E000609080B090600246569090F0909090127F
:1011F0003656E040404040E002465670202020A095
:101200004002465690A0C0A0A09002465680808022
:101210008080F002465690F0F090909002465690F2
:10122000D0F0B0B090024656609090909060024628
:1012300056E09090E08080014757609090D0B06079
:1012400010024656E09090E0909002465660904022
:10125000209060123656E040404040400246569092
:1012600090909090600246569090909060600246F8
:1012700056909090F0F0900246569090606090905A
:10128000025656888850202020024656F0102040F2
:1012900080F0123656E080808080E00246568080E2
:1012A00040201010123656E020202020E016325246
:1012B00040A0014151F016225280400244547090E7
:1012C00090700246568080E09090E0123454608026
:1012D000806002465610107090907002445460B0C6
:1012E000C060024656205040E040400145556090A5
:1012F0007010600246568080E09090901236564002
:1013000000C04040E01137572000202020A04002BC
:101310004656808090E09090123656C04040404043
:10132000E0025454D0A8A8A8024454E0909090023F
:10133000445460909060014555E090E08080014504
:10134000557090701010024454A0D0808012345414
:1013500060C020C00246564040E040502002445445
:1013600090909070123454A0A0A04002545488A8C9
:10137000A850024454906060900145559090709040
:1013800060024454F02040F0024757304020C02013
:101390004030221656808080808080024757C020CF
:1013A00040304020C006425250A0FFFFFFFFFFFF29
:1013B000FFFFFFFFFFFFFFFFFFFFFFFFFFFFFFFF3D
:1013C000FFFFFFFFFFFFFFFFFFFFFF090050221697
:1013D000568000808080800146562070A0A070203A
:1013E0000246562050E04050A0025555887050707B
:1013F000880256568850F820F8202217578080809F
:10140000008080800247577080E0907010E01731B4
:1014100051A002565670A8C8C8A87014355560A0CF
:101420006000E003435350A050123353E0202014D7
:101430003151E002565670E8D8E8D870173151E0C3
:1014400015335340A04012355540E04000E01435BC
:101450005540A02040E0143555C020C020C01622C1
:10146000524080014555909090E08002565678E8B1
:10147000E8682828241151801122524080143555E3
:1014800040C04040E014355540A04000E0034353C5
:10149000A050A0024757808080A060F020024757EC
:1014A0008080A0D010207002475780408060A0F05C
:1014B0002012365640004080A0400247574020602E
:1014C00090F0909002475720406090F09090024733
:1014D0005760906090F0909002475750A06090F055
:1014E000909002475790006090F0909002475760AC
:1014F000906090F0909002465670A0A0F0A0B001CD
:101500004757609080809060400247574020F080AD
:10151000E080F00247572040F080E080F00247571B
:101520006090F080E080F00247579000F080E0800B
:10153000F01237578040E0404040E01237572040DB
:10154000E0404040E012375740A0E0404040E01209
:101550003757A000E0404040E00256567048E84847
:10156000487002475750A090D0B090900247574023
:10157000206090909060024757204060909090606B
:101580000247576090609090906002475750A0606B
:101590009090906002475790006090909060123356
:1015A00053A040A002465670B0B0D0D0E0024757DA
:1015B00040209090909060024757204090909090EB
:1015C000600247576090909090906002475790005B
:1015D0009090909060025757102088502020200251
:1015E000465680E09090E0800246566090A0A09021
:1015F000A00247574020007090907002475720404B
:1016000000709090700247572050007090907002C8
:10161000475750A00070909070024656500070904E
:10162000907002475760906070909070025454F030
:1016300068B078113555608080604002475740207F
:101640000060B0C06002475720400060B0C0600238
:10165000475760900060B0C060024656500060B0CE
:10166000C060123757804000C04040E0123757201A
:101670004000C04040E012375740A000C04040E06A
:10168000123656A000C04040E0024757A040A010CC
:1016900070906002475750A000E09090900247572A
:1016A000402000609090600247572040006090907A
:1016B000600247576090006090906002475750A0CA
:1016C00000609090600246569000609090601235E5
:1016D000554000E0004002445470B0D0E00247574B
:1016E00040200090909070024757204000909090CA
:1016F000700247576090009090907002465690009C
:101700009090907001485820400090907090600137
:1017100047578080E090E08080014757900090908C
:1017200070906025753A2530327500253032753A53
:101730002530327500202020200025202000252083
:1017400000253164002532640025336400253464AB
:101750000025356400253664000000007E0060002E
:10176000600060F87ECC60CC60CC60F860CC00CCCF
:1017700000CC00CC00000000000000FE7F0E7026B0
:1017800064724E7A5E324C8241324C7A5E724E26E0
:10179000640E70FE7F000000000000FE7F0E70C629
:1017A00063C24382411A58BA5D1A588241C243C685
:1017B000630E70FE7F00000000000088088808109B
:1017C0001120222022101188088808101100000022
:1017D000000000000000000000000020221011881E
:1017E000088808101120222022101188080000000B
:1017F00000000000000000000000000000000000E9
:10180000000000000000000000000000000000FEDA
:101810007FFE7F06600000000000000000F00FF86F
:101820001FF81FF81FF00FF00FF81FF81FF81FE048
:1018300007C0038001000000003048483045727244
:101840003A207574663820666F6E74206E6F74204F
:10185000696E697469616C697A65642E004572729B
:101860003A207574663820666F6E74206E6F74202F
:10187000696E697469616C697A65642E004572727B
:101880003A207574663820666F6E74206E6F74200F
:10189000696E697469616C697A65642E00506C6563
:1018A000617365207265736574005052494E5445EA
:1018B000522048414C544544007F80FFC0FFC0FF88
:1018C000C07F807F80FFC0FFC0FFC03F001E000CB4
:1018D00000FFFFFF0E000E000E000E000E000E00B7
:1018E0000E000E007FC03F801F000E0004000400A9
:1018F0000E001F003F807FC00E000E000E000E0085
:101900000E000E000E000E0000FE0003FF80078395
:10191000C00E01C00E00E01C00E07F00E03E00E0D1
:101920001C00E00800E00000E00001C00E01C00F54
:10193000078007FF0001FC0003F8000FFE001E0FE8
:1019400000380700380380700380700FE07007C014
:101950007003807001007000003800003807001E1E
:101960000F000FFE0003F80000060C00FE07022621
:1019700003BC017FFE08FE08FE05080806000040C3
:10198000F0C88888987810050808060000C0F88814
:1019900088888888F80505050600012030F8302081
:1019A0000508080600002070F820202020E0050926
:1019B000090600FF2070A8A8B888887020050606D0
:1019C000060001E08CEA8C8A0A0509090600FFF886
:1019D000A88888888888A8F8050A0A0600FE20508A
:1019E00050505088A8A8887003030306000340A045
:1019F00040FFFFFFFFFFFFFFFFFFFFFFFFFFFFFFB6
:101A0000FFFFFFFFFFFFFF0000000605FF010707C4
:101A100006020080808080800080030303060105A9
:101A2000A0A0A005060606000050F85050F850058A
:101A300009090600FF2070A8A07028A870200507DB
:101A400007060000C8C81020409898050707060040
:101A50000040A0A040A89068010303060205808012
:101A6000800309090601FF2040408080804040201B
:101A70000309090601FF80404020202040408005E6
:101A8000070706000020A8702070A820050505069D
:101A900000012020F820200203030601FFC040803F
:101AA000050101060003F8020202060100C0C0059C
:101AB00007070600000810102040408005070706B1
:101AC0000000708898A8C8887003070706010040C6
:101AD000C040404040E0050707060000708808103D
:101AE0002040F8050707060000F808103008887045
:101AF00005070706000010305090F8101005070782
:101B0000060000F880F00808887005070706000046
:101B1000304080F0888870050707060000F808103C
:101B2000102020200507070600007088887088882C
:101B300070050707060000708888780810600205A5
:101B400005060100C0C000C0C00206060601FFC0B5
:101B5000C000C040800305050601012040804020F0
:101B6000050303060002F800F803050506010180DD
:101B700040204080050707060000708810202000E4
:101B8000200507070600007088B8A8B88070050710
:101B900007060000708888F888888805070706000F
:101BA00000F04848704848F00507070600007088B4
:101BB0008080808870050707060000F04848484884
:101BC00048F0050707060000F88080F08080F805DF
:101BD0000707060000F88080F08080800507070670
:101BE00000007088808098887005070706000088CC
:101BF0008888F8888888030707060100E04040408D
:101C00004040E005070706000038101010109060F3
:101C10000507070600008890A0C0A0908805070768
:101C2000060000808080808080F80507070600009D
:101C300088D8A8888888880507070600008888C88B
:101C4000A898888805070706000070888888888813
:101C500070050707060000F08888F080808005077F
:101C60000706000070888888A890680507070600A6
:101C700000F08888F0A090880507070600007088AB
:101C80008070088870050707060000F820202020D3
:101C90002020050707060000888888888888700546
:101CA0000707060000888888885050200507070627
:101CB000000088888888A8A85005070706000088C3
:101CC0008850205088880507070600008888502023
:101CD000202020050707060000F80810204080F8A3
:101CE0000309090601FFE080808080808080E00594
:101CF000070706000080404020101008030909066D
:101D000001FFE020202020202020E0050303060022
:101D1000052050880501010600FEF80303030601B3
:101D200005804020050505060000700878887805C4
:101D300007070600008080F0888888F00505050602
:101D4000000070808088700507070600000808788A
:101D5000888888780505050600007088F080700581
:101D60000707060000304840E040404005070706EE
:101D700000FE7088888878087005070706000080D4
:101D800080F0888888880307070601004000C0406B
:101D90004040E00409090601FE1000301010101048
:101DA000906005070706000080808890E090880317
:101DB0000707060100C04040404040E00505050619
:101DC0000000D0A8A8A8A8050505060000B0C8888E
:101DD0008888050505060000708888887005070753
:101DE0000600FEF0888888F080800507070600FE60
:101DF00078888888780808050505060000B0C8803E
:101E0000808005050506000078807008F00507074A
:101E10000600002020F820202018050505060000F7
:101E200088888898680505050600008888885020FD
:101E30000505050600008888A8A8500505050600C8
:101E40000088502050880507070600FE88888850C3
:101E5000204080050505060000F8102040F8030921
:101E6000090601FF20404040804040402001090910
:101E70000602FF80808080808080808003090906C0
:101E800001FF8040404020404040800503030600A1
:101E90000248A890FF01FFFFFFFFFFFFFFFFFFFFCA
:101EA000FFFFFF0FFFFFFFFFFFFFFFFFFFFFFFFF32
:101EB000FF1E0000000000000000000007FFFF38C8
:101EC0000000000000000000000003FFFF700000A1
:101ED000000000000000000001FFFF6000000000A3
:101EE00000000000000000FFFF6000000000000094
:101EF00000000000007FFFC00000000000000000A4
:101F00007800003FFFC00FC0FC0000000000781800
:101F1000001FFFC03FE1FF0000000000783C000F01
:101F2000FFC07FF3FF8000000000783C0007FFC087
:101F3000FFFFFFC000000000783C0003FFC1F87FF6
:101F400087E00000000078000001FFC1F03F03E0DF
:101F50000000000078000000FFC1E01E01E01F004B
:101F600003E0783C03F07FC1E01E01E07FC00FF882
:101F7000783C07FC3FC1E01E01E1FFE01FFC783C1C
:101F80000FFE1FC1E01E01E3FFF03FFE783C1FFE85
:101F90000FC1E01E01E3F3F83F3E783C3F3F07C12D
:101FA000E01E01E7E0FC7C1F783C3E1F07C1E01EFD
:101FB00001E7C07C7C0F783C3C0F03C1E01E01E7C9
:101FC000807C780F783C3C0F03C1E01E01E7803C29
:101FD0007800783C3C0F03C1E01E01E7803C7800AC
:101FE000783C3C0F03C1E01E01E7803C7800783C60
:101FF0003C0F03C1E01E01E7C03C7800783C3C0F79
:1020000003C1E01E01E3E03C78007C3C3C0F03C1CF
:10201000E01E01E3FF3FF8007FBC3C0F03C1E01E60
:1020200001E1FF3FF8003FBFFC0F03C1E01E01E0EC
:10203000FF3FF8001FBFFC0F03C1E01E01E07F3F20
:10204000F8000FBFFC0F036000000000000000005C
:102050000000000007600000000000000000000019
:1020600000000670000000000000000000000000FA
:102070000E380000000000000000000000001C1EE0
:10208000000000000000000000000000780FFFFFCB
:10209000FFFFFFFFFFFFFFFFFFFFF001FFFFFFFF5D
:1020A000FFFFFFFFFFFFFFFF8000000000000000B8
:1020B0000000000000000000000000000000000020
:1020C0000000000000000000000000000C00000004
:1020D000000000000C0000000000000012000000E2
:1020E00000000000230000000000000021000000AC
:1020F000000000004C800000000000005E80000036
:10210000000000009240000000000000A14000001C
:102110000000000121200000000000027F9000006C
:10212000000000020010000000000007FFF800009F
:102130000000000400080000000000080004000087
:10214000000000080006000000000010000200006F
:10215000000000301E010000000000207F81000010
:1021600000000041FFE0800000000043FCF0800020
:10217000000000873B7840000000018EDBFC60001F
:102180000000010FEBCC20000000021FEDB6100094
:102190000000021FDEB6100000000439CD7F0800E9
:1021A00000000436E0FF08000000087EC0BB840089
:1021B0000000187F005D86000000107FC0ED8200E7
:1021C0000000203CC07301000000203B337F010071
:1021D0000000701BE77E03800000C81DEEDE04C017
:1021E0000000880FDEDC04400001240FDF3C0920E2
:1021F00000012607DBF8192000027203E7F01390B4
:1022000000025101FFE02290000489007F802448F1
:10221000000904801E004824000BFE400000DFF48B
:102220000010004000008002001FFFFFFFFFFFFEC4
:10223000000000000000000000000000000000009E
:102240000000000000000000001022103C3C0E1FA7
:102250000010221004221104001022100822110480
:1022600000102210083C110400102210102211044A
:102270000010221020221104001E1C1E3C3C0E04E3
:10228000000000000000000000000000000000004E
:10229000000000000000000000000000000000003E
:1022A000000000000000000000000000000000002E
:1022B000000000000000000000000000000000001E
:1022C000000000000000000000000000000000000E
:1022D00000000000000000000000000000000000FE
:1022E0000000000000000000060900FE060189024F
:1022F000FE20FFFE07FE06FE0000000600070106A6
:10230000060602008080808000800303030601032C
:10231000A0A0A00507070600FF5050F850F8505045
:102320000509090600FE2070A8A07028A8702006E4
:1023300008080600FF40A848102048540805070771
:102340000600FF6090906098906801030306020306
:102350008080800207070602FF40808080808040E6
:102360000207070602FF8040404040408005050507
:102370000600008850F8508805050506000020205A
:10238000F820200204040602FEC04040800501013E
:10239000060002F8020202060200C0C00406060699
:1023A00001001010204080800406060601006090A5
:1023B0009090906003060606010040C0404040E057
:1023C0000406060601006090102040F00406060690
:1023D0000100F020601010E0050606060000103035
:1023E0005090F810040606060100F080E01010E09E
:1023F0000406060601006080E09090600406060670
:102400000100F01010204040040606060100609014
:102410006090906004060606010060909070106065
:10242000020505060200C0C000C0C0020707060280
:10243000FEC0C000C04040800505050600001860D1
:10244000806018050303060001F800F8050505067D
:102450000000C0300830C00407070601006090107B
:10246000604000400506060600007090A8B080702D
:10247000050606060000205088F88888050606062E
:102480000000F088F08888F00406060601006090DD
:1024900080809060040606060100E090909090E035
:1024A000040606060100F080E08080F004060606BF
:1024B0000100F080E0808080040606060100609044
:1024C00080B090600406060601009090F090909015
:1024D000030606060100E040404040E0050606060F
:1024E000000038101010906004060606010090A04D
:1024F000C0A090900406060601008080808080F0D5
:1025000005060606000088D8A8A8888804060606DE
:10251000010090D0B09090900506060600007088EB
:1025200088888870040606060100E09090E08080AC
:102530000407070601FF609090D0B0601004060603
:10254000060100E09090E09090040606060100600D
:102550009040209060050606060000F8202020200C
:1025600020040606060100909090909060040606F4
:10257000060100909090F060600506060600008855
:1025800088A8A8D888050606060000885020205094
:1025900088050606060000888850202020040606CC
:1025A000060100F010204080F0030606060100E05E
:1025B00080808080E00406060601008080402010B4
:1025C00010030606060100E020202020E00503039A
:1025D0000600032050880501010600FEF8020202F1
:1025E0000602048040040404060100709090700408
:1025F00006060601008080E09090E00404040601D5
:102600000070808070040606060100101070909023
:102610007004040406010060B0C0700406060601E0
:1026200000205040E040400406060601FE60909005
:102630007010600406060601008080E09090900310
:1026400006060601004000C04040E00308080601FD
:10265000FE200060202020A0400406060601008025
:1026600080A0C0A090030606060100C04040404084
:10267000E0050404060000D0A8A8880404040601AC
:1026800000E09090900404040601006090906004C3
:1026900006060601FEE09090E08080040606060132
:1026A000FE709090701010040404060100A0D08009
:1026B0008004040406010070C030E0040606060130
:1026C000004040E040502004040406010090909037
:1026D0007004040406010090906060050404060084
:1026E0000088A8A8500404040601009060609004CB
:1026F00006060601FE9090907090600404040601A6
:1027000000F02040F0030707060100204040804011
:1027100040200107070602FF8080808080808003C0
:102720000707060100804040204040800402020666
:10273000010350A0FFFFFFFFFFFFFFFFFFFFFFFFB1
:10274000FFFFFFFFFFFFFFFFFFFFFFFFFFFFFFFF99
:10275000FFFFFFFFFF00000006000701060606025C
:10276000008000808080800406060601FF2070A0A3
:10277000A070200507070600FF304840F04040F8F1
:10278000050505060000A8508850A80506060600A5
:10279000008850F820F8200107070602FF8080809B
:1027A000008080800407070601FF70806090601041
:1027B000E0030101060105A0060707060000788472
:1027C00094A494847803050506010160A06000E0EC
:1027D0000505050600002850A05028040303060143
:1027E00000F01010040101060102F00607070600C0
:1027F000007884B4A4A48478040101060105F004DF
:1028000003030601026090600507070600FF202011
:10281000F8202000F803050506010140A02040E053
:10282000030505060101C0204020C0020202060285
:102830000440800405050601FF9090B0D080050695
:102840000606000078E8E86828280101010602026F
:10285000800202020602FE408003050506010140D7
:10286000C04040E003050506010140A04000E0052E
:102870000505060000A0502850A00508080600FF26
:1028800040C04050703078100508080600FF40C076
:102890004050680810380508080600FFC020403086
:1028A000F0307810040707060100200020608090B7
:1028B0006005070706000040202050708888050743
:1028C00007060000102020507088880507070600C2
:1028D0000020502050708888050707060000285007
:1028E00020507088880507070600005000205070AF
:1028F000888805070706000020502050708888054A
:10290000060606000078A0F0A0A0B804080806019A
:10291000FE60908080906020400407070601004020
:1029200020F080E080F00407070601002040F080DE
:10293000E080F00407070601002050F080E080F0FE
:102940000407070601005000F080E080F00307074D
:102950000601008040E0404040E003070706010018
:102960002040E0404040E003070706010040A0E0AF
:10297000404040E0030707060100A000E04040405F
:10298000E00506060600007048E84848700407079E
:1029900006010050A090D0B09090040707060100F7
:1029A000402060909090600407070601002040607E
:1029B000909090600407070601002050609090906E
:1029C0006004070706010050A06090909060040723
:1029D0000706010050006090909060050505060014
:1029E0000088502050880408080601FF1070B0B01D
:1029F000D0D0E0800407070601004020909090901E
:102A00006004070706010020409090909060040742
:102A1000070601002050909090906004070706017F
:102A2000005000909090906005070706000010206D
:102A3000885020202004060606010080E09090E0E7
:102A4000800406060601006090A0A090A00407077D
:102A500006010040200070909070040707060100F6
:102A6000204000709090700407070601002050007D
:102A70007090907004070706010050A000709090BD
:102A8000700406060601005000709090700407075D
:102A9000060100205020709090700504040600008C
:102AA00070A8B0780406060601FE70808070204091
:102AB00004070706010040200060B0C0700407074B
:102AC00006010020400060B0C07004070706010046
:102AD00020500060B0C0700406060601005000607F
:102AE000B0C070030707060100804000C04040E00E
:102AF000030707060100204000C04040E00307072D
:102B000006010040A000C04040E0030606060100A8
:102B1000A000C04040E004070706010030601070CC
:102B200090906004070706010050A000E09090908C
:102B3000040707060100402000609090600407072A
:102B40000601002040006090906004070706010025
:102B50002050006090906004070706010050A0001C
:102B6000609090600406060601005000609090603E
:102B70000505050600002000F800200404040601F5
:102B80000070B0D0E00407070601004020009090DC
:102B90009070040707060100204000909090700498
:102BA000070706010020500090909070040606066A
:102BB00001005000909090700409090601FE204029
:102BC000009090907090600408080601FE8080E0FC
:102BD0009090E080800408080601FE5000909090DC
:102BE000709060536E346B3300496E766164657229
:102BF0007300427269636B6F7574004D61696E009A
:102C00005072696E742066726F6D2053440050726A
:102C1000696E742066726F6D20534400022E2E0080
:102C20004D61696E005072696E740043616E636538
:102C30006C005374617274207072696E7420003F6E
:102C400000536D6F6F7468696E6700536D6F6F74BA
:102C500068696E67005A005A0059005900580058B8
:102C600000436F7272656374696F6E00436F7272B6
:102C7000656374696F6E004D61696E0046696C61D1
:102C80006D656E7400544D4320647269766572738D
:102C9000004261636B6C6173680053746570732FDD
:102CA0006D6D004A65726B00416363656C657261AE
:102CB00074696F6E0056656C6F6369747900436F59
:102CC0006E66696775726174696F6E0045737465CD
:102CD00070732F6D6D004573746570732F6D6D008B
:102CE0005A73746570732F6D6D005A7374657073C9
:102CF0002F6D6D005973746570732F6D6D0059736E
:102D0000746570732F6D6D005873746570732F6DDB
:102D10006D005873746570732F6D6D00416476613A
:102D20006E6365642053657474696E6773005665DD
:102D30002D6A65726B0056652D6A65726B00567A56
:102D40002D6A65726B00567A2D6A65726B00567932
:102D50002D6A65726B0056792D6A65726B00567824
:102D60002D6A65726B0056782D6A65726B0041643E
:102D700076616E6365642053657474696E67730071
:102D8000416D6178204500416D6178204500416DBD
:102D90006178205A00416D6178205A00416D617858
:102DA000205900416D6178205900416D61782058AB
:102DB00000416D6178205800412D74726176656C18
:102DC00000412D74726176656C00412D72657472DC
:102DD00061637400412D72657472616374004163B4
:102DE00063656C00416363656C00416476616E638A
:102DF00065642053657474696E677300565472611C
:102E000076206D696E005654726176206D696E0091
:102E1000566D696E00566D696E00566D617820457D
:102E200000566D6178204500566D6178205A005635
:102E30006D6178205A00566D6178205900566D6199
:102E400078205900566D6178205800566D617820C1
:102E50005800416476616E636564205365747469DB
:102E60006E6773004C6F6164206D6D004C6F616420
:102E7000206D6D00556E6C6F6164206D6D00556E38
:102E80006C6F6164206D6D00416476616E636520D6
:102E90004B00416476616E6365204B00416476614E
:102EA0006E6365642053657474696E67730044696A
:102EB0007361626C65207374657070657273004D28
:102EC0003834004175746F2D63616C69627261748E
:102ED00065004C6576656C20582041786973004D1B
:102EE000313137204C6576656C696E67205820411A
:102EF0007869730A4732380A473020583136302013
:102F000046393939390A4730205A3520463630306B
:102F1000300A4739310A4D3231312053300A4D34AD
:102F200030300A4D393036205A3630300A4730209A
:102F30005A2D313520463530300A4730205A352059
:102F4000463530300A4739300A4D3430300A4D3971
:102F50003036205A3936300A4D3231312053310A59
:102F60004732380A4D313137204C6576656C696ED1
:102F70006720646F6E652E0A004175746F20686F5C
:102F80006D6500473238004D6F7665206178697352
:102F9000004D61696E004578747275646572200039
:102FA0004175746F20686F6D6500473238004D6F52
:102FB0007665205A004D6F76652059004D6F766515
:102FC0002058004D6F76656D656E7400457874729B
:102FD0007564657220004D6F766520302E316D6D01
:102FE000004D6F766520316D6D004D6F7665203137
:102FF000306D6D004D6F7665206178697300486FA4
:1030000074656E6420746F6F20636F6C6400457824
:1030100074727564657220004D6F7665205A004D9C
:103020006F76652059004D6F76652058004D6F769C
:1030300065205A004D6F76652059004D6F766520EA
:1030400058005761697420666F720066696C616D23
:10305000656E742070757267650000506C656173F1
:103060006520776169742E005072657373206275F4
:1030700074746F6E00746F20726573756D65207067
:1030800072696E74005761697420666F72006669B8
:103090006C616D656E74206C6F616400496E736560
:1030A00072742066696C616D656E7400616E642077
:1030B000707265737320627574746F6E00746F2024
:1030C000636F6E74696E756500507265737320620C
:1030D0007574746F6E00746F2068656174206E6F14
:1030E0007A7A6C65004E6F7A7A6C652068656174D7
:1030F000696E6700506C6561736520776169742E35
:103100002E2E005761697420666F720066696C61CB
:103110006D656E7420756E6C6F61640057616974C3
:1031200020666F720066696C616D656E74206368FD
:10313000616E676500746F20737461727400506112
:10314000726B696E672E2E2E004368616E67696E22
:10315000672046696C616D656E7400554E4C4F4139
:10316000442046494C414D454E54004C4F4144206B
:1031700046494C414D454E540020204E6F7A7A6CA2
:10318000653A20002000456E642066696C616D65BB
:103190006E74206368616E676500507572676520A4
:1031A0006D6F726500004368616E67652066696CCB
:1031B000616D656E7400556E6C6F61642066696C3C
:1031C000616D656E74004C6F61642066696C616D41
:1031D000656E74004D363030204230205425640036
:1031E0004D373032203B2564004D37303220542596
:1031F00064004D3730312054256400507265686595
:10320000617420437573746F6D00507265686561F9
:103210007420437573746F6D0050726568656174D6
:1032200020414253005072656865617420504C41E2
:10323000004261636B004E6F2053442063617264EF
:10324000005072696E742066726F6D2053440041A5
:10325000626F7574205072696E74657200436861A4
:103260006E67652066696C616D656E7400436861A8
:103270006E67652066696C616D656E74004D3630F1
:103280003020423000436F6E666967757261746901
:103290006F6E0054656D7065726174757265004D76
:1032A0006F76656D656E7400526573756D6520701F
:1032B00072696E740054756E650053746F7020707F
:1032C00072696E74005061757365207072696E74F6
:1032D00000496E666F2073637265656E0047616DAD
:1032E0006573005072696E746572205374617473F3
:1032F000004669726D776172652056657273696FF9
:103300006E004D61696E0053746F70207072696E4B
:1033100074004D61696E005072696E742061626F55
:1033200072746564004D3234004D323520500A4DC0
:1033300032340050726F6265205A204F66667365A2
:103340007400426162797374657020590042616251
:103350007973746570205800466C6F7700466C6F07
:10336000770046616E2073706565640046616E206B
:1033700073706565640042656400426564004E6F69
:103380007A7A6C65004E6F7A7A6C65005370656569
:1033900064005370656564004D61696E004261624E
:1033A0007973746570205900426162797374657035
:1033B0002058002569730025696D20256973002553
:1033C00069682025696D20256973002569642025B9
:1033D00069682025696D2025697300256979202594
:1033E0006964202569682025696D20256973003E80
:1033F0002000457874727564656420746F74616C24
:103400003A00256C642E25696D003E20004C6F6EDD
:1034100067657374206A6F622074696D653A003E57
:103420002000546F74616C207072696E742074692E
:103430006D653A00436F6D706C657465643A200089
:103440005072696E7420436F756E743A2000436F3A
:103450006F6C646F776E0046616E20737065656493
:103460000046616E207370656564004265640042C9
:103470006564004E6F7A7A6C65004E6F7A7A6C657F
:10348000004D61696E006F6F6F0000001FC07FF01C
:10349000DDD8FFF87FF04440248000003180000038
:1034A00024804440107CFEFEFE04000E000E007FCF
:1034B000C0FFE0FFE0FFE0FFE006000F001F8036E6
:1034C000C03FC009001680294006000F001F80364B
:1034D000C03FC0168020401080104008801FC037B9
:1034E000607FF05FD050500D80104048905FD077E3
:1034F000707FF01FC0104020200F007FE0FFF0E63B
:1035000070FFF0198036C0C0300F007FE0FFF0E69A
:1035100070FFF0198036C0198047414D45204F5645
:10352000455200526573746F7265206661696C73F1
:10353000616665004C6F61642073657474696E67C1
:10354000730053746F72652073657474696E67736A
:103550000050726F6265205A204F66667365740072
:10356000416476616E6365642053657474696E6747
:1035700073004D61696E0050726F6265205A204F72
:103580006666736574005374657070696E67206D4C
:103590006F64650053656E736F726C65737320683A
:1035A0006F6D696E67004879627269642074687231
:1035B0006573686F6C640044726976657220637528
:1035C0007272656E7400436F6E74726F6C0045307A
:1035D000004F6666004F6E004530005A004F666629
:1035E000004F6E005A0059004F6666004F6E00593A
:1035F0000058004F6666004F6E005800544D43203F
:103600006472697665727300537465616C746843A3
:10361000686F7020656E61626C65640059005900C6
:1036200058005800544D43206472697665727300E7
:103630004530004530005A005A00590059005800E2
:103640005800544D432064726976657273004530AA
:10365000004530005A005A005900590058005800DF
:10366000544D432064726976657273004D696E69CA
:1036700020322072656164792E005072696E74691F
:103680006E672E2E2E005072696E742070617573F5
:10369000656400436172642072656D6F76656400D5
:1036A0004361726420696E736572746564004D33A2
:1036B000310043616E6E6F7420656E7465722073A5
:1036C00075626469723A20002E0A006F70656E2080
:1036D0006661696C65642C2046696C653A200061FE
:1036E00075746F25632E67006572726F7220777232
:1036F0006974696E6720746F2066696C650A004E94
:103700006F74205344207072696E74696E670A008A
:103710005344207072696E74696E672062797465B3
:1037200020002E0A0044656C6574696F6E20666126
:10373000696C65642C2046696C653A200046696CAA
:10374000652064656C657465643A005772697469D4
:103750006E6720746F2066696C653A20002E0A003F
:103760006F70656E206661696C65642C2046696CBB
:10377000653A20002E0A006F70656E206661696CE4
:1037800065642C2046696C653A200046696C6520AA
:1037900073656C65637465640A002053697A653AE1
:1037A000200046696C65206F70656E65643A200084
:1037B0002066696C653A2000667265736800646F04
:1037C000696E67004E6F772000454E442053554286
:1037D000524F5554494E450A002220706F73002203
:1037E00020706172656E743A2200535542524F55F3
:1037F00054494E452043414C4C20746172676574B6
:103800003A2200747279696E6720746F2063616C6C
:103810006C207375622D67636F64652066696C65E3
:1038200073207769746820746F6F206D616E7920E2
:103830006C6576656C732E204D4158206C657665FD
:103840006C2069733A310A004D3234004D32332016
:1038500025730053442063617264206F6B0A006F0C
:1038600070656E526F6F74206661696C65640A00E2
:10387000766F6C756D652E696E6974206661696C12
:1038800065640A00534420696E6974206661696C3E
:103890000A00286E6F2066696C65290043616E6EB0
:1038A0006F74206F70656E2073756264697220009A
:1038B0007C3C3E5E2B3D3F2F5B5D3B2C2A225C0017
:1038C00066616C73650074727565004F4646004F03
:1038D0004E006563686F3A004572726F723A004538
:1038E00072726F722077726974696E6720746F20CC
:1038F000454550524F4D210A005072657373206246
:103900007574746F6E20286F72204D313038292005
:10391000746F2068656174206E6F7A7A6C650A0036
:10392000507265737320627574746F6E20286F72A5
:10393000204D3130382920746F20726573756D65A4
:103940000A00496E736572742066696C616D656EFC
:103950007420616E64207072657373206275747474
:103960006F6E20286F72204D313038290A004D3695
:1039700030303A20546F6F20636F6C6400486F746E
:10398000656E6420746F6F20636F6C640A00486F0B
:1039900074656E6420746F6F20636F6C640A0049F5
:1039A0006E736572742066696C616D656E742061FA
:1039B0006E6420707265737320627574746F6E200C
:1039C000286F72204D313038290A004C4F5700487B
:1039D000494748004F4B004572726F723A20416C64
:1039E0006C200020636F6E6E656374696F6E2E2E9F
:1039F0002E200054657374696E6720004C4F570089
:103A000048494748004F4B004572726F723A204157
:103A10006C6C200020636F6E6E656374696F6E2E30
:103A20002E2E200054657374696E6720004C4F572A
:103A30000048494748004F4B004572726F723A2068
:103A4000416C6C200020636F6E6E656374696F6EED
:103A50002E2E2E200054657374696E6720004C4F23
:103A6000570048494748004F4B004572726F723A01
:103A700020416C6C200020636F6E6E656374696F0B
:103A80006E2E2E2E200054657374696E67200054CC
:103A90004D4320434F4E4E454354494F4E204552CF
:103AA000524F52004452565F5354415455530900EB
:103AB00050574D5F5343414C45090050574D434FBC
:103AC0004E460900434F4F4C434F4E460900434872
:103AD0004F50434F4E460900544849474809090092
:103AE00054434F4F4C5448525309005450574D546F
:103AF0004852530900545354455009090054504F3B
:103B0000574552444F574E0900494F494E09090045
:103B1000475354415409090049484F4C445F4952A6
:103B2000554E090047434F4E460909000900092038
:103B300042616420726573706F6E736521000920A5
:103B400042616420726573706F6E73652100092095
:103B500042616420726573706F6E73652100092085
:103B600042616420726573706F6E73652100303D31
:103B70002E33323500313D2E3138006D6178002F03
:103B80003331002F3331002F333100303D2E3332AB
:103B90003500313D2E3138006D6178002F33310012
:103BA0002F3331002F333100303D2E333235003189
:103BB0003D2E3138006D6178002F3331002F3331C5
:103BC000002F333100303D2E33323500313D2E3160
:103BD00038006D6178002F3331002F3331002F33DF
:103BE0003100447269766572207265676973746525
:103BF00072733A0A006F7409006F7470770900736A
:103C000032676109007332676209006F6C610900F5
:103C10006F6C620900737473740900667361637476
:103C2000697665090073675F726573756C74090066
:103C30007374616C6C677561726409004452565309
:103C40005441545553005374616C6C6775617264D0
:103C50002074687273002D7374617274090068793E
:103C600073746572657369730A2D656E6409006209
:103C70006C616E6B2074696D65006F666620746997
:103C80006D6509004F54207072657761726E20680F
:103C900061730A6265656E20747269676765726533
:103CA00064004F54207072657761726E005B6D6DB9
:103CB0002F735D090070776D0A7468726573686FA1
:103CC0006C640900747374657009006D73746570B9
:103CD000730900737465616C746843686F70007673
:103CE00073656E7365090050574D207363616C6591
:103CF0000043532061637475616C0900486F6C6404
:103D00002063757272656E740052756E20637572F1
:103D100072656E74004D41582063757272656E74E1
:103D200000524D532063757272656E740053657452
:103D30002063757272656E7400456E61626C6564B5
:103D400009000900617869733A70776D5F73636188
:103D50006C652F63757272656E745F7363616C65F9
:103D60002F6D6563685F6C6F61647C666C616773FF
:103D70007C7761726E636F756E740A006D41290AFB
:103D80000020647269766572206F76657274656D65
:103D90007065726174757265207761726E696E67A5
:103DA000212028003A20002063757272656E74200D
:103DB00064656372656173656420746F20006D4192
:103DC000290A0020647269766572206F76657274C4
:103DD000656D7065726174757265207761726E6968
:103DE0006E67212028003A20002063757272656E8C
:103DF000742064656372656173656420746F20006C
:103E00006D41290A0020647269766572206F7665BB
:103E10007274656D70657261747572652077617218
:103E20006E696E67212028003A2000206375727247
:103E3000656E742064656372656173656420746F78
:103E4000200025756420253032753A253032750002
:103E50006D41290A0020647269766572206F76656B
:103E60007274656D706572617475726520776172C8
:103E70006E696E67212028003A20002063757272F7
:103E8000656E742064656372656173656420746F28
:103E90002000447269766572206572726F720063E9
:103EA0006F696C2073686F727420636972637569DF
:103EB000740A006F76657274656D706572617475F1
:103EC00072650A0020647269766572206572726F8D
:103ED000722064657465637465643A2030780063A9
:103EE000616E63656C00726573756D656400726503
:103EF00073756D650070617573656400706F7765CB
:103F0000726F6666002F2F616374696F6E3A0020CE
:103F1000573A0020573A00457874727564657220EC
:103F2000436F6F6C696E672E2E2E00457874727524
:103F30006465722048656174696E672E2E2E0020BC
:103F40002F002042403A0020403A00546865726DCC
:103F5000616C2052756E617761790045312054485B
:103F600045524D414C2052554E41574159004265F2
:103F70006400202D20496E76616C69642065787438
:103F80007275646572206E756D62657220210A001B
:103F900048656174696E67206661696C656400429A
:103FA00065640048656174696E67206661696C6567
:103FB000640045312048656174696E6720666169F7
:103FC0006C6564004D494E54454D502074726967CC
:103FD0006765726564004531204572723A204D492B
:103FE0004E54454D5000426564004D415854454D76
:103FF00050207472696767657265640045312045B9
:1040000072723A204D415854454D5000426564004B
:10401000626564002C2073797374656D2073746F0E
:104020007070656421204865617465725F49443A27
:10403000200023646566696E652044454641554C01
:10404000545F004B6420004B6920004B702000003F
:1040500062656400504944204175746F74756E65E3
:104060002066696E697368656421205075742074D8
:104070006865206C617374204B702C204B69206143
:104080006E64204B6420636F6E7374616E74732072
:1040900066726F6D2062656C6F7720696E746F2039
:1040A000436F6E66696775726174696F6E2E680A18
:1040B00000504944204175746F74756E65206661C7
:1040C000696C6564212074696D656F75740A0054AC
:1040D0006865726D616C2052756E6177617900451B
:1040E0003120544845524D414C2052554E41574184
:1040F00059004265640048656174696E67206661B5
:10410000696C65640045312048656174696E67209B
:104110006661696C656400426564005049442041F1
:1041200075746F74756E65206661696C65642120B5
:1041300054656D706572617475726520746F6F205F
:10414000686967680A00204B643A2000204B693A8E
:104150002000204B703A20000A20436C6173736981
:104160006320504944200A002054753A2000204B17
:10417000753A2000206D61783A2000206D696E3A12
:10418000200020643A200020626961733A200050C8
:104190004944204175746F74756E65207374617243
:1041A000740A00504944204175746F74756E65201F
:1041B0006661696C6564212054656D706572617417
:1041C00075726520746F6F20686967680A00100057
:1041D000AD0330016A0150022B0170030A01900403
:1041E000F500B005E500D006D800F007CE001009B4
:1041F000C500300ABE00500BB700700CB100900D26
:10420000AB00B00EA600D00FA200F0109D0010125F
:104210009900301395005014920070158E0090167E
:104220008B00B0178700D0188400F0198100101B94
:104230007E00301C7B00501D7900701E7600901FA0
:104240007300B0207000D0216E00F0226B001024AB
:1042500069003025660050266300702761009028B1
:104260005E00B0295C00D02A5900F02B5600102DBA
:104270005400302E5100502F4E0070304B009031C2
:104280004800B0324500D0334200F0343E001036D2
:104290003B00303737005038330070392E00903AE9
:1042A0002900B03B2300D03C1B00F03D1100103F23
:1042B0000100F03F00001000C90210012C01400174
:1042C000220170011801B0010E01F0010401500239
:1042D000FA00B002F0003003E600D003DC009004E6
:1042E000D2007005C800A006BE000008B400B009E6
:1042F000AA00D00BA000600E960060118C00001583
:10430000820020197800C01D6E00A0226400B02732
:104310005A00902C500000314600E0343C00103828
:104320003200903A2800603C1E00A03D1400803E00
:104330000A00203F00006F70656E005452494747E5
:1043400045524544003A20007A5F6D6178007A5FFB
:104350006D696E00795F6D617800785F6D696E00E0
:104360005265706F7274696E6720656E6473746FE6
:1043700070207374617475730A00456E6473746F92
:10438000707320256320256320256320256300208A
:104390005A3A0020593A0020583A00656E64737406
:1043A0006F7073206869743A2000486F6D696E679A
:1043B000206661696C6564000A53746174733A2005
:1043C00046696C616D656E7420757365643A200092
:1043D0002C204C6F6E67657374206A6F623A200000
:1043E000546F74616C2074696D653A200053746178
:1043F00074733A20002C204661696C65643A200091
:104400002C2046696E69736865643A2000507269B1
:104410006E74733A200053746174733A2000496ECD
:1044200076616C69642065787472756465720A00DF
:10443000205A3A0020593A0020436F756E74205874
:104440003A00C23100001C260000F4190000D80F09
:104450000000EB080000C0040000750200004001ED
:10446000000024F4D43050C38E20C2A24017828BA7
:104470007011127A910D816CD90AA861E108C758B0
:104480006607615143061E4B5D05C145A7041A41ED
:104490001104093D9803713931034036DB0265335D
:1044A0009102D4305402802E1D02632CEE01752A35
:1044B000C501B028A001102781018F2564012B249C
:1044C0004B01E0223401AC211F018D200D01801F22
:1044D000FC00841EED00971DDF00B81CD200E61B17
:1044E000C600201BBC00641AB200B219A8000A1949
:1044F000A0006A189900D117910040178B00B516DB
:10450000840031167E00B31579003A157300C71484
:104510006F0058146A00EE136600881363002513B9
:104520005E00C7125B006C12570015125400C111D7
:10453000510070114F0021114B00D61049008D1011
:1045400047004610440002104200C00F4000800F98
:104550003E00420F3C00060F3B00CB0E3800930E8E
:1045600037005C0E3500270E3400F30D3200C10D0C
:104570003100900D3000600D2E00320D2D00050D24
:104580002C00D90C2B00AE0C2900850C29005C0CEA
:104590002700350C27000E0C2600E80B2400C40B66
:1045A0002400A00B23007D0B23005A0B2100390BA4
:1045B0002100180B2000F80A1F00D90A1E00BB0AB0
:1045C0001E009D0A1D00800A1D00630A1C00470A88
:1045D0001B002C0A1B00110A1A00F7091A00DD093A
:1045E0001900C4091900AB091900920917007B09C9
:1045F0001800630917004C09160036091600200937
:1046000016000A091500F5081500E0081400CC088A
:104610001400B8081400A4081400900813007D08C2
:1046200012006B08130058081200460812003408E4
:104630001100230811001208110001081100F007F1
:104640001000E0071000D0071000C0071000B007EE
:104650000F00A107100091070E0083070F007407D9
:104660000F0065070E0057070E0049070E003B07B5
:104670000D002E070E0020070D0013070D00060782
:104680000D00F9060C00ED060D00E0060C00D40646
:104690000C00C8060C00BC060C00B0060C00A406FA
:1046A0000B0099060C008D060B0082060B007706A6
:1046B0000B006C060B0061060A0057060B004C0647
:1046C0000A0042060A0038060A002E060A002406DE
:1046D0000A001A060A001006090007060A00FD056E
:1046E0000900F4050900EB050900E2050900D905F8
:1046F0000900D0050900C7050900BE050900B50578
:104700000800AD050800A50509009C0508009405F2
:1047100008008C050800840508007C050800740565
:1047200008006C050700650508005D0507005605D3
:1047300008004E050700470507004005080038053A
:104740000700310507002A050700230507001C059F
:104750000600160507000F050700080506000205FC
:104760000700FB040600F5040700EE040600E80459
:104770000600E2040700DB040600D5040600CF04AF
:104780000600C9040600C3040600BD040600B70401
:104790000600B1040500AC040600A6040600A0044F
:1047A00005009B04060095040500900406008A0499
:1047B000050085040500800406007A0405007504E0
:1047C0000500700405006B04050066040500610423
:1047D00005005C04050057040500520405004D0463
:1047E000050048040500430405003E0404003A04A3
:1047F000050035040500300404002C0405002704DE
:104800000400230405001E0404001A040400160416
:104810000500110404000D0404000904050004044B
:10482000040000040400FC030400F8030400F40383
:104830000400F0030400EC030400E8030400E403B4
:104840000400E0030400DC030400D8030400D403E4
:104850000400D0030400CC030400C8030300C50314
:10486000030024F404D9201BC40C5C0E9804C40972
:104870005F0265077101F405F900FB04B300480409
:104880008700C10369005803550003034500BE02B9
:104890003A008402310053022A0029022500040252
:1048A0002000E4011C00C8011900AF0117009801A5
:1048B0001400840113007101100061011000510106
:1048C0000E0043010D0036010B002B010B002001EF
:1048D0000B00150109000C01090003010800FB0091
:1048E0000800F3000800EB000700E4000600DE000B
:1048F0000600D8000600D2000600CC000500C70064
:104900000500C2000500BD000400B9000400B500A8
:104910000400B1000400AD000400A9000400A500DB
:104920000300A20003009F0004009B000300980006
:1049300003009500020093000300900003008D0027
:1049400002008B0003008800020086000200840041
:104950000300810002007F0002007D0002007B0056
:104960000200790002007700010076000200740066
:10497000020072000100710002006F0002006D0071
:1049800001006C0002006A0001006900020067007B
:104990000100660001006500010064000200620081
:1049A000010061000100600001005F0002005D0085
:1049B00001005C0001005B0001005A000100590089
:1049C0000100580001005700010056000100550089
:1049D0000100540001005300000053000100520088
:1049E000010051000100500001004F0001004E0085
:1049F00000004E0001004D0001004C0001004B0082
:104A000000004B0001004A0001004900010048007D
:104A10000000480001004700010046000000460079
:104A20000100450000004500010044000100430072
:104A3000000043000100420000004200010041006C
:104A4000000041000100400001003F0000003F0065
:104A500001003E0000003E0001003D0000003D005E
:104A600001003C0000003C0000003C0001003B0055
:104A700000003B0001003A0000003A00010039004C
:104A80000000390001003800000038000000380044
:104A9000010037000000370001003600000036003A
:104AA0000000360001003500000035000000350030
:104AB0000100340000003400000034000100330025
:104AC000000033000000330001003200000032001B
:104AD0000000320001003100000031000000310010
:104AE00001003000000030000000300001002F0005
:104AF00000002F0000002F0000002F0001002E00FA
:104B000000002E0000002E0001002D0000002D00EE
:104B100000002D0000002D0001002C0000002C00E2
:104B200000002C0000002C0001002B0000002B00D6
:104B300000002B0000002B0001002A0000002A00CA
:104B400000002A0000002A000100290000002900BE
:104B500000002900000029000000290001002800B1
:104B600000002800000028000000280000002800A5
:104B70000100270000002700000027000000270098
:104B8000000027000100260000002600000026008B
:104B9000000026000000260001002500000025007E
:104BA0000000250000002500000025000000250071
:104BB0000100240000002400000024000000240064
:104BC0000000240001002300000023000000230057
:104BD0000000230000002300000023000000230049
:104BE000010022000000220000002200000022003C
:104BF000000022000000220001002100000021002E
:104C00000000210000002100000021000000210020
:104C10000000210001002000000020000000200012
:104C20000000200000002000000020000000200004
:104C30000000200001001F0000001F0000001F00F6
:104C400000001F0000001F0000001F0000001F00E8
:104C500001001E0000001E0000001E0000001E00DB
:104C6000000020204D363033200020204D393134D3
:104C70000020204D3931330020204D393036003AA4
:104C80000A0020286D6D29002055004C0046696CF3
:104C9000616D656E74206C6F61642F756E6C6F61F1
:104CA00064206C656E677468733A0A0020204D3981
:104CB0003030204B004C696E656172204164766132
:104CC0006E63653A0A005430204500205A0020598E
:104CD00000205800447269766572207374657070A4
:104CE000696E67206D6F64653A0A0020590020588C
:104CF00000544D4332313330205374616C6C47752E
:104D0000617264207468726573686F6C643A0A003B
:104D1000205430204500205A0020590020580048D7
:104D20007962726964205468726573686F6C643A62
:104D30000A00205430204500205A002059002058F5
:104D400000537465707065722064726976657220B4
:104D500063757272656E743A0A0020204D383531E1
:104D6000205A005A2D50726F6265204F6666736537
:104D7000740020440020490020204D33303420505E
:104D80000020440020490020204D333031205000C5
:104D90005049442073657474696E67733A0A002041
:104DA000460020420020480020204D313435205359
:104DB000004D6174657269616C206865617475701D
:104DC00020706172616D65746572733A0A0020200B
:104DD0004D3432302053004175746F204265642099
:104DE0004C6576656C696E673A0A00204500205A6A
:104DF0000020590020580020540020530020204D4E
:104E000032303520420020453C6D61785F655F6A35
:104E100065726B3E0020583C6D61785F785F6A6513
:104E2000726B3E20593C6D61785F795F6A65726B89
:104E30003E205A3C6D61785F7A5F6A65726B3E0016
:104E4000416476616E6365643A20423C6D696E5FD1
:104E50007365676D656E745F74696D655F75733ECC
:104E600020533C6D696E5F66656564726174653E72
:104E700020543C6D696E5F74726176656C5F666527
:104E80006564726174653E00205400205200202049
:104E90004D323034205000416363656C657261743B
:104EA000696F6E2028756E6974732F7332293A20EA
:104EB000503C7072696E745F616363656C3E205232
:104EC0003C726574726163745F616363656C3E20FC
:104ED000543C74726176656C5F616363656C3E0A15
:104EE00000204500205A0020590020204D3230314A
:104EF0002058004D6178696D756D20416363656C64
:104F000065726174696F6E2028756E6974732F7392
:104F100032293A0A00204500205A0020590020205A
:104F20004D3230332058004D6178696D756D2066C3
:104F300065656472617465732028756E6974732F7A
:104F400073293A0A00537465707320706572207576
:104F50006E69743A0A0020204D3134392043203BD9
:104F600020556E69747320696E2043656C73697592
:104F7000730A002020473231202020203B20556E2C
:104F800069747320696E206D6D0020204D353639AF
:104F90002053310048617264636F64656420446526
:104FA0006661756C742053657474696E6773204C08
:104FB0006F616465640A002823000028230000C88C
:104FC000000000E803000000009643000096430044
:104FD000009643000020420000C8420000C8420082
:104FE0000048430000D243290A00206279746573A7
:104FF0003B2063726320002073746F7265642073BA
:10500000657474696E67732072657472696576651C
:1050100064202800202863616C63756C617465648A
:1050200029210A0020213D2000454550524F4D20A6
:10503000435243206D69736D61746368202D20288D
:1050400073746F7265642920002053697A653A2071
:1050500000496E6465783A2000204D61726C696E7B
:105060003D563634290A00454550524F4D2076654D
:105070007273696F6E206D69736D61746368202847
:10508000454550524F4D3D00290A00206279746514
:10509000733B20637263200053657474696E677399
:1050A0002053746F7265642028000A003B20454538
:1050B00050524F4D20496E6465783A200055706417
:1050C0006174696E67207A6F666673657420696EB5
:1050D00020454550524F4D3A2000454550524F4DC6
:1050E000206461746173697A65206572726F722ED3
:1050F0000A0050726F62696E67206661696C656450
:105100000A0050726F62696E67206661696C65643F
:10511000005761726E696E673A20486F6D696E67FD
:105120002042756D702044697669736F72203C204F
:10513000310A00020204486F6D652025732573252E
:1051400073206669727374002066697273740A0052
:10515000486F6D65200020746F6F206C6F6E672044
:10516000657874727573696F6E2070726576656E9E
:105170007465640A0020636F6C64206578747275CE
:1051800073696F6E2070726576656E7465640A006F
:1051900020453A00205A3A0020593A00583A000077
:1051A0000048420000484200002042FF0101000088
:1051B000000000000000000000400000304300003C
:1051C000454300003743000040C00000404300005A
:1051D000374300002D4300004043000037430000E8
:1051E00040C00000A0C00000000020746F6F206C61
:1051F0006F6E6720657874727573696F6E20707258
:105200006576656E7465640A0020636F6C64206562
:105210007874727573696F6E2070726576656E74DE
:1052200065640A00627573793A207061757365640C
:1052300020666F7220696E7075740A0062757379EA
:105240003A2070617573656420666F7220757365AE
:10525000720A00627573793A2070726F63657373B6
:10526000696E670A004D3131372050726F626520D8
:105270007375636365737366756C0A0020496E7697
:10528000616C6964206578747275646572200020B1
:105290005A3A200020593A200042656420583A20AA
:1052A0000050726F6265205A204F66667365743ACB
:1052B00020003F5A206F7574206F662072616E6700
:1052C0006520282D3220746F2035290A004D313495
:1052D0003520533C696E6465783E206F7574206F8D
:1052E000662072616E67652028302D31290A0043DF
:1052F0006C69636B20746F20726573756D652E2EFB
:105300002E00220A00556E6B6E6F776E20636F6DF4
:105310006D616E643A202200454550524F4D204F3A
:105320004B0A004E6F206D6F76652E004543484F47
:1053300000494E464F004552524F52530044525975
:1053400052554E00434F4D4D554E49434154494FE0
:105350004E006F6666002C53315336533D53445311
:1053600044454255473A004C756C7A426F74204D63
:10537000696E692032204F46462E00205A0020597F
:1053800000580020204D61783A2000205A00205912
:1053900000580020204D696E3A2000536F6674203B
:1053A000656E6473746F70733A20005072696E7426
:1053B0002074696D653A20004D3131332053002F40
:1053C0002F20004361703A004348414D4245525FEF
:1053D00054454D5045524154555245004D4F544946
:1053E0004F4E5F4D4F44455300544845524D414C3C
:1053F0005F50524F54454354494F4E004155544F0E
:105400005245504F52545F53445F53544154555387
:105410000050524F4D50545F535550504F5254000E
:10542000454D455247454E43595F504152534552B1
:1054300000434153455F4C494748545F42524947F6
:1054400048544E45535300544F47474C455F4C49D1
:105450004748545300534F4654574152455F504FAD
:10546000574552004255494C445F50455243454EC2
:1054700054004C4556454C494E475F444154410009
:105480005A5F50524F4245004155544F4C45564586
:105490004C005052494E545F4A4F420050524F47C1
:1054A00052455353004155544F5245504F52545F4B
:1054B00054454D5000564F4C554D455452494300AC
:1054C000454550524F4D0042494E4152595F464961
:1054D0004C455F5452414E53464552005345524944
:1054E000414C5F584F4E5F584F4646004649524D1B
:1054F000574152455F4E414D453A4D61726C696E60
:1055000020204649524D574152455F564552534916
:105510004F4E3A322E302E302E31313520455854F0
:1055200052554445525F545950453A48617264653A
:105530006E6564537465656C20534F555243455FE7
:10554000434F44455F55524C3A68747470733A2F18
:105550002F636F64652E616C6570686F626A656346
:1055600074732E636F6D2F646966667573696F6EF1
:105570002F4D41524C494E2050524F544F434F4CA7
:105580005F56455253494F4E3A312E30204D4143DC
:1055900048494E455F545950453A4C756C7A426FB4
:1055A00074204D696E692032204558545255444547
:1055B000525F434F554E543A3120555549443A6550
:1055C000353530323431312D643436642D34323156
:1055D000642D626133612D61323031323664373986
:1055E0003330660A0020284E6F7420796574206D70
:1055F000656173757265642900202041766572616A
:105600006765206D65617375726564206261636BA7
:105610006C61736820286D6D293A002020536D6FEE
:105620006F7468696E6720286D6D293A20202020EC
:105630002020202020202020202020202053002057
:10564000204261636B6C6173682044697374616E9E
:10565000636520286D6D293A2020202020202020FD
:105660000020202020202846312E30203D20667545
:105670006C6C2C2046302E30203D206E6F6E6529DC
:105680000A002020436F7272656374696F6E204157
:105690006D6F756E742F466164652D6F75743A2059
:1056A0002020202046006163746976653A0A00690B
:1056B0006E004261636B6C61736820636F72726528
:1056C0006374696F6E2069732000205A0020506F48
:1056D000736974696F6E616C204572726F723A0AF9
:1056E000004E6F7A7A6C6520546970204F7574652E
:1056F000722044696D656E73696F6E733A0A00209B
:1057000020546F703A2000202046726F6E743A2049
:105710000020204C6566743A20004261636B6C6126
:1057200073683A0A00205A0043656E7465723A0A3B
:1057300000202046726F6E743A200020204C65666F
:10574000743A20002020546F703A20005369646539
:10575000733A0A00426564204C6576656C696E6731
:1057600020004661696C656420746F20656E61621B
:105770006C6520426564204C6576656C696E670ACD
:1057800000426564204C6576656C20436F727265DB
:105790006374696F6E204D61747269783A000A0A09
:1057A000426564204C6576656C20436F7272656358
:1057B00074696F6E204D61747269783A00202B0015
:1057C0000A436F72726563746564204265642048A1
:1057D00065696768742076732E2042656420546F73
:1057E000706F6C6F67793A0A00202B000A4265647B
:1057F0002048656967687420546F706F67726170C4
:1058000068793A0A2020202B2D2D2D204241434B30
:10581000202D2D2B0A2020207C202020202020201D
:10582000202020207C0A204C207C20202020282B97
:1058300029202020207C20520A2045207C20202066
:1058400020202020202020207C20490A2046207C67
:1058500020282D29204E20282B29207C20470A2073
:1058600054207C20202020202020202020207C204C
:10587000480A2020207C20202020282D292020209C
:10588000207C20540A2020207C2020202020202042
:10589000202020207C0A2020204F2D2D2046524FF2
:1058A0004E54202D2D2B0A2028302C30290A00346C
:1058B00074682070726F626520706F696E742C203E
:1058C00064697374616E63652066726F6D20706CBD
:1058D000616E653A2000202844525952554E2900E5
:1058E000473239204175746F20426564204C6576DB
:1058F000656C696E67003F20284C2C522C462C4268
:1059000029206F7574206F6620626F756E64732E28
:105910000A003F50726F626520706F696E74732069
:1059200028592920697320696D706C6175736962EB
:105930006C652028322D32292E0A003F50726F628A
:105940006520706F696E7473202858292069732050
:10595000696D706C61757369626C652028322D32D7
:10596000292E0A003F2856296572626F7365206CE4
:105970006576656C20697320696D706C61757369FB
:10598000626C652028302D34292E0A00437572720E
:10599000656E742066696C653A2000456E64206609
:1059A000696C65206C6973740A00426567696E20D2
:1059B00066696C65206C6973740A00416476616E77
:1059C0006365204B3D003F4B2076616C7565206F11
:1059D0007574206F662072616E67652028302D31E6
:1059E00030292E0A004D31313720486F7420456E22
:1059F000642048656174696E672E2E2E0A4D313021
:105A00003420533137302054300A473238204F3158
:105A10000A473120593235205A313020463530304E
:105A2000300A4D31303920523137302054300A4D50
:105A3000313137205265776970696E67206E6F7AF1
:105A40007A6C650A54300A47312058343520593170
:105A500037342046353030300A4731205A310A4D2C
:105A600031303920523137300A473120583435200F
:105A7000593137342046343030300A4731205834D9
:105A80003520593137342046343030300A47312000
:105A900058343520593137342046343030300A47B5
:105AA00031205834352059313734204634303030A5
:105AB0000A473120583435205931373420463430A4
:105AC00030300A4731205834352059313734204698
:105AD000343030300A47312058343520593137348A
:105AE0002046343030300A4731205834352059317F
:105AF00037342046343030300A473120583435208E
:105B0000593137342046343030300A473120583448
:105B10003520593137342046343030300A4731206F
:105B200058343520593137342046343030300A4724
:105B30003120583435205931373420463430303014
:105B40000A4731205A31350A4D313036205332352B
:105B500035200A47302058302059300A4D3130392D
:105B600020523136302054300A4D3130370A00731C
:105B700070726561644379636C6500737465616C10
:105B8000746843686F700020647269766572206D76
:105B90006F64653A09007370726561644379636C80
:105BA0006500737465616C746843686F700020648D
:105BB0007269766572206D6F64653A090073707260
:105BC0006561644379636C6500737465616C7468C6
:105BD00043686F700020647269766572206D6F642F
:105BE000653A09007370726561644379636C65009E
:105BF000737465616C746843686F700020647269C7
:105C0000766572206D6F64653A090020686F6D6972
:105C10006E672073656E73697469766974793A206A
:105C20000020686F6D696E672073656E73697469B3
:105C3000766974793A200020737465616C746843E6
:105C4000686F70206D61782073706565643A20001C
:105C500020737465616C746843686F70206D61783F
:105C60002073706565643A200020737465616C74FC
:105C70006843686F70206D61782073706565643A61
:105C8000200020737465616C746843686F70206DC8
:105C900061782073706565643A20002070726577C2
:105CA00061726E20666C616720636C656172656409
:105CB0000A00207072657761726E20666C616720E1
:105CC000636C65617265640A002070726577617249
:105CD0006E20666C616720636C65617265640A00A2
:105CE000207072657761726E20666C616720636CEC
:105CF00065617265640A002074656D706572617417
:105D0000757265207072657761726E207472696752
:105D100067657265643A20002074656D7065726114
:105D200074757265207072657761726E2074726925
:105D30006767657265643A20002074656D706572EE
:105D40006174757265207072657761726E2074720D
:105D5000696767657265643A20002074656D7065D7
:105D6000726174757265207072657761726E2074ED
:105D700072696767657265643A20002064726976AB
:105D800065722063757272656E743A2000206472C9
:105D9000697665722063757272656E743A200020B0
:105DA0006472697665722063757272656E743A20EA
:105DB00000206472697665722063757272656E7414
:105DC0003A20004D6163726F20746F6F206C6F6EAC
:105DD000672E0A0020466C6F773A200020643A0054
:105DE00020693A0020703A00204500205A002059CE
:105DF00000204D393220580043290A0061626C6549
:105E00006420286D696E2074656D7020006469736C
:105E100000656E00436F6C6420657874727564650C
:105E2000732061726520002054002052004163639A
:105E3000656C65726174696F6E3A205000496E76C8
:105E4000616C69642065787472756465720A0020FB
:105E5000643A0020693A0020703A00536C6565701E
:105E60002E2E2E0047322F4733206261642070614E
:105E700072616D65746572730A0050726F6265209D
:105E80005A204F66667365743A2000446F6E652031
:105E9000736176696E672066696C652E0A005344EB
:105EA0002072656164206572726F720A00446F6EC1
:105EB00065207072696E74696E672066696C650A28
:105EC0000053544F505045442E20005072696E7458
:105ED00065722073746F70706564206475652074DA
:105EE0006F206572726F72732E2046697820746815
:105EF00065206572726F7220616E64207573652013
:105F00004D39393920746F20726573746172742E43
:105F1000202854656D7065726174757265206973AF
:105F20002072657365742E20536574206974206136
:105F3000667465722072657374617274696E672924
:105F40000A004E6F20436865636B73756D20776937
:105F50007468206C696E65206E756D6265722C20A8
:105F60004C617374204C696E653A20004E6F20437B
:105F70006865636B73756D2077697468206C696EF2
:105F800065206E756D6265722C204C617374204CB7
:105F9000696E653A2000636865636B73756D206D8B
:105FA00069736D617463682C204C617374204C6953
:105FB0006E653A20004C696E65204E756D626572A3
:105FC000206973206E6F74204C617374204C696E6D
:105FD00065204E756D6265722B312C204C61737497
:105FE000204C696E653A20004D31313000526573A6
:105FF000656E643A20002042002050006F6B002242
:106000000A00656E7175657565696E6720220050BE
:106010004944204175746F74756E65206661696CC2
:1060200065642120426164206578747275646572CC
:10603000206E756D6265720A0042656420636F6F41
:106040006C696E672E2E2E0042656420686561744F
:10605000696E672E2E2E006F6B0030780047323845
:10606000205A0A47302058383020593139302046DC
:10607000333030300A4D313137205072696E742020
:1060800061626F727465642E002020506C616E6EC8
:10609000657242756666657242797465733A20006E
:1060A0002046726565204D656D6F72793A20004318
:1060B0006F6D70696C65643A204D617920203620DF
:1060C000323031390A00207C20417574686F723A91
:1060D0002028416C657068204F626A656374732084
:1060E000496E632E2C204C756C7A426F7420476980
:1060F00074205265706F7369746F7279290A000099
:10610000204C61737420557064617465643A20009A
:10611000322E302E302E3131350A004D61726C69CD
:106120006E0020536F6674776172652052657365E7
:10613000740A00205761746368646F672052657346
:1061400065740A002042726F776E206F757420525A
:10615000657365740A002045787465726E616C2001
:1061600052657365740A00506F77657255700A0046
:1061700073746172740A004B494C4C45442E2000E4
:106180005072696E7465722068616C7465642E204B
:106190006B696C6C28292063616C6C6564210A0052
:1061A0004B494C4C20636175736564206279204BC8
:1061B000494C4C20627574746F6E2F70696E0A00C2
:1061C0004B494C4C2063617573656420627920747F
:1061D0006F6F206D75636820696E616374697665A1
:1061E0002074696D65202D2063757272656E742050
:1061F000636F6D6D616E643A20004D313034205311
:106200003137302054300A4D313137204C657665B6
:106210006C696E67205820417869730A4732380AE2
:10622000473020583136302046393939390A47301D
:10623000205A352046363030300A4739310A4D323F
:1062400031312053300A4D3430300A4D3930362048
:106250005A3630300A4730205A2D313520463530F5
:10626000300A4730205A3520463530300A47393019
:106270000A4D3430300A4D393036205A3936300A1A
:106280004D3231312053310A4732380A4D313137DE
:10629000204C6576656C696E6720646F6E652E0AAA
:1062A0004731320A4D31303920523136300A4D31C2
:1062B00031372050726F62696E67206265640070CA
:1062C000726F62655F7265776970650050726F62A8
:1062D000696E67206661696C6564004D31313720F5
:1062E000426564206C6576656C696E6720666169DD
:1062F0006C65642E0A4730205A31300A47302045F9
:10630000300A4D3330302050323520533838300A7F
:106310004D333030205035302053300A4D3330303B
:106320002050323520533838300A4D333030205029
:1063300035302053300A4D33303020503235205321
:106340003838300A47342053310070726F62655F0D
:106350006661696C65640050726F7465637465642E
:106360002050696E0A0025311D402924301C452724
:10637000232F1B0A0743222B1A42043803FF36043B
:1063800008060600010080537B94349EDCB8DBE6EF
:1063900042EDAE01AA01A801AC01549E11241FBE1A
:1063A000CFEFD1E2DEBFCDBF00E00CBF15E0A0E033
:1063B000B2E0E6EAFAE003E00BBF02C007900D92FC
:1063C000AC3BB107D9F72AE1ACEBB5E001C01D92B7
:1063D000A938B207E1F711E3CDECD1E300E006C044
:1063E00021970109802FFE010F940D7DC33CD10739
:1063F00080E00807A9F70E94CB460D9441850C94D4
:1064000000001F920F920FB60F9211242F933F930B
:106410008F939F93AF93BF938091BD059091BE05DD
:10642000A091BF05B091C0053091BC0523E0230FBA
:106430002D3720F40196A11DB11D05C026E8230FBC
:106440000296A11DB11D2093BC058093BD059093BC
:10645000BE05A093BF05B093C0058091C105909182
:10646000C205A091C305B091C4050196A11DB11D3F
:106470008093C1059093C205A093C305B093C40552
:10648000BF91AF919F918F913F912F910F900FBE30
:106490000F901F9018952FB7F8946091BD057091DB
:1064A000BE058091BF059091C0052FBF08953FB7ED
:1064B000F8948091C1059091C205A091C305B09157
:1064C000C40526B5A89B05C02F3F19F00196A11D54
:1064D000B11D3FBFBA2FA92F982F8827820F911D7A
:1064E000A11DB11DBC01CD0142E0660F771F881FC1
:1064F000991F4A95D1F708958F929F92AF92BF92BC
:10650000CF92DF92EF92FF926B017C01D0DF4B01C3
:106510005C01C114D104E104F104F1F091D3C7DFAF
:10652000DC01CB0188199909AA09BB09883E93406F
:10653000A105B10570F321E0C21AD108E108F10804
:1065400088EE880E83E0981EA11CB11CC114D104F2
:10655000E104F10421F7DDCFFF90EF90DF90CF90C1
:10656000BF90AF909F908F900895789484B582608B
:1065700084BD84B5816084BD85B5826085BD85B5E7
:10658000816085BDEEE6F0E0808181608083E1E896
:10659000F0E01082808182608083808181608083CE
:1065A000E0E8F0E0808181608083E1EBF0E08081D1
:1065B00084608083E0EBF0E0808181608083E1E9AA
:1065C000F0E0808182608083808181608083E0E967
:1065D000F0E0808181608083E1EAF0E08081826088
:1065E0008083808181608083E0EAF0E08081816047
:1065F0008083E1E2F1E0808182608083808181603C
:106600008083E0E2F1E0808181608083EAE7F0E06E
:1066100080818460808380818260808380818160CA
:1066200080838081806880831092C10008951F93C9
:10663000CF93DF93182FEB0161E016D1209711F46F
:1066400060E004C0CF3FD10531F461E0812FDF91DC
:10665000CF911F9145C1E12FF0E0E556FC4FE49149
:106660004E2F50E0FA013197E231F10508F09DC05C
:106670008827EE58FF4F8F4F0D940D7D84B58068AD
:1066800084BDC7BD97C084B5806284BDC8BD92C0BB
:1066900080918000806880938000D0938900C093AF
:1066A000880088C080918000806280938000D093B1
:1066B0008B00C0938A007EC08091800088608093A8
:1066C0008000D0938D00C0938C0074C08091B00086
:1066D00080688093B000C093B3006CC08091B0001C
:1066E00080628093B000C093B40064C08091900039
:1066F000806880939000D0939900C09398005AC00E
:1067000080919000806280939000D0939B00C09312
:106710009A0050C080919000886080939000D09340
:106720009D00C0939C0046C08091A000806880932B
:10673000A0008091A0008F7B8093A000D093A9003F
:10674000C093A80037C08091A00080628093A00011
:10675000D093AB00C093AA002DC08091A0008860A8
:106760008093A000D093AD00C093AC0023C0809173
:106770002001806880932001D0932901C0932801D3
:1067800019C080912001806280932001D0932B0159
:10679000C0932A010FC0809120018860809320015E
:1067A000D0932D01C0932C0105C0C038D1050CF049
:1067B0004CCF46CFDF91CF911F91089590E0FC011F
:1067C0003197E231F10508F04EC08827EC57FF4FB2
:1067D0008F4F0D940D7D809180008F7703C0809145
:1067E00080008F7D80938000089580918000877F56
:1067F000F9CF84B58F7702C084B58F7D84BD0895AD
:106800008091B0008F7703C08091B0008F7D80931E
:10681000B0000895809190008F7707C0809190001C
:106820008F7D03C080919000877F809390000895B2
:106830008091A0008F7707C08091A0008F7D03C05A
:106840008091A000877F8093A0000895809120010F
:106850008F7707C0809120018F7D03C08091200138
:10686000877F809320010895CF93DF9390E0FC0110
:10687000EF51FC4F2491FC01E95DFB4F849188238B
:1068800061F190E0880F991FFC01EF55FB4FC59116
:10689000D491FC01E957FB4FA591B491611109C056
:1068A0009FB7F8948881209582238883EC912E23CA
:1068B0000BC0623061F49FB7F8943881822F8095C5
:1068C00083238883EC912E2B2C939FBF06C08FB718
:1068D000F894E8812E2B28838FBFDF91CF91089504
:1068E0001F93CF93DF93282F30E0F901E556FC4F3B
:1068F0008491F901EF51FC4FD491F901E95DFB4F0F
:10690000C491CC23C1F0162F811158DFEC2FF0E099
:10691000EE0FFF1FE957FB4FA591B4918FB7F89485
:10692000111105C09C91ED2FE095E92302C0EC9177
:10693000ED2BEC938FBFDF91CF911F910895CF93F3
:10694000DF93282F30E0F901E556FC4F8491F901DF
:10695000EF51FC4FD491F901E95DFB4FC491CC2379
:1069600089F081112BDFEC2FF0E0EE0FFF1FE359D0
:10697000FB4FA591B491EC91ED2381E090E021F4DF
:1069800080E002C080E090E0DF91CF91089508950B
:106990001F920F920FB60F9211240BB60F922F93E6
:1069A0003F934F935F936F937F938F939F93AF9397
:1069B000BF93EF93FF93E0910802F09109021995BC
:1069C000FF91EF91BF91AF919F918F917F916F91C7
:1069D0005F914F913F912F910F900BBE0F900FBE83
:1069E0000F901F9018951F920F920FB60F921124BF
:1069F0000BB60F922F933F934F935F936F937F93B9
:106A00008F939F93AF93BF93EF93FF93E0910A020D
:106A1000F0910B021995FF91EF91BF91AF919F916A
:106A20008F917F916F915F914F913F912F910F9037
:106A30000BBE0F900FBE0F901F9018951F920F92D4
:106A40000FB60F9211240BB60F922F933F934F93D3
:106A50005F936F937F938F939F93AF93BF93EF93C6
:106A6000FF93E0910C02F0910D021995FF91EF91C7
:106A7000BF91AF919F918F917F916F915F914F9156
:106A80003F912F910F900BBE0F900FBE0F901F9054
:106A900018951F920F920FB60F9211240BB60F92FA
:106AA0002F933F934F935F936F937F938F939F9316
:106AB000AF93BF93EF93FF93E0910E02F0910F021B
:106AC0001995FF91EF91BF91AF919F918F917F9118
:106AD0006F915F914F913F912F910F900BBE0F904F
:106AE0000FBE0F901F9018951F920F920FB60F9226
:106AF00011240BB60F922F933F934F935F936F9395
:106B00007F938F939F93AF93BF93EF93FF93E09106
:106B10000402F09105021995FF91EF91BF91AF9199
:106B20009F918F917F916F915F914F913F912F91A5
:106B30000F900BBE0F900FBE0F901F9018951F92D5
:106B40000F920FB60F9211240BB60F922F933F9313
:106B50004F935F936F937F938F939F93AF93BF9365
:106B6000EF93FF93E0910602F09107021995FF91D0
:106B7000EF91BF91AF919F918F917F916F915F91B5
:106B80004F913F912F910F900BBE0F900FBE0F9022
:106B90001F9018951F920F920FB60F9211240BB6EB
:106BA0000F922F933F934F935F936F937F938F93A6
:106BB0009F93AF93BF93EF93FF93E0911002F091F7
:106BC00011021995FF91EF91BF91AF919F918F9114
:106BD0007F916F915F914F913F912F910F900BBEDD
:106BE0000F900FBE0F901F9018951F920F920FB627
:106BF0000F9211240BB60F922F933F934F935F93F5
:106C00006F937F938F939F93AF93BF93EF93FF9374
:106C1000E0911202F09113021995FF91EF91BF914B
:106C2000AF919F918F917F916F915F914F913F9124
:106C30002F910F900BBE0F900FBE0F901F901895C5
:106C400008951F93CF93DF93EC011D821C821F8256
:106C50001E82198681E0888782E28A871F861E86C7
:106C6000FE01B396CE01C1962FEF2193E817F907E5
:106C7000E1F711E018A3CE0113D61F8B188E198EE1
:106C800080E48A8F1B8E81E29AE39AAB89ABDF9115
:106C9000CF911F910895DB01ED91FC911994EF9232
:106CA000FF921F93CF93DF931F921F92CDB7DEB752
:106CB0007C01DC01D196ED91FC91D29782E0698351
:106CC0007A83199520E030E04AE069817A81C70132
:106CD000E2DF182FD701D196ED91FC91D29783E096
:106CE0001995D701D196ED91FC91D29780E0199535
:106CF000812F0F900F90DF91CF911F91FF90EF9018
:106D000008950F931F93CF93DF93EC018B01E9A9B3
:106D1000FAA982E01995E9A9FAA981E0199520E07C
:106D200030E044E1B801CE01B6DF9E012D5C3F4F5B
:106D300047E1B801CE01AFDFE9A9FAA980E0DF9110
:106D4000CF911F910F911994EF92FF921F93CF93C0
:106D5000DF93EC017B01E9A9FAA982E01995E9A981
:106D6000FAA981E0199520E030E045E1B701CE01B4
:106D700092DF182F882339F09E012D5C3F4F47E1A9
:106D8000B701CE0188DFE9A9FAA980E01995812F22
:106D9000DF91CF911F91FF90EF900895CF93DF93F4
:106DA0001F92CDB7DEB79E012F5F3F4F46E473DFE2
:106DB00089810F90DF91CF910895CF93DF931F9238
:106DC000CDB7DEB79E012F5F3F4F47E464DF898177
:106DD0000F90DF91CF91089520E030E048E45BCF41
:106DE000CF93DF93EC016A817B81D8DF88836A814E
:106DF0007B81CE01E2DF89836A817B81CE01ECDF7A
:106E00008B879E012D5C3F4F6A817B8147E1CE01DC
:106E1000DF91CF9140CFCF93DF93EC016A817B81EB
:106E20003EDF882319F0CE01DBDF81E0DF91CF91D7
:106E300008958F929F92AF92BF92CF92EF920F934D
:106E4000CF93DF931F921F92CDB7DEB74C015B014A
:106E50002A834983F6DEF401B382A282498147A3E3
:106E60002A8120A705A3E4A2C3A2C4010F900F901A
:106E7000DF91CF910F91EF90CF90BF90AF909F9007
:106E80008F90C9CFFC01628173813BCFCF93DF9399
:106E9000EC01EE85FF85309709F019956A817B81B9
:106EA000CE01DF91CF9150CF0F93FC01828193816E
:106EB000648F458F278F068F9F01245E3F4F4BE3E2
:106EC000BC01CF010F91E7CEFC0160A30895BF92F2
:106ED000CF92DF92EF92FF920F931F93CF93DF93A6
:106EE0006C01D62FB42EC22F7801CC2369F0F701A4
:106EF000049120E04B2D6D2FC601D6DFFFEFEF1A76
:106F0000FF0AC150D85FF1CFDF91CF911F910F9150
:106F1000FF90EF90DF90CF90BF9008958F929F9257
:106F2000AF92BF92CF92DF92EF92FF920F931F9397
:106F3000CF93DF935C01C62EC42FD22ED02F220F09
:106F4000220F220F1ED0882379F0DC0F8D2C912C7C
:106F5000CD1751F087012D2D4C2F6C2DC501B7DFBA
:106F6000E80CF91CCF5FF4CFDF91CF911F910F9107
:106F7000FF90EF90DF90CF90BF90AF909F908F9059
:106F800008950F93FC010150040F84A996A994174A
:106F900018F0081728F402C0081750F0041740F43E
:106FA0002150260F83A995A9961720F4281720F4BD
:106FB00080E007C0281720F481E0261710F0F8CFF2
:106FC00081E00F91089581E008952EE93FE0009758
:106FD00029F0F9013197F1F70197F9CF0895FC01F4
:106FE000128280818150838314820895FC01808104
:106FF0009281980F92832181921760F494819F5F10
:1070000094839381890F821710F08FEF820F83830F
:1070100081E0089580E00895FC0191E08381861766
:1070200008F490E031E0461708F030E0832F892B18
:1070300021E05281451708F420E02823832F89237B
:10704000822B0895DC01FB01108212968C9112971D
:10705000818315968C9115978150828313968C911C
:1070600083830895FB0141812381213029F023305E
:1070700031F468EF640F04C0642F485F01C0642FCF
:10708000CBCFDC0115962C9115971696ED91FC91BE
:107090001797CF01820F911D820F911D1192E81752
:1070A000F907E1F70895FC01A681B7818281481BA9
:1070B0008581483018F0A80FB11D4770382F3695DC
:1070C00036953695562F577080E890E002C095951A
:1070D00087955A95E2F7439F402D11246695669552
:1070E0006695E62FF0E0E40FF11DEA0FFB1F3081FB
:1070F000222311F0832B02C080958323808308957F
:10710000FB014181DC0112962C911297421760F02D
:1071100013962C911397241738F0608115962C91B3
:10712000621710F42481BFCF0895CF92DF92FF92AF
:107130000F931F93CF93DF936C01EB01FA809B8138
:10714000913051F030F0923049F0933051F41FEF0C
:1071500009C010E001E007C011E004C010E00FEF2B
:1071600002C010E000E0F7FE03C0BE01C601C8DFA8
:107170009881900F98839981910F9983FF0C99F7CB
:10718000DF91CF911F910F91FF90DF90CF900895E5
:107190000F931F93CF93DF938901FB01C281D381AA
:1071A0004233D9F058F44531E1F0473109F1443127
:1071B00041F5CE0166DFCE0112DF23C04634E1F097
:1071C0004734E1F04B33E9F4B901CE014BDF8823BA
:1071D000C1F0B801CE01A9DF14C0B901CE0190DF22
:1071E00010C0CE0103DF882369F0CE014ADF09C059
:1071F000B901CE0127DF05C08D8101C08981F80169
:10720000808381E0DF91CF911F910F910895CF92FC
:10721000DF92EF92FF920F931F93CF93DF937C0146
:10722000D62FD42EC22F122FC62EC20E6C2D611B4C
:10723000183038F00FEF20E04D2DC70135DE185023
:10724000F5CF6C2F687F6D0F2C2F277071F097E0B2
:1072500029272F5F27700FEF10E001C0000F2A953C
:10726000EAF720E04D2DC7011FDEDF91CF911F917E
:107270000F91FF90EF90DF90CF900895CF92DF9223
:10728000EF92FF920F931F93CF93DF937C01D62E43
:10729000D42FC22F122FC42EC20E4C2D411B1830DA
:1072A00038F00FEF21E06D2DC701FEDD1850F5CF4E
:1072B0004C2F487F4D0F2C2F277071F097E0292716
:1072C0002F5F27700FEF10E001C0000F2A95EAF73B
:1072D00021E06D2DC701E8DDDF91CF911F910F9166
:1072E000FF90EF90DF90CF900895EF92FF920F9371
:1072F0001F93CF93DF93EC01162FF42EE22E01E0C3
:1073000040DE882359F02E2D4F2D612FCE01DF91C5
:10731000CF911F910F91FF90EF9079CFDF91CF9197
:107320001F910F91FF90EF900895EF92FF920F93AE
:107330001F93CF93DF93EC01162FF42EE22E022F32
:1073400021E01FDE882359F02E2D4F2D612FCE0115
:10735000DF91CF911F910F91FF90EF908FCFDF9131
:10736000CF911F910F91FF90EF900895DF92EF92D0
:10737000FF920F931F93CF93DF937C01162FC42F9F
:10738000D22ED02FFEDD8823F9F02D2D4C2F612F2A
:10739000C7013DDF2D2F4C2F612FC7016FDF6FEF2E
:1073A0006D0D610F2D2F4C2FC70168DF4FEF4D0F73
:1073B0004C0F2D2D612FC701DF91CF911F910F91A0
:1073C000FF90EF90DF9023CFDF91CF911F910F912E
:1073D000FF90EF90DF900895EF92FF920F931F932D
:1073E000CF93DF937C01D62F122FC42F040F212FB0
:1073F0004C2F6D2FC7010BDFCF5F0C13F8CFDF9140
:10740000CF911F910F91FF90EF900895DF92EF922F
:10741000FF920F931F93CF93DF93EC01162FF42E5F
:10742000E22EAFDD882329F02E2D4F2D612FCE01C6
:10743000D3DFDF91CF911F910F91FF90EF90DF90FD
:1074400008950895FC01E60FF11D849190E0982FB6
:1074500088273196E4918E0F911D0895FC01849147
:107460000895FCDF882321F0823011F083E0089535
:1074700086E0089580E00895FC018081089566E02B
:10748000E1CF68E0DFCF0A96FC01849108950B9666
:10749000FC0184910895DC011496ED91FC911597FF
:1074A000319684910895BF92CF92DF92EF92FF922E
:1074B0000F931F93CF93DF938C01E62EDC0114967C
:1074C000CD91DC911597CE01C9DFF82EF8018481AA
:1074D0009581C7DFC82EF1E0FF1203C02FE0B22E66
:1074E00002C0BB24BA94D80114968D919C91159733
:1074F000CADFF82EF80184819581C9DFD82ED80122
:1075000014968D919C911597BCDFB0E6BE1538F4AA
:10751000009729F0C80FD91F91E6F92E0FC0F80186
:1075200084819581ACDFF0E4FE1538F4009729F0F2
:10753000C80FD91F81E4F82E01C06196DE1490F4C3
:10754000D80150961C92509753961C92539754967C
:107550001C92549751961C92519752961C9280E01F
:1075600090E066C0DF1460F38C2D90E0FE01249162
:107570002F3F11F4219657C0FE104CC0D80114962D
:107580008D919C9115976ADF9E012F5F3F4FFE0101
:10759000882311F08230E1F48491D80153968C93C2
:1075A0005397F901249154962C935497FE013396E6
:1075B000E4915096EC935097FE013496E4915196E5
:1075C000EC935197FE013596E4915296EC9320C0CE
:1075D0008491982F9F709250D80152969C93529705
:1075E00082958F7051968C935197F9012491822F37
:1075F0008F7054968C93549722952F7053962C939A
:107600005397FE013296E491E295EF705096EC9319
:10761000CE010EC0FE013296E491EB219C012E0FAB
:10762000311DC20FD31FFD1409F48ACFF3949ECFEE
:10763000DF91CF911F910F91FF90EF90DF90CF904E
:10764000BF9008954F925F926F927F929F92AF92F8
:10765000BF92CF92DF92EF92FF920F931F93CF933F
:10766000DF931F92CDB7DEB72C01C62E942E622F6A
:107670001ADF7C01892B09F43AC0F20184819581DB
:10768000F0DEB82EF201138904898189C80E82893F
:10769000981AD92CD01A212F4D2D6C2DC20171DCD6
:1076A000882311F1EB0CF11C195F169516951695B0
:1076B000612E712CD914C1F03C2D57018A2D8E19E1
:1076C000811770F4F501049120E04D2D632FC20164
:1076D0003983EADBFFEFAF1ABF0A3981385FEECF9B
:1076E000E60CF71CD394E6CFF201808901C080E05C
:1076F0000F90DF91CF911F910F91FF90EF90DF904E
:10770000CF90BF90AF909F907F906F905F904F9081
:1077100008950F931F93CF93DF9300D0CDB7DEB7BB
:107720008C01DC015596ED91FC9156972B834A8391
:10773000698319954A81480F2B816981C8010F908F
:107740000F900F90DF91CF911F910F917BCFAF9250
:10775000BF92DF92EF92FF920F931F93CF93DF932D
:107760001F921F92CDB7DEB77C01D62E042FDC010D
:107770005596ED91FC91569729833A831995080FF8
:107780002981A22E3A81B32E10E0F50121915F01EB
:10779000222339F0402F6D2DC70154DFD80E180F6A
:1077A000F4CF812F0F900F90DF91CF911F910F9108
:1077B000FF90EF90DF90BF90AF900895DF92EF922F
:1077C000FF920F931F93CF93DF937C01D62FD42E7C
:1077D0008901DC015596ED91FC9156971995D80ECB
:1077E000C0E0F8012491222349F04D2D6D2FC701EF
:1077F00029DFD80FC80F0F5F1F4FF3CF8C2FDF91FA
:10780000CF911F910F91FF90EF90DF900895DC01D1
:1078100014962D913C9115972115310509F43FC01F
:1078200057968C915797F901811108C03596E491CC
:107830005896EC935897F9013C9611C0813041F469
:107840003F96E4915896EC935897F901709607C0CB
:107850003D96E4915896EC935897F9013E96E49141
:107860005996EC93599758968C915897082E000C7E
:10787000990B59962C915997821B910927FD939545
:107880005A962C915A97203441F0829FC0011124BE
:1078900026E0969587952A95E1F75B968C93089557
:1078A0002AE33AE3FC01368B258B0895CF92DF92D1
:1078B000EF92FF920F931F93CF93DF938C017B0185
:1078C0006A01CB01FA011995D82F882311F1682F8D
:1078D000C801E9DDF801C189C195FFEFEF1AFF0A80
:1078E000C701F6011995F801882351F08089C80F66
:1078F000C701F6011995D82F682FC801D4DDEDCF47
:10790000D03221F091898389890F01C080898C0F41
:1079100001C080E0DF91CF911F910F91FF90EF9018
:10792000DF90CF9008954CE35AE3C0CFCF93DF931D
:10793000FC01248135812617370741F0EC0175835E
:10794000648365DF8AE39AE39E8B8D8BDF91CF9111
:107950000895CF93DF9300D01F92CDB7DEB76115A6
:1079600071058105910579F09B01AC0169833A832A
:107970004B835C830F947D7D29813A814B815C81AF
:107980000F94F17C03C060E070E0CB010F900F908A
:107990000F900F90DF91CF910895CF92DF92EF92E9
:1079A000FF920F931F9362177307840795077CF468
:1079B00089019A016B017C01C901B8016C197D092B
:1079C0008E099F09C6DF6C0D7D1D8E1D9F1D1F91A9
:1079D0000F91FF90EF90DF90CF9008954F925F92BC
:1079E0006F927F92AF92BF92CF92DF92EF92FF920F
:1079F0000F931F93CF93DF93CDB7DEB729013A01E1
:107A00009B01AC0124193509460957098A899B89CC
:107A1000AC89BD89BC01CD016A197B098C099D091E
:107A20000F948D7CA801970124193509460957093F
:107A30000F94F17CCA01B9016A0D7B1D8C1D9D1D3F
:107A4000DF91CF911F910F91FF90EF90DF90CF903A
:107A5000BF90AF907F906F905F904F90089580E0BF
:107A600090E008950895CF92DF92EF92FF920F93E6
:107A70001F93CF93DF936C017A018B01C0E0D0E0BC
:107A8000CE15DF0589F0D8016D918D01D601ED91FC
:107A9000FC910190F081E02DC6011995892B11F41C
:107AA0007E0102C02196ECCFC701DF91CF911F91DB
:107AB0000F91FF90EF90DF90CF90089561157105C1
:107AC00079F0FB0101900020E9F73197AF01461BE7
:107AD000570BDC01ED91FC910280F381E02D1994AC
:107AE00080E090E00895DC01ED91FC910190F0813F
:107AF000E02D19944F925F926F927F92EF92FF92D6
:107B00000F931F93CF93DF93CDB7DEB7A1970FB637
:107B1000F894DEBF0FBECDBF7C01FA01CB0119A2E4
:107B2000223008F42AE08E010F5D1F4F422E512CA7
:107B3000612C712CBF01A30192010F94CF7CF9013C
:107B4000CA01015011096A3014F4605D01C0695C1A
:107B5000D8016C93232B242B252B61F7B801C70187
:107B6000ADDFA1960FB6F894DEBF0FBECDBFDF919B
:107B7000CF911F910F91FF90EF907F906F905F904A
:107B80004F900895CF92DF92EF92FF920F931F9341
:107B9000CF93DF93EC016A017B012115310579F464
:107BA000E881F9810190F081E02D642FDF91CF9180
:107BB0001F910F91FF90EF90DF90CF9019942A3092
:107BC0003105D9F477FF18C06DE28DDF8C014427B1
:107BD0005527BA014C195D096E097F092AE0CE01CB
:107BE00089DF800F911FDF91CF911F910F91FF903F
:107BF000EF90DF90CF9008952AE0B701A601CE0163
:107C0000DF91CF911F910F91FF90EF90DF90CF9078
:107C100071CF9A01AB01770F660B770BB3CFCF9380
:107C2000CFB7F8948091C805811127C0ECE5F4E046
:107C30008491E6E1F4E09491E82FF0E0EE0FFF1F6D
:107C4000EF55FB4FA591B491EC91E92321F461E04C
:107C500085E30E94703461E085E30E9434348CB582
:107C600080618CBD8CB580648CBD61E084E30E9432
:107C7000343461E083E30E9434348091C8058F5F1F
:107C80008093C805CFBFCF910895CF92EF920F9305
:107C9000FC0113AE14AE15AE0496CBD80F91EF9045
:107CA000CF900895CF92DF92EF92FF921F93CF93E0
:107CB000DF93EC0180E090E00F94257A25ED34E02D
:107CC00045E352E40F94C37B20E030E04AE754E4FC
:107CD0000F948C796B017C012AE037ED43EA5CE379
:107CE00069857A858B859C850F94AC789B01AC0166
:107CF000C701B6010F94C37B26E636E646EA5EE38B
:107D00000F948C7920E030E040E85FE30F94AB788B
:107D10000F94F979162FE881F9810480F581E02D1F
:107D2000603118F561E0CE0119952AE037ED43EA9C
:107D30005CE369857A858B859C850F94AC789B0183
:107D4000AC01C701B6010F94C37B2CEE31E548E3CB
:107D50005EE30F948C7920E030E040E85FE30F941D
:107D6000AB780F94F979162F03C060E0CE01199516
:107D7000612FCE01C6D2612F70E080E090E00F94B9
:107D8000277A2D853E854F8558890F94C37B0F94A4
:107D9000F979CE01DF91CF911F91FF90EF90DF90A5
:107DA000CF9092C2FC01258736874787508B7ACFC8
:107DB000CF92DF92EF92FF92CF93DF93EC01DED26E
:107DC000682F70E06F5F7F4F072E000C880B990BB8
:107DD0000F94277A20E030E040E05DE30F94C37B0E
:107DE0006B017C01E881F9810680F781E02DCE01ED
:107DF0001995811105C026E636E646EA5EE304C021
:107E00002CEE31E548E35EE3C701B6010F94C37B76
:107E10006B017C012AE037ED43EA5CE369857A85F2
:107E20008B859C850F94AC789B01AC01C701B60192
:107E30000F948C7925ED34E045EB5FE30F948C795A
:107E400020E030E04AE754E40F94C37B0F94F979C3
:107E5000CB01DF91CF91FF90EF90DF90CF9008950D
:107E6000DC01ED91FC910084F185E02D19956115FF
:107E700071058105910539F06F3F7F4F8F4F9F4FFF
:107E800021F080E0089582E0089581E00895DC010A
:107E9000ED91FC910484F585E02D199583500895AA
:107EA000DC01ED91FC910088F189E02D19958F5F3F
:107EB00008956031710509F441C088F4623071059C
:107EC00009F454C020F4672B09F458C008956430B5
:107ED000710509F443C068307105C1F1089560343B
:107EE0007105E1F020F46032710501F10895603808
:107EF000710561F06115714009F048C0DC01ED9138
:107F0000FC910288F389E02D60E03FC0DC01ED9137
:107F1000FC910288F389E02D61E037C0DC01ED912E
:107F2000FC910288F389E02D62E02FC0DC01ED9125
:107F3000FC910288F389E02D63E027C0DC01ED911C
:107F4000FC910288F389E02D64E01FC0DC01ED9113
:107F5000FC910288F389E02D65E017C0DC01ED910A
:107F6000FC910288F389E02D66E00FC0DC01ED9101
:107F7000FC910288F389E02D67E007C0DC01ED91F8
:107F8000FC910288F389E02D68E019940895DC01E2
:107F9000ED91FC910488F589E02D1995893048F41C
:107FA000E82FF0E0EE0FFF1FE85EFC4F808191812B
:107FB000089580E090E00895DC01ED91FC91008C43
:107FC000F18DE02D1995843030F4E82FF0E0EC5E6F
:107FD000FC4F8081089580E00895DC01ED91FC91D3
:107FE0000280F381E02D61E01995862F0895FC0150
:107FF00085810895DC0115966C931597ED91FC91A0
:10800000262F30E040E050E00190F081E02D61E16A
:108010001994DC01ED91FC910280F381E02D62E185
:108020001994FC01268137818085482F4F70842F59
:10803000B90190E00895DC019A01462F4F70169621
:108040002C93169717963C931797942F9F7018961A
:108050008C911897807F892B18968C931897ED91A7
:10806000FC91119750E00190F081E02D63E1CD018A
:108070001994FC0167A170A592A581A5917008953E
:10808000DC0197964C93979798965C93989799965E
:108090006C9399979A968C919A9770FB80F99A961F
:1080A0008C939A97ED91FC9111979A01AB015170C5
:1080B0000190F081E02D6DE6CD011994DC016F7027
:1080C00097962C919797207F262B97962C9397978E
:1080D000ED91FC91119798963C91989799964C91B7
:1080E00099979A965C9151700190F081E02D6DE620
:1080F0001994DC016F7098963C919897307F362BDD
:1081000098963C939897ED91FC91119797962C91A6
:10811000979799964C9199979A965C915170019086
:10812000F081E02D6DE61994DC016F7799964C9102
:1081300099974078462B99964C939997ED91FC919D
:10814000119797962C91979798963C9198979A9615
:108150005C9151700190F081E02D6DE61994FC0165
:1081600091A5990F9595292F092E000C330B20749A
:108170003327220F331F892F8F77822B0895DC013D
:10818000ED91FC910280F381E02D6FE61994DC0102
:10819000ED91FC910084F185E02D1995CB01937050
:1081A0000895DC01ED91FC910084F185E02D199595
:1081B00077FB882780F90895DC01ED91FC9100841C
:1081C000F185E02D19958F710895DC01ED91FC91F9
:1081D0000084F185E02D1995892F81700895DC01C7
:1081E000ED91FC910084F185E02D199591FB882794
:1081F00080F90895DC01ED91FC910084F185E02D7A
:10820000199592FB882780F90895DC01ED91FC9186
:108210000084F185E02D199593FB882780F9089556
:10822000DC01ED91FC910084F185E02D199594FB22
:10823000882780F90895DC01ED91FC910084F18597
:10824000E02D199595FB882780F90895DC01ED91C3
:10825000FC910084F185E02D199596FB882780F923
:108260000895DC01ED91FC910084F185E02D1995D4
:1082700097FB882780F90895FC012281338184814E
:10828000482F4F70842FB90190E00895DC019A01C6
:10829000462F4F7012962C93129713963C93139778
:1082A000942F9F7014968C911497807F892B14962D
:1082B0008C931497ED91FC91119750E00190F0810F
:1082C000E02D60E1CD011994DC016F7112968C9163
:1082D0001297807E682B12966C931297ED91FC9109
:1082E0001197262F13963C91139714968C911497FF
:1082F000482F4F7050E00190F081E02D60E1CD01FA
:108300001994DC016F7113968C911397807E682B02
:1083100013966C931397ED91FC91119712962C91F3
:108320001297362F14968C911497482F4F7050E067
:108330000190F081E02D60E1CD011994DC016F70B6
:1083400014968C911497807F682B14966C931497D5
:10835000ED91FC91119712962C91129713963C91E6
:108360001397462F4F7050E00190F081E02D60E1AF
:10837000CD011994FC0182818F710895FC018381E4
:108380008F710895DC016770962F9295907F929679
:108390006C9192976F78692B92966C939297ED916E
:1083A000FC91119792962D913D914D915C919597ED
:1083B0000190F081E02D6CE6CD011994DC019296DC
:1083C0008C91929760FB87F992968C939297669521
:1083D000677093968C919397887F682B93966C9394
:1083E0009397ED91FC91119792962D913D914D911E
:1083F0005C9195970190F081E02D6CE6CD01199488
:10840000DC0193968C91939760FB87F993968C93FC
:10841000939761FB882780F994966C9194976E7F6F
:10842000682B94966C939497ED91FC91119792968A
:108430002D913D914D915C9195970190F081E02DAA
:108440006CE6CD011994DC0194962C91949760FB15
:1084500021F994962C939497ED91FC911197929613
:108460002D913D914D915C9195970190F081E02D7A
:108470006CE619946F70DC0195962C919597207F8E
:10848000622B95966C939597ED91FC91119792962E
:108490002D913D914D915C9195970190F081E02D4A
:1084A0006CE61994CF93DF93EC01E881F9810280A7
:1084B000F381E02D6CE619956AA37BA38CA39DA3A1
:1084C000DF91CF910895CF93DF93EC01EBDF8AA189
:1084D00082958770DF91CF910895CF93DF93EC0160
:1084E000E1DF9AA1991F9927991F8BA18770880FA7
:1084F000892BDF91CF910895CF93DF93EC01D2DFE9
:108500009BA1991F9927991F8CA18170880F892B96
:10851000DF91CF910895CF93DF93EC01C3DF8CA15E
:1085200086958170DF91CF910895CF93DF93EC0111
:10853000B9DF8DA18F70DF91CF910895DC01929604
:108540004D935D936D937C939597ED91FC91019084
:10855000F081E02D9A01AB016CE619946F70DC019B
:1085600092962C919297207F622B92966C93929781
:10857000ED91FC91119792962D913D914D915C91C9
:1085800095970190F081E02D6CE61994CF93DF93DD
:10859000EC0188DF8AA18F70DF91CF910895CF928F
:1085A000DF92EF92CF93DF93EC01E881F9810280B3
:1085B000F381E02D60E019956B01E82E23E0E222C3
:1085C000CA8ADB8A2E2D23709C899C7F922B9C8BE0
:1085D0008E2DB60190E0DF91CF91EF90DF90CF909C
:1085E0000895DC019A01462F437052962C935297BE
:1085F00053963C935397942F937054968C91549721
:108600008C7F892B54968C935497ED91FC91119704
:1086100050E00190F081E02D60E0CD011994DC0183
:1086200052968C91529760FB82F952968C93529796
:10863000ED91FC911197282F53963C9153975496A6
:108640008C915497482F437050E00190F081E02DB9
:1086500060E0CD011994DC0152968C91529760FB39
:1086600084F952968C935297ED91FC911197282F93
:1086700053963C91539754968C915497482F43703E
:1086800050E00190F081E02D60E0CD011994DC0113
:1086900053968C91539760FB80F953968C93539724
:1086A000ED91FC91119752962C915297382F549638
:1086B0008C915497482F437050E00190F081E02D49
:1086C00060E0CD011994CF93DF93EC0168DF8A89D4
:1086D00082FB882780F9DF91CF910895FC0123A5C3
:1086E00034A585A5482F4F73842FB90190E00895D4
:1086F000DC019A01462F4F739B962C939B979C9677
:108700003C939C97942F9F739D968C919D97807C12
:10871000892B9D968C939D97ED91FC91119750E03C
:108720000190F081E02D60E7CD011994CF93DF93A4
:10873000EC0161E088810E94343461E08C810E9408
:10874000343462E08A810E943434E881F981EF5147
:10875000FC4FE491EE83EA81FB81EF51FC4FE49101
:10876000EF83EC81FD81EF51FC4FE491E887DF91CD
:10877000CF9108959F92AF92BF92CF92DF92EF92E6
:10878000FF920F931F93CF93DF938C01942E87E07A
:10879000C82ED12CE12CF12CC0E0A62EB12CC501A5
:1087A000911019C00E2C02C0959587950A94E2F796
:1087B00080FF02C061E001C060E0F80180810E949A
:1087C000703461E0F80184810E947034F801828184
:1087D000911016C007C00C2C02C0959587950A947D
:1087E000E2F7E6CF0E949F3421E030E0892B11F4BC
:1087F00020E030E00E2C01C0220F0A94EAF70DC0F1
:108800000E949F3421E030E0892B11F420E030E019
:108810000C2C01C0220F0A94EAF7C22B60E0F80189
:1088200084810E947034FFEFEF1AFF0A81E0C81ABA
:10883000D108E8E0EE16F10409F0B1CF8C2FDF91FA
:10884000CF911F910F91FF90EF90DF90CF90BF904D
:10885000AF909F9008950F931F93CF93DF938C0158
:10886000D62F672F41E086DFC82F41E06D2FC8016A
:1088700081DF2C2F30E0322F2227A901482BCA019B
:10888000DF91CF911F910F9108950F93FC0130E07C
:1088900080E092E1AAE7B0E0481759076A077B0732
:1088A00040F4B695A795979587953F5F3630A1F729
:1088B00037E091E09327222311F020E501C020E763
:1088C000892F86950C70082B022B00839170918361
:1088D0000F9108952091C705222399F04FB7F8947E
:1088E0002091C705213059F42DB32093C5053DB320
:1088F0002091C605209523232DBB4FBF02C0409376
:10890000C5058CBD9DBD08958EBD00000DB407FE4C
:10891000FDCF8EB508950CB405FC0DC09EBD0000C2
:108920000DB407FEFDCF9EB58EBD00000DB407FE51
:10893000FDCF8EB508958EBD00000DB407FEFDCFAE
:108940008EB59EBD00000DB407FEFDCF9EB5089507
:108950008091C705882361F09FB7F8942091C705DF
:108960008091C505213019F48DBB9FBF08958FBF3D
:108970000895CF93DF93FC01128213828481807F5C
:1089800084831582168217828085807F8087218765
:1089900032874387548780E090E0A0E0BFE385877B
:1089A0009687A787B08B8EE293E091838083128AAB
:1089B000138A84898C7F848B158A168A8789807FA5
:1089C000878B108E118E828D807F828F138E148EF6
:1089D000158E868D8E7F868F178E10A281A180784E
:1089E00081A3DF01929685E0ED0119928A95E9F75E
:1089F00017A210A611A682A58E7F82A713A614A681
:108A000085A5807C85A786A58C7F86A770AB67A788
:108A100012AA11AADF91CF910895FC0187A50C94A9
:108A20007034AF92BF92CF92DF92EF92FF920F938A
:108A3000CF93DF931F921F92CDB7DEB75C01F62E66
:108A4000FC0181A992A9892B09F44EC060E0C501FF
:108A5000E4DF41E06F2DF50181A992A98BDE60E092
:108A600070E0F50181A992A9F6DE60E070E0F50101
:108A700081A992A9F0DE61E0C501CFDF60E0C50108
:108A8000CCDF41E06F2DF50181A992A973DEF501DC
:108A9000818B41E060E081A992A96CDEC82ED12CC7
:108AA000E12CF12CFE2CED2CDC2CCC2441E060E000
:108AB000F50181A992A95EDEC82AFE2CED2CDC2CE2
:108AC000CC2441E060E0F50181A992A953DEC82AD7
:108AD000FE2CED2CDC2CCC2441E060E0F50181A9DA
:108AE00092A948DEC82A41C0409114025091150253
:108AF00060911602709117020CE021E0CE01019600
:108B0000C4DE89819A81E6DE60E0C50186DF8F2DB3
:108B1000FBDE80E090E0FFDE80E090E0FCDE61E0E4
:108B2000C5017BDF60E0C50178DF8F2DEDDEF5014B
:108B3000818B80E0E9DEC82ED12CE12CF12CFE2CBB
:108B4000ED2CDC2CCC2480E0DFDEC82AFE2CED2CC2
:108B5000DC2CCC2480E0D8DEC82AFE2CED2CDC2CCA
:108B6000CC2480E0D1DEC82AF3DE61E0C50155DF08
:108B7000C701B6010F900F90DF91CF910F91FF9039
:108B8000EF90DF90CF90BF90AF9008954F925F929B
:108B90006F927F928F929F92AF92BF92EF92FF92CD
:108BA0000F931F93CF93DF931F921F92CDB7DEB722
:108BB0007C0149015A01162F1068FC0181A992A974
:108BC000250166247724892BA9F060E0C70125DF01
:108BD00041E0612FF70181A992A9CCDDF701818BDA
:108BE000B20181A992A937DEB401F70181A992A946
:108BF00032DE1CC0409114025091150260911602A1
:108C0000709117020CE021E0CE0101963EDE8981D1
:108C10009A8160DE60E0C70100DF812F75DEF70119
:108C2000818BC20178DEC40176DE92DE61E0C7018D
:108C3000F4DE0F900F90DF91CF911F910F91FF9075
:108C4000EF90BF90AF909F908F907F906F905F90CC
:108C50004F900895CF93DF93EC0161E08FA50E94C0
:108C6000343461E0CE01D9DE89A99AA9009709F0D0
:108C70005DDD8A899B892C89A22FA370AC016A2FA4
:108C800070E0CE01AEDC4AA15BA16CA17DA1CE015A
:108C900055DC4FA158A569A57AA57170CE01F0D910
:108CA0008BA59CA52DA5A22FAF73AC016A2F70E0F8
:108CB000CE011EDD8A819B812C81A22FAF70AC0179
:108CC0006A2F70E0CE01E2DA68E0CE0147DCE8818D
:108CD000F9810688F789E02D61E0CE01DF91CF911F
:108CE0001994DC01ED91FC910280F381E02D64E0A8
:108CF0001994F7DF64FB882780F90895CF93DF93F9
:108D0000EC01F7DF811105C0CE0140DC91E081115B
:108D100001C090E0892FDF91CF910895FC01258952
:108D200036898789482F4F70842FB90190E00895C4
:108D3000DC019A01462F4F7055962C935597569605
:108D40003C935697942F9F7057968C915797807F9E
:108D5000892B57968C935797ED91FC91119750E082
:108D60000190F081E02D64E1CD011994FC01208D8A
:108D7000318D828D482F4F70842FB90190E0089576
:108D8000DC01ED91FC910280F381E02D61E7199502
:108D9000862F089508950E94B532FCDF0F94EE7778
:108DA000C0E0D0E00F9480782097E1F30E940000AB
:108DB000F9CF0E94868F4091490E90913A022091FE
:108DC000520E3091530E6091660270916702262711
:108DD000372760912E0E70912F0E26273727949FEC
:108DE000A0011124440F452F441F550B51952427F2
:108DF0003527A9014827CA012091CE053091CF051A
:108E00002817390731F09093CF058093CE0581E084
:108E1000089580E00895E4E7F8E080E091919923D7
:108E200011F08927FBCF9091D00591110BC091E0F3
:108E30002091CD05281301C090E09093CC0591E0DE
:108E40009093D0059091CC0591118093CD0581E050
:108E5000911101C080E008950E94868F982F81E0D3
:108E60002091CB05291302C080E008959093CB0593
:108E700008955D9A88E28A950000E9F78091D80507
:108E80008E7F8093D80508955D988091D8058E7F58
:108E90008093D805089588EF0E94A35388E28A95AD
:108EA0000000E9F708958AEF0E94A35388E28A95AB
:108EB0000000E9F708958091D805982F93709130BC
:108EC00029F081608D7F8093D805EDCF0895CF93F1
:108ED000C82F807F0E94A3538C2F8295807F0E9491
:108EE000A35388E28A950000E9F7CF910895CF93C4
:108EF000DF931F92CDB7DEB79091D805292F23704D
:108F0000233039F0916092609093D8058983C3DF54
:108F100089810F90DF91CF91DACF1F93CF93DF93A9
:108F20001F92CDB7DEB7182F811102C080E201C0B9
:108F300084E2611102C090E001C092E0892B698354
:108F4000D6DF9091D80510FB92F9892F698160FBDB
:108F500083F98093D8050F90DF91CF911F910895E9
:108F60006091D80562FB992790F9891721F063FB7E
:108F7000662760F9D2CF0895CF93C82F81E0F0DF44
:108F8000C11102C082E201C083E2B1DF9091D80535
:108F9000C0FB94F99093D805CF9108959091D8058E
:108FA000929591708913E8CF089561E081E0B5DF73
:108FB00061E081E0B2DF80E0DFCFCF93C82F80E0B7
:108FC000CFDF8C2F8F738068CF9191CFCF93C82F35
:108FD00080E0C6DF8C2F8F738064CF9188CF1F9382
:108FE000CF93DF931F92CDB7DEB7182F81E069834F
:108FF000B7DF6981862F80687ADF812F8F70806864
:109000000F90DF91CF911F9172CF80E0A9DF81E0B7
:109010006EDF6FE070E080E090E00C947C3229DF3E
:10902000F4DF61E081E079DF2FCF23DFBEDFEDDF0A
:1090300061E081E072DF28CFCF93C82F85E0BDDFEC
:109040003ADFC11102C0C6E001C0C4E080E03FDFEA
:109050008C2FCF913CCFCF92DF92EF92FF921F9354
:10906000CF93DF931F921F92CDB7DEB769837A83C8
:10907000ADDF21DF6981C62E7A81D72E11E1115033
:1090800059F0F601E590F4908F2D21DF8E2D1FDF32
:1090900082E0C80ED11CF3CF0F900F90DF91CF91DB
:1090A0001F91FF90EF90DF90CF900895CF93DF93C3
:1090B000C0E06C2F80E093DFFEDED1E1D15029F0DB
:1090C00080E005DF80E003DFF9CFCF5FC03289F7B2
:1090D000DF91CF910895CF92DF92EF92FF920F939D
:1090E0001F93CF93DF931F92CDB7DEB7982F6230D7
:1090F00010F06250985FC62EC29480EFC8228A0199
:10910000D12C6D2D6C0D892F998369DFD4DEF80188
:10911000E590F4908F2DDBDE8E2DD9DED3940E5F9B
:109120001F4F998180E1D812ECCF0F90DF91CF9142
:109130001F910F91FF90EF90DF90CF90089580E006
:109140002DDF69ED77E180E090E085DF69EB77E185
:1091500080E190E080DF69E977E180E290E07BDF09
:1091600069E777E180E390E076DF49E158E160E08C
:1091700080E0B1DF49EF57E161E080E0ACDF49E535
:1091800057E161E085E0A7DF80E056CFCF93DF9322
:10919000EC018991882311F09ADEFBCFDF91CF910A
:1091A00008950F931F93CF93DF93CDB7DEB7279723
:1091B0000FB6F894DEBF0FBECDBF6330B1F038F408
:1091C0006130B1F0623049F525E437E113C0653014
:1091D00031F040F0663009F525E537E10BC021E5B7
:1091E00037E108C02DE437E105C029E437E102C0CA
:1091F00021E437E19F938F933F932F938E010F5F6D
:109200001F4F1F930F930F942782C801BFDF0F904A
:109210000F900F900F900F900F9027960FB6F89425
:10922000DEBF0FBECDBFDF91CF911F910F9108958B
:109230000F931F93CF938C01C62FF80181918F015B
:10924000882329F0CC2319F042DEC150F6CFCF910C
:109250001F910F910895CF92DF92EF92FF920F939B
:109260001F93CF93DF93CDB7DEB727970FB6F89450
:10927000DEBF0FBECDBF8C0188E09FDEF8016081AC
:109280007181828193812CE3C22ED12CE12CF12CAF
:10929000A70196010F94CF7CCA01B901A7019601DD
:1092A0000F94CF7C8E010F5F1F4F2436310598F449
:1092B0007F936F933F932F938BE297E19F938F93CD
:1092C0001F930F930F9427820FB6F894DEBF0FBE43
:1092D000CDBF85E012C07F936F933F932F9383E2BE
:1092E00097E19F938F931F930F930F9427820FB64D
:1092F000F894DEBF0FBECDBF86E0F801E80FF11D88
:1093000080E28083D8DD66E0C80192DF27960FB641
:10931000F894DEBF0FBECDBFDF91CF911F910F91AB
:10932000FF90EF90DF90CF900895CF93DF93FC01F3
:109330008491EF012196882319F0C9DDFE01F8CF51
:10934000DF91CF910895CF92DF92EF92FF920F932A
:109350001F93CF93DF93C42E623010F06250805F72
:10936000982F9170D92EC82FC695D62FD295D07F21
:1093700089E3E82E88E1F82E01E0F7011491602FCF
:109380006D0F8C2F2CDE97DDCC2051F0D11002C058
:10939000812F01C080E09BDDDD2021F0812F03C003
:1093A00080E095DD80E093DD0F5FFFEFEF1AFF0AAD
:1093B000053019F7DF91CF911F910F91FF90EF903A
:1093C000DF90CF9008958F929F92AF92BF92DF92DD
:1093D000EF92FF920F931F93CF93DF93D82E69E103
:1093E0000F949C7C20E1929FC001112469E170E000
:1093F0000F94BC7C80E090E85C0102C0B594A79417
:109400006A95E2F711E0ED2CF12C612F8CE0E7DD9D
:1094100052DD20E030E000E0490189E1880E911C36
:10942000E814F90434F42E153F0534F0C0E0D0E020
:1094300004C0CFEFDFEF01C0E501113051F01D3066
:1094400041F0033011F4C16006C0011104C0D068BE
:1094500002C0CFEFDFEF8D2F3ADD8C2F38DD0F5FAD
:10946000940124363105C1F61F5F1E3071F68CE081
:10947000A4DD21DD80E22BDD29E02D1530F464E050
:10948000C7018FDE8EE397E105C063E0C70189DE87
:109490008AE397E1DF91CF911F910F91FF90EF90B9
:1094A000DF90BF90AF909F908F903FCFCF93C82F0A
:1094B0000E944894C11104C09091CA05981721F0E8
:1094C0008093CA05CF917FCFCF9108951F93CF93FB
:1094D000DF931F92CDB7DEB7182F80E169836DDD72
:1094E000EADC6981662349F0111102C012E001C073
:1094F00010E080E0ECDC812F03C080E2E8DC80E259
:109500000F90DF91CF911F91E2CCCF92DF92EF923B
:10951000FF920F93CF93DF93C82F6B017A01D22F65
:10952000813049F028F0823049F0833039F008C0AA
:1095300081E043DD05C081E140DD02C089E03DDD21
:10954000BADC63E0C6012DDEDD2341F08AE1BFDC39
:1095500063E0C70126DE011106C015C0002399F0A3
:1095600085E397E1E2DE41E04D276C2F85E0EBDEFD
:109570004D2F6C2F89E0DF91CF910F91FF90EF90ED
:10958000DF90CF90E0CEDF91CF910F91FF90EF90E1
:10959000DF90CF9008950F93CF936115710589F0F7
:1095A000C1E0681779073CF49C01261B370B233078
:1095B000310544F406C09B01281B390B23303105CB
:1095C0000CF4C0E02091180221702C1711F001E07A
:1095D00001C0042F2C2FAB01BC0180E096DF8091ED
:1095E0001802C0FB80F980931802CF910F91089563
:1095F0000F93CF936115710589F0C1E06817790762
:109600003CF49C01261B370B2330310544F406C083
:109610009B01281B390B233031050CF4C0E020914D
:10962000180222FB222720F92C1711F001E001C0BB
:10963000042F2C2FAB01BC0181E067DF8091180261
:10964000C0FB82F980931802CF910F910895CF93B8
:10965000C82F86E0B2DC2FDC63E08C2F90E0A1DD28
:1096600085E2CF9134CCCF93DF93EC0186E1A5DC8A
:1096700022DC63E0CE0195DD85E2DF91CF9127CC3E
:109680004F925F926F927F928F929F92AF92BF9212
:10969000CF92DF92EF92FF921F93CF93DF9300D090
:1096A0001F92CDB7DEB7F82E811104C082DB88236C
:1096B00009F467C00E94868F182F0F941174698374
:1096C0007A838B839C83A0906602B090670260913E
:1096D0002A0E70912B0E80912C0E90912D0E0F94CE
:1096E000F4792B013C01C0902E0ED0902F0E80906B
:1096F000520E9090530E60914E0E70914F0E8091CD
:10970000500E9091510E0F94F479DC01CB014F2D46
:10971000B40141DF4F2DB601C2016ADF2091490E2D
:10972000E22EF12C11110DC090913A0297FD09C063
:10973000929F900111247901EE0CEF2CEE1CFF0892
:10974000F19424E62E9DC0012F9D900D1124815887
:109750009F4F6FEF70E00F94BC7C862F78DFCE01B7
:10976000019679DDC5017FDFEF2811F0812F64DCE0
:1097700061E01C141D041CF060E080E001C0812F3A
:10978000A5DE0F900F900F900F90DF91CF911F915A
:10979000FF90EF90DF90CF90BF90AF909F908F9011
:1097A0007F906F905F904F900895CF9388E105DC94
:1097B00082DB84E798E00E94588EC82F65E184E739
:1097C00098E036DDC53120F480E281DBCF5FFACF4F
:1097D000CF910895811103C01EDB882311F0E5DFCE
:1097E0003BCB0895CF93C82F44DB8C2F49DF8C2FC0
:1097F000F1DF8C2F5BDECF9147CB3BDBD6DB05DC8B
:1098000055DC9DDC81E0EEDF3FCB80E0EBCF90913B
:10981000C905981729F08093C9058111EECFFFCBB8
:109820000895E6EEF5E083AF64AF08954AE050E0B6
:10983000BC0186EE95E00C94093EEF92FF920F93E7
:109840001F93CF93DF937A016F3F710581059105D7
:1098500009F058F486EE95E00E94733D8AEE95E09B
:109860000E944B3A282F30E014C0C0912106D091BD
:1098700022064D2F50E0EC2FF0E08B019C01BF0140
:109880008AEE95E0ADD1C80FC0932106D093220691
:109890009C01C901DF91CF911F910F91FF90EF9033
:1098A0000895EF92FF920F931F93CF93DF938B0155
:1098B000C6EED5E0FBACECAC4E2D50E06F2D70E069
:1098C0009C018AEE95E0E4D1F80EFBAEECAEDF91A0
:1098D000CF911F910F91FF90EF900895EF92FF921B
:1098E0000F931F93CF93DF938B01C6EED5E0FBACB4
:1098F000ECAC4E2D50E06F2D70E09C018AEE95E0AF
:1099000013D2F80EFBAEECAEDF91CF911F910F9109
:10991000FF90EF9008950F931F93CF93DF93CDB7F0
:10992000DEB728970FB6F894DEBF0FBECDBF8A0111
:1099300023E0660F771F2A95E1F7680F791F48E04B
:1099400050E0CE0101960F945B8129813A81F801A4
:10995000808191812817390790F08217930760F072
:109960009C818281981758F081E090E03B812381AF
:10997000231738F080E005C081E090E002C08FEF4F
:109980009FEF28960FB6F894DEBF0FBECDBFDF91D4
:10999000CF911F910F910895EF92FF920F931F9314
:1099A000CF93DF93EC018B017A018A859B85861723
:1099B000970731F0888199810E94963C1B870A871E
:1099C00088859985019689F00E811F81B70188816C
:1099D00099810E94933C080F111D888599858017F5
:1099E000910718F481E090E011C06E818A81680FC0
:1099F00097014C81888199810E94A73B2E813F81EC
:109A0000280F311D3F832E8380E090E0DF91CF91BE
:109A10001F910F91FF90EF9008954F925F926F9278
:109A20007F928F929F92AF92BF92CF92DF92EF92EE
:109A3000FF920F931F93CF93DF93CDB7DEB72D9790
:109A40000FB6F894DEBF0FBECDBF6C012A013B01FB
:109A5000490158011B861C86CE0101967C0188E0D5
:109A6000F70111928A95E9F7DB01CA0127E0B69563
:109A7000A795979587952A95D1F79A838983F42F8F
:109A8000FF77FD878F2F80588B838C831A861986EA
:109A90004F3F51056105710509F018F460E070E071
:109AA00026C06091DB057091DC058E01075F1F4FBA
:109AB00097014BE85CE48091D9059091DA050E940A
:109AC000A98C97FDEBCF69857A8583E0660F771FB8
:109AD0008A95E1F78091D9059091DA05680F791F91
:109AE00048E050E0C7010F945B816F817885611574
:109AF000710519F44B86B60106C0C616D70619F0D3
:109B00008D8580688B87AE01455F5F4FC401F5018D
:109B100019952D960FB6F894DEBF0FBECDBFDF911D
:109B2000CF911F910F91FF90EF90DF90CF90BF905A
:109B3000AF909F908F907F906F905F904F9008951F
:109B40006F927F928F929F92AF92BF92CF92DF924D
:109B5000EF92FF920F931F93CF93DF9300D01F924A
:109B6000CDB7DEB76C017B013A015901480119827A
:109B70001A821B821C82AE014F5F5F4FB301C70187
:109B80000E94098D7C0149815A816B817C8141153C
:109B900051056105710529F084019501C6013DDF7C
:109BA000E6CF0F900F900F900F90DF91CF911F9104
:109BB0000F91FF90EF90DF90CF90BF90AF909F906C
:109BC0008F907F906F90089521E02093DD05E9ED5F
:109BD000F5E0918380837383628380E090E0089551
:109BE0007F92AF92BF92CF92DF92EF92FF920F934C
:109BF0001F93CF93DF93CDB7DEB72C970FB6F894B2
:109C0000DEBF0FBECDBF6C01762EF72F842FE52F60
:109C1000B901A801D6011496AD90BC90159790910A
:109C2000DD0591110AC02DE738E1482F672DC601E7
:109C30000E94DE3B80E090E019C0DA82C9827B821C
:109C4000FC838D83EE8318861F82FA86E9861C8644
:109C50001B860CEC1CE49E012F5F3F4FC501DDDE2F
:109C6000B501C6010E94963C8F8198852C960FB64F
:109C7000F894DEBF0FBECDBFDF91CF911F910F9142
:109C8000FF90EF90DF90CF90BF90AF907F900895BE
:109C9000CF92DF92EF92FF920F931F93CF93DF93B8
:109CA000CDB7DEB72C970FB6F894DEBF0FBECDBF91
:109CB0007C01C901F701C480D5802091DD05211107
:109CC00008C02DE538E1C7010E94DE3B80E090E04E
:109CD0001CC0FA82E9826B837C834D835E83188685
:109CE0001F821A8709871C861B860CEC1CE49E01C8
:109CF0002F5F3F4F43EA5CE8BC01C60121DFB6019C
:109D0000C7010E94963C8F8198852C960FB6F894D7
:109D1000DEBF0FBECDBFDF91CF911F910F91FF909E
:109D2000EF90DF90CF900895CF92DF92EF92FF9265
:109D30000F931F93CF93DF93CDB7DEB72C970FB65A
:109D4000F894DEBF0FBECDBF7C01C901F701C4800E
:109D5000D5802091DD05211108C02DE338E1C70130
:109D60000E94DE3B80E090E01CC0FA82E9826B83B7
:109D70007C834D835E8318861F821A8709871C8621
:109D80001B860CEC1CE49E012F5F3F4F46EA5CE80B
:109D9000BC01C601D5DEB601C7010E94963C8F8189
:109DA00098852C960FB6F894DEBF0FBECDBFDF911D
:109DB000CF911F910F91FF90EF90DF90CF9008957A
:109DC000CF93DF93EC01262F4CAD6BAD04960E9430
:109DD000893B2BAD082E000C990B820F911D8BAF88
:109DE00081E090E0DF91CF9108950F939CE0899FEF
:109DF000802D112421E0280F2093E505845F8093B6
:109E0000E40590E0029640911E0650E08417950705
:109E100014F480E033C0822F90E02091200630E0DF
:109E200082179307B4F76623A9F061E08AEE95E004
:109E30000E9464374091E5054E5F0BE020E860E04A
:109E40008AEE95E00E94063A60E08AEE95E00E9474
:109E5000643705C061E08AEE95E00E946437609146
:109E6000E40580911E066817A0F29091E5058091A7
:109E70002006891770F280E0D4DC81E00F9108950C
:109E8000CF93DF93FC0185ADEF012496811105C0CE
:109E900081E085AFCE010E940B37CE01DF91CF91DB
:109EA0000C9442376FEF7FEF19CD6FEF7FEFF9CC56
:109EB0004FEF5FEFC2CC482F50E02091E305022E18
:109EC000000C330B4217530781F08093E305813078
:109ED00031F467EE72E28AEE95E00C94963C68E607
:109EE00079E18AEE95E00C94963C0895EF92FF920A
:109EF0000F9386EE95E0C4DF89EAE82E80E2F82E23
:109F000000E428E040E060E08AEE95E00E948E37B1
:109F10006BEB74E08AEE95E00E94963C28E433E017
:109F200041E169E38AEE95E00E94A73B6BE27DE0A8
:109F30008AEE95E00E94963C2FE433E04CE16AE320
:109F40008AEE95E00E94A73B66E870E18AEE95E014
:109F50000E94963C28E533E049E26BE38AEE95E007
:109F60000E94A73B66E870E18AEE95E00E94963C6D
:109F700024E633E04EE36DE38AEE95E00E94A73BD2
:109F800026E633E04EE362E48AEE95E00E94A73BCA
:109F90008AEE95E00E9446378111AECF64EC79E0FD
:109FA00080E090E00E94F8AB68E679E18AEE95E007
:109FB0000F91FF90EF900C94963C61E089EA90E25B
:109FC00095DF64EC79E080E090E00C94F8ABEF92E0
:109FD000FF920F93F2DF86EE95E052DF85E9E82EDF
:109FE0008EE1F82E06E22EE040E068E08AEE95E091
:109FF0000E948E3783E05FDF26E633E040E365E2D0
:10A000008AEE95E00E94A73B20E733E04CE367E04F
:10A010008AEE95E00E94A73B8AEE95E00E944637C3
:10A020008111DCCF64EC79E080E090E00F91FF904B
:10A03000EF900C94F8AB60E070E087EE92E2C4CD54
:10A040001F93CF93DF930E941548C091EB05C695EF
:10A05000C69586EE95E014DFDC2FDD0F1D2F1C0F5B
:10A0600083E029DF6C2F80E0DCDB84E798E01DDFF4
:10A070006D2F80E0D6DB8AEA98E114DF612F80E063
:10A08000D0DB8DE998E10EDF8AEE95E00E9446373D
:10A090008111E6CFDF91CF911F9108950895CF935D
:10A0A000E62F6CE0869F602D112481E0860F80935F
:10A0B000E505645F6093E405462F50E04E5F5F4F17
:10A0C00020911E0630E0421753070CF445C090E083
:10A0D0002091200630E0821793070CF03DC0CE2F70
:10A0E0008EE39FDB65E470E080E090E0E1DE61E319
:10A0F0006C0F062E000C770B880B990BD9DE60E2F3
:10A1000070E080E090E0D4DE60914E0E70914F0ED2
:10A110008091500E9091510E0F94F479CB010E94D2
:10A1200003ADC3DE6FE270E080E090E0C1DE0E942C
:10A13000868F811109C085E0C89FF0011124E35C7E
:10A14000F14F8481811108C08091520E9091530E7D
:10A150000E9403ADCF91A9CECF910895CF92DF9207
:10A16000EF92FF920F931F93CF93DF931F921F9253
:10A17000CDB7DEB77B01622F498337DE4981882363
:10A1800009F440C0442309F101151105F1F4C70198
:10A190000E94798E25E130E0281B310937FF02C08B
:10A1A0002F5F3F4F3595279530E82158822F830F39
:10A1B00087FD0CC060E270E080E090E02A83398384
:10A1C00077DE398131502A81F1CF30E8C32ED12C8E
:10A1D000B601C70183DB7601E81AF90A01151105FA
:10A1E00011F41E2D06C0FF24B701C8015ADB1E2D35
:10A1F000181B173038F060E270E080E090E058DE25
:10A20000181BF7CF0F900F90DF91CF911F910F91F7
:10A21000FF90EF90DF90CF9008950F93CF93DF934F
:10A22000982F862FEA01692FE0DD882309F162E784
:10A2300070E0CE0153DBC2E7C81BC73038F060E2E4
:10A2400070E080E090E034DEC81BF7CF6091E40559
:10A250008AE7E7DA602F000F770B880B990B28DE6F
:10A2600060E270E080E090E0DF91CF910F9120CE2E
:10A27000DF91CF910F910895CF92DF92EF92FF92ED
:10A280000F931F93CF93DF93982F862F6A01790145
:10A29000692FABDD882309F442C0C701002321F0F8
:10A2A0000E94798E182F03C00E94588E182FC3E188
:10A2B000D0E0C11BD1098C2F880FC80FCC0FD0E084
:10A2C000BE01C6010BDBC81B6AE370E080E090E0D2
:10A2D000EFDDC73038F060E270E080E090E0E8DD6C
:10A2E000C81BF7CF8AEF189F802D11246091E405D9
:10A2F000805897DAC701002349F0DF91CF911F9171
:10A300000F91FF90EF90DF90CF90CCCDDF91CF9168
:10A310001F910F91FF90EF90DF90CF90C6CDDF910E
:10A32000CF911F910F91FF90EF90DF90CF90089504
:10A33000BF92CF92DF92EF92FF920F931F93CF9332
:10A34000DF936C017B010E94798EC82FC7010E94A8
:10A35000588E03E110E0081B11098C2F90E0BB24FC
:10A36000B394081719071CF0B12CC5E201C0CFE166
:10A370002C2F30E0A9014E5F5F4F80911E0690E0C8
:10A380004817590744F0295031098091200690E080
:10A39000821793079CF5D0E0E114F104B1F16AE370
:10A3A00070E080E090E084DDBB2081F0C45F8091AC
:10A3B0001E06C81750F12C2F30E02950310980912A
:10A3C000200690E0821793071CF41FC0DD23E9F0FC
:10A3D000802F880F800F6C2F880F23DA60E270E0E7
:10A3E00080E090E065DDC701DF91CF911F910F9173
:10A3F000FF90EF90DF90CF90BF9057CD6C2F80E013
:10A4000010DAC6014FDDD1E0C7CFDF91CF911F91A8
:10A410000F91FF90EF90DF90CF90BF900895CF9273
:10A42000DF92EF92FF920F931F93CF93DF931F92D0
:10A43000CDB7DEB7182F7A01D22ECA0169830E94E8
:10A44000798E082F812F880F810FC82ECC0C1CE02D
:10A450006981169F100D1124DD20C1F061E08AEEA4
:10A4600095E00E946437202F220F200F220F2E5FCD
:10A470000BE047EF410F6FEF6C0D8AEE95E00E9405
:10A48000063A60E08AEE95E00E946437612F8C2DD9
:10A49000C8D9C70107DDDD2071F061E08AEE95E0E3
:10A4A0000F90DF91CF911F910F91FF90EF90DF9070
:10A4B000CF900C9464370F90DF91CF911F910F9143
:10A4C000FF90EF90DF90CF9008958F929F92AF9280
:10A4D000BF92DF92EF92FF920F931F93CF93DF9380
:10A4E000EC015B01D42E49016CE080E09AD9C401F3
:10A4F000D9DC0115110521F0B80181E00E94408FDF
:10A50000E114F10411F0C701CDDC91E02D2D2927D4
:10A51000A50164E081E083DFCE010E94798E2D2DBC
:10A52000AE0164E094E1981B892FDF91CF911F91D8
:10A530000F91FF90EF90DF90BF90AF909F908F9022
:10A540006ECFEF92FF920F93CF93DF93D82FC62F4A
:10A550007901682F8C2F49DC8823D9F0002329F05A
:10A5600062E070E080E090E0A3DC2D2F4C2F64E1EE
:10A57000C7010E94F18E68E770E093D9C8E7C81B55
:10A58000C73038F060E270E080E090E091DCC81BFA
:10A59000F7CFDF91CF910F91FF90EF9008958F92B9
:10A5A0009F92AF92BF92CF92DF92EF92FF920F9362
:10A5B0006B017C018090DF059090E005A090E105A3
:10A5C000B090E205A50194010F948579882301F1EB
:10A5D00020E030E0A901C701B6010F9485798823F6
:10A5E00051F0A5019401C701B6010F94857987FD4B
:10A5F00004C081E003C080E001C08FEF8093DE05DE
:10A60000C092DF05D092E005E092E105F092E2050C
:10A6100080911E06813128F480912006833008F055
:10A6200048C080911E06853128F48091200684312F
:10A6300008F04FC080911E068F3308F057C08091FC
:10A6400020068F3208F452C088E0E82E89E1F82E07
:10A6500000E123E04FE265E08AEE95E00E948E374C
:10A6600098E3E92E99E1F92E23E04FE26AE58AEEBC
:10A6700095E00E948E378091DE0540E3481B2EEE68
:10A68000E22E28E1F22E0DE022E06EE68AEE95E061
:10A690000E948E378091DE0541E3481B34EDE32EA6
:10A6A00038E1F32E22E069E18AEE95E00E948E37D0
:10A6B0001DC08091DE0544E0481B59EBE52E58E1B2
:10A6C000F52E0CE022E062E48AEE95E00E948E37DF
:10A6D000A8CF41EDE42E48E1F42E01E023E044E16F
:10A6E0006CE38AEE95E00E948E37A4CF0F91FF9025
:10A6F000EF90DF90CF90BF90AF909F908F90089594
:10A70000CF92EF920F93CF93DF93C6EED5E01B82EB
:10A710001A8288E893E099838883CC24CA94EE2433
:10A72000EA9402E522E143E169E172E0CE010E9490
:10A73000453E84E993E099838883DF91CF910F911F
:10A74000EF90CF9008955A9887FD52C05B98000013
:10A750000000000000005A9A5A98282F220F86FD08
:10A7600053C05B9800000000000000005A9A5A98FD
:10A77000922F990F26FD46C05B9800000000000054
:10A7800000005A9A5A98892F880F96FD39C05B9815
:10A7900000000000000000005A9A5A98982F990F64
:10A7A00086FD2CC05B9800000000000000005A9A53
:10A7B0005A98892F880F96FD1FC05B9800000000F3
:10A7C000000000005A9A5A98982F990F86FD12C0DF
:10A7D0005B9800000000000000005A9A5A9896FD0D
:10A7E00015C05B9800000000000000005A9A089510
:10A7F0005B9AADCF5B9AEDCF5B9AE0CF5B9AD3CFFC
:10A800005B9AC6CF5B9AB9CF5B9AACCF5B9AEACF23
:10A810002F923F925F927F929F92AF92BF92CF9280
:10A82000DF92EF92FF920F931F93CF93DF937C0100
:10A830001B01942E69018AE0481709F47BC0A5E149
:10A840004A134EC0DB011296ED91FC9113971281D1
:10A85000C681D7815D9A88E28A950000E9F700EE0B
:10A86000010F80E1582E510E98E2792E88EF6BDFB0
:10A87000872D8A950000E9F7103208F046C0812F35
:10A880008077806860DF812F8295807F5CDF872DF5
:10A890008A950000E9F780E856DF80E054DF872DD5
:10A8A0008A950000E9F78AEF4EDF872D8A95000030
:10A8B000E9F75E01B0E1AB0EB11C8881807F43DF18
:10A8C00089918295807F3FDFCA15DB05B1F7872D1F
:10A8D0008A950000E9F71F5F0F5F1511C7CF5D98DC
:10A8E0009601492DB101C701DF91CF911F910F91C1
:10A8F000FF90EF90DF90CF90BF90AF909F907F90B0
:10A900005F903F902F900C94C838802F807780689C
:10A910001ADF802F8295807F16DF872D8A950000B1
:10A92000E9F780E810DF80E80EDF872D8A950000C8
:10A93000E9F7B9CF559A5D98539A5B98529A5A9A0B
:10A940005D9AC8E28C2F8A950000E9F788E790E0CD
:10A950000E94E53788EFF7DE8C2F8A950000E9F733
:10A9600080E2F1DE80E0EFDE8C2F8A950000E9F7CF
:10A9700080E0E9DE80E8E7DE8C2F8A950000E9F7C9
:10A9800080E0E1DE80E1DFDE8C2F8A950000E9F7D0
:10A990008FE090E00E94E53780E2D5DE80E4D3DEF0
:10A9A0008C2F8A950000E9F780E2CDDE80E6CBDED1
:10A9B000CA950000E9F710E0D8E208E2812F80771D
:10A9C0008068C1DE812F8295807FBDDE8D2F8A95C4
:10A9D0000000E9F780E8B7DE80E0B5DE8D2F8A95CC
:10A9E0000000E9F78AEFAFDE8D2F8A950000E9F7C6
:10A9F000C0E280E0A8DE80E0A6DE9D2F9A950000F0
:10AA0000E9F7C150B1F788EF9EDE802F8A950000EC
:10AA1000E9F71F5F103209F0D1CF80E094DE80ECBF
:10AA200092DE88E28A950000E9F75D9859CFCF93CE
:10AA3000DF931F921F92CDB7DEB789839A830E945E
:10AA4000E68320E040E060E070E089819A810F9029
:10AA50000F90DF91CF910C94F8840F93CF93DF93F5
:10AA600061E081E00E94AC85D0914208C0E0D11144
:10AA700017C080914108811104C00E943B8F811151
:10AA800065C080912702882309F457C081E0909126
:10AA90004108911180E004E024E04BEF5BE24BC001
:10AAA000D130C1F480914108813021F40E943B8F64
:10AAB000811154C080912702882309F43EC081E0AF
:10AAC00090914108913009F080E003E02EE342EFDD
:10AAD0005BE231C0D230B9F480914108823021F478
:10AAE0000E943B8F811143C080912702882329F166
:10AAF00081E090914108923009F080E003E02EE37C
:10AB000049EE5BE218C0D330C1F480914108833034
:10AB100021F40E943B8F811133C08091270288234A
:10AB200061F081E090914108933009F080E003E00A
:10AB30002EE343EE5BE26C2F70DBCF5FDF5FC5304F
:10AB400009F095CF84E08093400821C00E942485BD
:10AB500080910E08882309F494CF19C08BE19AE7FD
:10AB600066DF80910E08882309F4A4CF10C080E02E
:10AB70009FE75DDF80910E08882309F4B5CF07C0F9
:10AB800082EC92E854DF80910E08882331F2DF9145
:10AB9000CF910F910895EF92FF920F931F938091A1
:10ABA00027028823B9F080918A0A811103C00CEC36
:10ABB0001AE002C00AE81AE08FE3E82E8CE2F82ED1
:10ABC00022E33CE244E257E06BE27CE285E29CE275
:10ABD0000E94B0860E943B8F8823B1F080912407A9
:10ABE000882361F08CEC9AE00E94A5980E941D8554
:10ABF0001F910F91FF90EF900C9428941F910F914B
:10AC0000FF90EF900C9424851F910F91FF90EF908F
:10AC100008950E94F59C21E030E0811102C020E0FF
:10AC200030E030936908209368081092420881E070
:10AC300080930E0883E0809327020895CF92DF92DD
:10AC4000EF92FF920F931F93CF93DF930E94F29D99
:10AC50006C0161E081E00E94AC85C0914208D0E0C7
:10AC600081E0C81AD108C11117C080914108811133
:10AC700004C00E943B8F811195C0809127028823D8
:10AC800059F081E090914108911180E004E024E0C6
:10AC900040E25CE26D2FC1DA6CEC7AE083E59AE089
:10ACA0000E94D9A38091CC0A8F3201F18091D90AF8
:10ACB00083FF1CC0C130C1F480914108813021F470
:10ACC0000E943B8F811176C080912702882361F01A
:10ACD00081E090914108913009F080E000E22EE39C
:10ACE0004CE15CE26D2F99DA92E001C091E0809135
:10ACF0002702882309F44EC0760111E01C0F8FEF64
:10AD0000E816F80609F446C0C9133FC060E070E0D9
:10AD1000C7010E941A9A9091D90A8091410894FF24
:10AD20001CC08C134EC00E943B8F882309F449C07D
:10AD30008CEC9AE00E949F9C1092420882E090E086
:10AD4000909369088093680881E080930E081092C0
:10AD50006B0883E08093270254C08C1304C00E94C8
:10AD60003B8F81113DC080912702882361F081E0F3
:10AD7000909141089C1380E000E022E83AE140E035
:10AD80005CE26D2FDEDB912F01C09F5F81E0E81A4E
:10AD9000F108B5CFDF5FCF5FD53009F064CF909376
:10ADA00040082FC00E94248580910E08882309F452
:10ADB00064CF27C02EDF80910E08882309F484CF4A
:10ADC00020C0809127028823F1F281E09091410810
:10ADD0009C1380E001E022E83AE14EE05CE2D1CF52
:10ADE000109224070E94E68320E040E060E070E0DB
:10ADF0008BEC95E50E94F88480910E08882309F475
:10AE0000B2CFDF91CF911F910F91FF90EF90DF9024
:10AE1000CF900895FC0160830895CF93DF93EC01F8
:10AE2000072E000C880B990B0F94277A2FE632E13E
:10AE300043E85AE30F94C37B688379838A839B83B7
:10AE4000DF91CF9108956AE077E58FE297E50C9462
:10AE500039856DE077E587E497E50C9439850C94A6
:10AE60003CACCF93DF9300D01F92CDB7DEB76983A0
:10AE70007A838B839C8360E2CE0101960E947BAE35
:10AE80000F900F900F900F90DF91CF910895BC011C
:10AE9000990F880B990B0F94277A2FE632E143E83C
:10AEA0005AE30F94C37BDDCF2F923F924F925F9274
:10AEB0006F927F928F929F92AF92CF92DF92EF929A
:10AEC000FF920F931F93CF93DF9300D01F92CDB7C4
:10AED000DEB74C011B01CA01B901E982FA820B837A
:10AEE0001C8320E030E04AE754E40F94C37B0F94C6
:10AEF000F4792B013C0120E030E04AE754E4F10111
:10AF000060817181828193810F94C37B0F94F47966
:10AF10008B010419150920E030E04AE754E4698107
:10AF20007A818B819C810F94C37B0F94F4799B0170
:10AF30002419350989E2E82E87E5F82EA201B1012E
:10AF4000C4010E940D840F900F900F900F90DF911D
:10AF5000CF911F910F91FF90EF90DF90CF90AF9026
:10AF60009F908F907F906F905F904F903F902F9029
:10AF70000895AF92CF92DF92EF92FF920F931F93BB
:10AF8000CF93DF9361E081E00E94AC85D0914208CD
:10AF9000C0E0D11119C080914108811104C00E9404
:10AFA0003B8F8111C4C080912702882309F4B6C069
:10AFB00081E090914108911180E004E024E047E7AE
:10AFC0005CE26C2F2AD9AAC0D130E1F4809141080B
:10AFD000813021F40E943B8F8111B1C08091270202
:10AFE000882309F49BC011E080914108813009F069
:10AFF00010E08091B9160E943CAC00E09C0141E653
:10B000005CE289C0D23009F580914108823021F498
:10B010000E943B8F8111B0C080912702882309F4E0
:10B020007DC011E080914108823009F010E060910C
:10B03000BA167091BB168091BC169091BD1611DFA7
:10B0400000E09C014DE55CE266C0D33009F58091DB
:10B050004108833021F40E943B8F8111A6C080916A
:10B060002702882309F45AC011E0809141088330F7
:10B0700009F010E06091BE167091BF168091C01665
:10B080009091C116EEDE00E09C0149E55CE243C010
:10B09000D43001F580914108843021F40E943B8F27
:10B0A00081119CC0809127028823C1F111E0809119
:10B0B0004108843009F010E06091C2167091C31607
:10B0C0008091C4169091C516CCDE00E09C0145E548
:10B0D0005CE221C0D53011F580914108853021F422
:10B0E0000E943B8F811193C0809127028823B1F089
:10B0F00011E080914108853009F010E060918302F1
:10B10000709184028091850290918602AADE00E00F
:10B110009C0141E45CE26C2F812FAED8CF5FDF5FF2
:10B12000C53009F036CF86E08093400888C00E9481
:10B13000248580910E08882309F435CF80C081E0F2
:10B140000E94308F0091B91610E0A12CC12CD12C97
:10B1500043E2E42E47E5F42E2FEF30E040E050E0EC
:10B1600069EB76E18CE69CE20E940D8480910E08EA
:10B17000882309F433CF63C081E00E94308FA12C73
:10B18000C12CD12C16E6E12EFE2C0EE111E420E0BC
:10B1900030E0A9016AEB76E18FE59CE285DE8091E3
:10B1A0000E08882309F438CF4AC081E00E94308F0E
:10B1B000A12CC12CD12C16E6E12EFE2C0EE111E4BF
:10B1C00020E030E0A9016EEB76E18BE59CE26CDEDD
:10B1D00080910E08882309F442CF31C081E00E949B
:10B1E000308FA12CC12CD12C16E6E12EFE2C0EE1C5
:10B1F00011E420E030E0A90162EC76E187E59CE211
:10B2000053DE80910E08882309F44CCF18C081E0EA
:10B210000E94308FA12CC12CD12C16E6E12EFE2CE1
:10B220000EE111E420E030E0A90163E872E08BE474
:10B230009CE23ADE80910E08882309F455CFDF9115
:10B24000CF911F910F91FF90EF90DF90CF90AF9033
:10B250000895CF93DF93EC01072E000C880B990B18
:10B260000F94277A2AE037ED43E25CE30F94C37B27
:10B27000688379838A839B83DF91CF910895CF93ED
:10B28000DF93EC01072E000C880B990B0F94277AA3
:10B29000688379838A839B83DF91CF910895CF93CD
:10B2A000DF93EC01072E000C880B990B0F94277A83
:10B2B00020E030E048EC52E40F94C37B688379834C
:10B2C0008A839B83DF91CF910895CF93DF93EC0125
:10B2D000072E000C880B990B0F94277A20E030E0A2
:10B2E00048EC52E40F94C37B0F94F9796883798317
:10B2F0008A839B83DF91CF910895CF93DF93EC01F5
:10B30000072E000C880B990B0F94277A2AE037ED53
:10B3100043E25CE30F94C37B688379838A839B83D6
:10B32000DF91CF91089569E279E586ED99E50C9476
:10B3300039856FE379E58BE39AE50C9439856FE401
:10B3400079E587EF99E50C94398565E679E58BE534
:10B350009AE50C9439856DE779E585EB99E50C94D0
:10B3600039850D94E32B0D942A2CCF93DF9300D0D5
:10B370001F92CDB7DEB7BC01990F880B990B0F94C4
:10B38000277A2AE037ED43E25CE30F94C37B6983BD
:10B390007A838B839C83CE0101960E947CB00F90B0
:10B3A0000F900F900F90DF91CF910895CF93DF937F
:10B3B00000D01F92CDB7DEB7BC01990F880B990B57
:10B3C0000F94277A2AE037ED43E25CE30F94C37BC6
:10B3D00069837A838B839C83CE0101960E9465AD3D
:10B3E0000F900F900F900F90DF91CF910895CF9312
:10B3F000DF9300D01F92CDB7DEB7BC01990F880B49
:10B40000990B0F94277A20E030E048EC52E40F9437
:10B41000C37B69837A838B839C83CE0101960E94D0
:10B42000C4AF0F900F900F900F90DF91CF910895C0
:10B43000CF92DF92EF92FF926B017C0120E030E02F
:10B44000A9010F94857987FD05C020E030E040E038
:10B450005FE304C020E030E040E05FEBC701B601ED
:10B460000F94AC780F94F479CB01FF90EF90DF90BC
:10B47000CF900C9403ADBC01990F880B990B0F94DE
:10B48000277AD6CFCF93DF9300D01F92CDB7DEB708
:10B490000F94F9790F94257A69837A838B839C833F
:10B4A000CE0101960E94C4AF0F900F900F900F90A5
:10B4B000DF91CF910895BC01990F880B990B0F94E0
:10B4C000277A20E030E048EC52E40F94C37BDACFD7
:10B4D0000F931F93CF93DF9361E081E00E94AC85CF
:10B4E000C0914208D0E0C1111AC080914108811179
:10B4F00004C00E943B8F8111E8C0809127028823FD
:10B5000009F461C081E090914108911180E004E06C
:10B5100024E04EEB5CE26D2F0E940D5154C0C1300F
:10B52000D9F480914108813021F40E943B8F811130
:10B53000D4C080912702882309F445C081E090910E
:10B540004108913009F080E003E02EE345EB5CE236
:10B550006D2F0E940D5137C0C230D1F48091410847
:10B56000823021F40E943B8F8111C0C0809127025C
:10B57000882349F181E090914108923009F080E000
:10B5800003E02EE348EA5CE26D2F0E940D511BC0E0
:10B59000C330C9F480914108833021F40E943B8F6D
:10B5A0008111ADC080912702882369F081E09091DC
:10B5B0004108933009F080E003E02EE343EA5CE2C7
:10B5C0006D2F0E940D510E94E18481111DC0C43075
:10B5D000E9F480914108843021F40E943B8F81116D
:10B5E00097C080912702882309F49BC081E0909145
:10B5F0004108943009F080E003E02EE34AE95CE280
:10B600006D2F0E940D518DC014E001C015E0C113D3
:10B610001BC0809141088C1304C00E943B8F811194
:10B6200082C080912702882371F081E090914108C7
:10B630009C1380E003E02EE341E95CE26D2F0E9461
:10B640000D511C2F01C01C2F81E0810FC81318C0A1
:10B65000809141088C1304C00E943B8F81116CC003
:10B6600080912702882361F081E0909141089C132A
:10B6700080E003E02EE345E85CE26D2F0E940D516F
:10B6800082E0810FC81318C0809141088C1304C058
:10B690000E943B8F811159C080912702882361F05D
:10B6A00081E0909141089C1380E003E02EE34CE799
:10B6B0005CE26D2F0E940D51DF5FCF5FD53009F046
:10B6C00012CF1D5F1093400848C00E9424858091CE
:10B6D0000E08882309F411CF40C08CE29DE5A7D95C
:10B6E00080910E08882309F424CF37C084E892E6BD
:10B6F0009ED980910E08882309F438CF2EC083E4A8
:10B7000090E695D980910E08882309F44BCF25C087
:10B7100084EF9EE58CD980910E08882309F461CFCF
:10B720001CC015E091CF89EB97E581D980910E0877
:10B73000882309F476CF11C082EF99E878D98091F7
:10B740000E08882309F48CCF08C085E09CE56FD9EA
:10B7500080910E08882309F49FCFDF91CF911F912C
:10B760000F9108952F923F924F925F926F927F9226
:10B770008F929F92AF92CF92DF92EF92FF920F93B0
:10B780001F93CF93DF9300D01F92CDB7DEB74C014C
:10B790001B01E982FA820B831C83CA01B9010F9451
:10B7A000F4792B013C01F1016081718182819381E7
:10B7B0000F94F4798B010419150969817A818B81C1
:10B7C0009C810F94F4799B012419350989E9E82EAD
:10B7D00089E5F82EA201B101C4010E940D840F90E9
:10B7E0000F900F900F90DF91CF911F910F91FF90CD
:10B7F000EF90DF90CF90AF909F908F907F906F9061
:10B800005F904F903F902F9008959F92AF92BF927C
:10B81000CF92DF92EF92FF920F931F93CF93DF931C
:10B8200000D01F92CDB7DEB761E081E00E94AC8509
:10B8300090904208B12C91101AC08091410881115A
:10B8400004C00E943B8F811198C0809127028823F9
:10B8500009F48AC081E090914108911180E004E0F0
:10B8600024E04CE95EE26B2D0E940D517DC081E029
:10B8700098122CC080914108813021F40E943B8FA6
:10B88000811183C080912702882309F46DC011E0E3
:10B8900080914108813009F010E08091371090913B
:10B8A0003810A0913910B0913A1089839A83AB83F4
:10B8B000BC83CE0101960E9465AD00E09C0148E882
:10B8C0005EE26B2D812F0E943C514EC082E09812A7
:10B8D00025C080914108823021F40E943B8F811164
:10B8E0007CC080912702882309F43EC011E080913A
:10B8F0004108823009F010E06091AF0D7091B00DF9
:10B900008091B10D9091B20D93DD00E09C0144E770
:10B910005EE26B2D812F0E943C5126C083E098127D
:10B9200023C080914108833021F40E943B8F811114
:10B930006CC0809127028823B9F011E08091410802
:10B94000833009F010E06091B30D7091B40D8091D7
:10B95000B50D9091B60D6CDD00E09C0144E65EE211
:10B960006B2D812F0E943C51B394939485E0B812C3
:10B9700062CF84E0809340085FC00E94248580915C
:10B980000E08882309F461CF57C020E030E048EC6E
:10B9900052E4609137107091381080913910909175
:10B9A0003A100F94C37B0F94F479A12CC12CD12CA5
:10B9B00023E9E22E29E5F22E8B012FEF3FE740E04D
:10B9C00050E067E370E182E99EE20E940D8480917D
:10B9D0000E08882309F456CF2FC081E00E94308FD3
:10B9E000A12CC12CD12CE12CF12C08E413E420E093
:10B9F00030E0A9016FEA7DE08EE79EE2B3DE809140
:10BA00000E08882309F46DCF17C081E00E94308FA3
:10BA1000A12CC12CD12CE12CF12C08E413E420E062
:10BA200030E0A90163EB7DE08CE69EE29BDE809135
:10BA30000E08882309F47DCF0F900F900F900F9080
:10BA4000DF91CF911F910F91FF90EF90DF90CF90FA
:10BA5000BF90AF909F900895AF92CF92DF92EF92F8
:10BA6000FF920F931F93CF93DF9361E081E00E94D9
:10BA7000AC85D0914208C0E0D1111AC08091410834
:10BA8000811104C00E943B8F811103C18091270264
:10BA9000882309F4F5C081E090914108911180E07C
:10BAA00004E024E042E55EE26C2F0E940D51E8C004
:10BAB000D13029F580914108813021F40E943B8FDB
:10BAC0008111EFC080912702882309F4D9C011E0C9
:10BAD00080914108813009F010E06091E910709187
:10BAE000EA108091EB109091EC10A2DC00E09C0138
:10BAF00044E45EE26C2F812F0E943C51C1C0D230E1
:10BB000029F580914108823021F40E943B8F8111F8
:10BB1000E2C080912702882309F4B2C011E080912D
:10BB20004108823009F010E06091ED107091EE1044
:10BB30008091EF109091F0107BDC00E09C0146E3D7
:10BB40005EE26C2F812F0E943C519AC0D33029F5C0
:10BB500080914108833021F40E943B8F8111D5C030
:10BB600080912702882309F48BC011E0809141085D
:10BB7000833009F010E06091F1107091F210809123
:10BB8000F3109091F41054DC00E09C0148E25EE276
:10BB90006C2F812F0E943C5173C0D43029F58091C5
:10BBA0004108843021F40E943B8F8111C8C08091EC
:10BBB0002702882309F464C011E080914108843091
:10BBC00009F010E06091F5107091F6108091F71077
:10BBD0009091F8102DDC00E09C014AE15EE26C2FB0
:10BBE000812F0E943C514CC0D53029F580914108ED
:10BBF000853021F40E943B8F8111BBC080912702C8
:10BC0000882309F43DC011E080914108853009F096
:10BC100010E06091051170910611809107119091CB
:10BC2000081106DC00E09C0140E15EE26C2F812FF0
:10BC30000E943C5125C0D63019F5809141088630CC
:10BC400021F40E943B8F8111ADC08091270288238F
:10BC5000B9F011E080914108863009F010E0609160
:10BC6000091170910A1180910B1190910C11E0DB78
:10BC700000E09C014CEF5DE26C2F812F0E943C5153
:10BC8000CF5FDF5FC53009F0F7CE87E080934008D3
:10BC9000A1C00E94248580910E08882309F4F6CE65
:10BCA00099C081E00E94308FA12CC12CD12CE12CB5
:10BCB00010ECF12E09E714E420E030E040E85FE307
:10BCC00069EE70E18BE49EE24DDD80910E088823E1
:10BCD00009F4F8CE7FC081E00E94308FA12CC12CE6
:10BCE000D12CE12C10ECF12E09E714E420E030E037
:10BCF00040E85FE36DEE70E18DE39EE233DD80911D
:10BD00000E08882309F405CF65C081E00E94308FBA
:10BD1000A12CC12CD12CE12C10ECF12E09E714E45C
:10BD200020E030E040E85FE361EF70E18FE29EE207
:10BD300019DD80910E08882309F412CF4BC081E0F1
:10BD40000E94308FA12CC12CD12CE12C10ECF12EB3
:10BD500009E714E420E030E040E85FE365EF70E1DC
:10BD600081E29EE2FFDC80910E08882309F41FCF58
:10BD700031C081E00E94308FA12CC12CD12CE12C4C
:10BD800010ECF12E09E714E420E030E0A90165E0B1
:10BD900071E185E19EE2E6DC80910E08882309F4DA
:10BDA0002DCF18C081E00E94308FA12CC12CD12C46
:10BDB000E12C10ECF12E09E714E420E030E0A901B9
:10BDC00069E071E186E09EE2CDDC80910E08882377
:10BDD00009F43BCFDF91CF911F910F91FF90EF902E
:10BDE000DF90CF90AF900895AF92CF92DF92EF9215
:10BDF000FF920F931F93CF93DF9361E081E00E9446
:10BE0000AC85D0914208C0E0D1111AC080914108A0
:10BE1000811104C00E943B8F8111B4C08091270220
:10BE2000882309F4A7C081E090914108911180E036
:10BE300004E024E04CE15DE26C2F0E940D519AC0B9
:10BE4000D13029F580914108813021F40E943B8F47
:10BE50008111A0C080912702882309F48BC011E0D2
:10BE600080914108813009F010E06091D910709103
:10BE7000DA108091DB109091DC10DADA00E09C019E
:10BE800048E05DE26C2F812F0E943C5173C0D2309C
:10BE900029F580914108823021F40E943B8F811165
:10BEA00095C080912702882309F464C011E0809135
:10BEB0004108823009F010E06091DD107091DE10D1
:10BEC0008091DF109091E010B3DA00E09C0144EF24
:10BED0005CE26C2F812F0E943C514CC0D33029F57D
:10BEE00080914108833021F40E943B8F81118AC0E8
:10BEF00080912702882309F43DC011E08091410818
:10BF0000833009F010E06091E1107091E2108091AF
:10BF1000E3109091E4108CDA00E09C0140EE5CE2CA
:10BF20006C2F812F0E943C5125C0D43019F580918F
:10BF30004108843021F40E943B8F81117FC08091A1
:10BF400027028823B9F011E080914108843009F07C
:10BF500010E06091E5107091E6108091E7109091EB
:10BF6000E81066DA00E09C014CEC5CE26C2F812F5B
:10BF70000E943C51CF5FDF5FC53009F045CFC093D1
:10BF8000400877C00E94248580910E08882309F418
:10BF900045CF6FC081E00E94308FA12C63EBC62E8D
:10BFA00069E5D62EE12C1CE3F12E0CE116E420E02D
:10BFB00030E040EA50E469ED70E182E19DE2D2DBDD
:10BFC00080910E08882309F445CF53C081E00E9478
:10BFD000308FA12C43EBC42E49E5D42EE12C1CE379
:10BFE000F12E0CE116E420E030E040EA50E46DED83
:10BFF00070E18EEF9CE2B6DB80910E08882309F495
:10C0000050CF37C081E00E94308FA12C23EBC22E8D
:10C0100029E5D22EE12C1CE3F12E0CE116E420E000
:10C0200030E040EA50E461EE70E18AEE9CE29ADB97
:10C0300080910E08882309F45BCF1BC081E00E9429
:10C04000308FA12C83EBC82E89E5D82EE12C1CE380
:10C05000F12E0CE116E420E030E040EA50E465EE19
:10C0600070E186ED9CE27EDB80910E08882309F466
:10C0700066CFDF91CF911F910F91FF90EF90DF90EE
:10C08000CF90AF9008959F92AF92BF92CF92DF92E0
:10C09000EF92FF920F931F93CF93DF9300D01F92E5
:10C0A000CDB7DEB761E081E00E94AC859090420898
:10C0B000B12C91101AC080914108811104C00E94D6
:10C0C0003B8F8111BFC080912702882309F4B2C041
:10C0D00081E090914108911180E004E024E04EE677
:10C0E0005DE26B2D0E940D51A5C081E0981225C024
:10C0F00080914108813021F40E943B8F8111AAC0B8
:10C1000080912702882309F495C011E080914108AD
:10C11000813009F010E06091951070919610809137
:10C1200097109091981084D900E09C014EE55DE253
:10C130006B2D812F0E943C517DC082E0981225C05A
:10C1400080914108823021F40E943B8F81119CC074
:10C1500080912702882309F46DC011E08091410885
:10C16000823009F010E06091991070919A108091DE
:10C170009B1090919C105CD900E09C014EE45DE224
:10C180006B2D812F0E943C5155C083E098122CC02A
:10C1900080914108833021F40E943B8F81118EC031
:10C1A00080912702882309F445C011E0809141085D
:10C1B000833009F010E080919D1090919E10A09125
:10C1C0009F10B091A01089839A83AB83BC83CE016A
:10C1D00001960E947CB000E09C014EE35DE26B2D75
:10C1E000812F0E943C5126C084E0981223C0809188
:10C1F0004108843021F40E943B8F81118CC08091D2
:10C2000027028823B9F011E080914108843009F0B9
:10C2100010E06091A1107091A2108091A3109091F4
:10C22000A41006D900E09C014EE25DE26B2D812F47
:10C230000E943C51B394939485E0B8123ACFB092E7
:10C24000400882C00E94248580910E08882309F44A
:10C250003ACF7AC081E00E94308FA12CC12CD12C22
:10C26000E12C10E8F12E07E714E420E030E040E88C
:10C270005FE365E970E186E69DE274DA80910E087D
:10C28000882309F43DCF60C081E00E94308FA12C4B
:10C29000C12CD12CE12C10E8F12E07E714E420E0AA
:10C2A00030E040E85FE369E970E186E59DE25ADA53
:10C2B00080910E08882309F44BCF46C081E00E948C
:10C2C000308F20E030E048EC52E460919D10709196
:10C2D0009E1080919F109091A0100F94C37B0F949B
:10C2E000F4798B010A501109A12CC12CD12C9BEAA5
:10C2F000E92E99E5F92E25EF3FE74AE050E06DE998
:10C3000070E186E49DE20E940D8480910E088823EE
:10C3100009F446CF19C081E00E94308FA12CC12CB6
:10C32000D12CE12C10E8F12E07E714E420E030E0F6
:10C3300040E85FE361EA70E186E39DE213DA809111
:10C340000E08882309F45BCF0F900F900F900F9089
:10C35000DF91CF911F910F91FF90EF90DF90CF90E1
:10C36000BF90AF909F9008952F923F924F925F920F
:10C370006F927F928F929F92AF92CF92DF92EF92C5
:10C38000FF920F931F93CF93DF9300D01F92CDB7EF
:10C39000DEB74C011B01CA01B901E982FA820B83A5
:10C3A0001C832AE037ED43E25CE30F94C37B0F94D8
:10C3B000F4792B013C012AE037ED43E25CE3F10123
:10C3C00060817181828193810F94C37B0F94F47992
:10C3D0008B01041915092AE037ED43E25CE369811A
:10C3E0007A818B819C810F94C37B0F94F4799B019C
:10C3F000241935098FE9E82E89E5F82EA201B1014B
:10C40000C4010E940D840F900F900F900F90DF9148
:10C41000CF911F910F91FF90EF90DF90CF90AF9051
:10C420009F908F907F906F905F904F903F902F9054
:10C4300008952F923F924F925F926F927F928F92C8
:10C440009F92AF92CF92DF92EF92FF920F931F9342
:10C45000CF93DF9300D01F92CDB7DEB74C011B0105
:10C46000E982FA820B831C83CA01B9010F94257AF1
:10C470002AE037ED43E25CE30F94C37B0F94F47939
:10C480002B013C01F10160817181828193810F94C4
:10C49000257A2AE037ED43E25CE30F94C37B0F94E7
:10C4A000F4798B010419150969817A818B819C814A
:10C4B0000F94257A2AE037ED43E25CE30F94C37BC7
:10C4C0000F94F4799B012419350985EAE82E89E552
:10C4D000F82EA201B101C4010E940D840F900F90AB
:10C4E0000F900F90DF91CF911F910F91FF90EF90E0
:10C4F000DF90CF90AF909F908F907F906F905F90E4
:10C500004F903F902F9008959F92AF92BF92CF92FD
:10C51000DF92EF92FF920F931F93CF93DF9300D0A0
:10C520001F92CDB7DEB761E081E00E94AC859090AC
:10C530004208B12C91101AC080914108811104C0A9
:10C540000E943B8F811152C180912702882309F4F8
:10C5500044C181E090914108911180E004E024E021
:10C560004AEE5DE26B2D0E940D5137C181E09812B9
:10C570002CC080914108813021F40E943B8F8111B1
:10C580003DC180912702882309F427C111E08091E1
:10C590004108813009F010E08091F9109091FA1073
:10C5A000A091FB10B091FC1089839A83AB83BC836C
:10C5B000CE0101960E94C4AF00E09C014EED5DE209
:10C5C0006B2D812F0E943C5108C182E098122CC033
:10C5D00080914108823021F40E943B8F811128C153
:10C5E00080912702882309F4F8C011E08091410866
:10C5F000823009F010E08091FD109091FE10A09122
:10C60000FF10B091001189839A83AB83BC83CE0164
:10C6100001960E94C4AF00E09C014AEC5DE26B2DE4
:10C62000812F0E943C51D9C083E098122CC0809188
:10C630004108833021F40E943B8F811113C1809106
:10C640002702882309F4C9C011E080914108833092
:10C6500009F010E08091011190910211A091031155
:10C66000B091041189839A83AB83BC83CE01019678
:10C670000E94C4AF00E09C0148EB5DE26B2D812F6E
:10C680000E943C51AAC084E0981228C080914108C1
:10C69000843021F40E943B8F8111FEC080912702DB
:10C6A000882309F49AC011E080914108843009F090
:10C6B00010E06091C5107091C6108091C7109091E4
:10C6C000C8100F94257A0E94425A00E09C014AEA61
:10C6D0005DE26B2D812F0E943C517FC085E0981256
:10C6E00028C080914108853021F40E943B8F811140
:10C6F000F0C080912702882309F46FC011E0809177
:10C700004108853009F010E06091C9107091CA109D
:10C710008091CB109091CC100F94257A0E94425AB0
:10C7200000E09C014CE95DE26B2D812F0E943C51A1
:10C7300054C086E0981228C080914108863021F4C8
:10C740000E943B8F8111E2C080912702882309F467
:10C7500044C011E080914108863009F010E06091FA
:10C76000CD107091CE108091CF109091D0100F9479
:10C77000257A0E94425A00E09C014EE85DE26B2D52
:10C78000812F0E943C5129C087E0981226C08091D9
:10C790004108873021F40E943B8F8111D4C08091E1
:10C7A00027028823D1F011E080914108873009F0F9
:10C7B00010E06091D1107091D2108091D3109091BF
:10C7C000D4100F94257A0E94425A00E09C0140E860
:10C7D0005DE26B2D812F0E943C51B394939485E0D0
:10C7E000B812A8CE88E080934008C9C00E94248572
:10C7F00080910E08882309F4A7CEC1C081E00E9471
:10C80000308FA12CC12CD12CE12C1CE5F12E01EC98
:10C8100017E420E030E040E251E469EF70E184EE9B
:10C820009DE2A2DD80910E08882309F4AACEA7C05C
:10C8300081E00E94308FA12CC12CD12CE12C1CE571
:10C84000F12E01EC17E420E030E048EC52E46DEF0B
:10C8500070E184ED9DE288DD80910E08882309F463
:10C86000BFCE8DC081E00E94308FA12CC12CD12C75
:10C87000E12C1CE5F12E01EC17E420E030E048EC5F
:10C8800052E461E071E181EC9DE26EDD80910E0881
:10C89000882309F4D4CE73C081E00E94308FA12C8C
:10C8A00061EBC62E69E5D62E18EBE12E12E8F12ECB
:10C8B00001E010E024E630E040E050E065EC70E19B
:10C8C00081EB9DE2B6DD80910E08882309F4E6CE67
:10C8D00056C081E00E94308FA12C41EBC42E49E567
:10C8E000D42E18EBE12E12E8F12E01E010E024E640
:10C8F00030E040E050E069EC70E183EA9DE299DDD0
:10C9000080910E08882309F4F4CE39C081E00E949A
:10C91000308FA12C21EBC22E29E5D22E18EBE12E6F
:10C9200012E8F12E01E010E02AE030E040E050E0B3
:10C930006DEC70E185E99DE27CDD80910E08882335
:10C9400009F402CF1CC081E00E94308FA12C81EB42
:10C95000C82E89E5D82E18EBE12E12E8F12E01E061
:10C9600010E024E630E040E050E061ED70E187E85F
:10C970009DE25FDD80910E08882309F410CF0F90AF
:10C980000F900F900F90DF91CF911F910F91FF901B
:10C99000EF90DF90CF90BF90AF909F9008950F934E
:10C9A000CF93DF9361E081E00E94AC85C0914208A3
:10C9B000D0E0C11118C080914108811104C00E94CB
:10C9C0003B8F8111B5C080912702882361F081E0FF
:10C9D00090914108911180E004E024E043EC5FE293
:10C9E0006D2F0E940D5180910D108770873009F0D6
:10C9F00058C0C130D9F480914108813021F40E949F
:10CA00003B8F81119DC080912702882309F4C0C00B
:10CA100081E090914108913009F080E003E02EE33D
:10CA20004CEB5FE26D2F0E940D51B2C0C230D9F4C1
:10CA300080914108823021F40E943B8F81118AC08D
:10CA400080912702882309F4A3C081E090914108D6
:10CA5000923009F080E003E02EE345EB5FE26D2FBA
:10CA60000E940D5195C0C330D1F5809141088330AB
:10CA700021F40E943B8F811177C080912702882387
:10CA800009F486C081E090914108933009F080E07C
:10CA900003E02EE34EEA5FE26D2F0E940D5184E029
:10CAA0003EC0C130F1F480914108813021F40E94F0
:10CAB0003B8F811163C080912702882309F46AC0EB
:10CAC00081E090914108913009F080E000E22EE38E
:10CAD00040EA5FE26D2F0E940D5182E020C084E0A9
:10CAE00001C082E0C8131BC0809141088C1304C0B0
:10CAF0000E943B8F811150C080912702882371F0E2
:10CB000081E0909141089C1380E003E02EE346E928
:10CB10005FE26D2F0E940D518C2F01C08C2FDF5FC3
:10CB2000CF5FD53009F045CF8F5F809340083DC07F
:10CB30000E94248580910E08882309F444CF35C0D3
:10CB400086E699E60E94175580910E08882309F41D
:10CB50005ACF2BC08BE699E60E94175580910E089C
:10CB6000882309F46DCF21C080E799E60E9417550C
:10CB700080910E08882309F480CF17C08AEA9FE2CB
:10CB80000E940B8480910E08882309F494CF0DC075
:10CB900084E0C5CF82E0C3CF85E799E60E941755B0
:10CBA00080910E08882309F4A7CFDF91CF910F91D0
:10CBB0000895CF92DF92EF92FF92CF93C82F0E94F9
:10CBC0004B326B017C0124EA30E74DE75FE3609173
:10CBD000590870915A0880915B0890915C080F94F5
:10CBE000857987FD05C04AEF50E060E070E003C042
:10CBF00040E050E0BA01C40ED51EE61EF71EC092FA
:10CC00005508D0925608E0925708F0925808C09301
:10CC10002802CF91FF90EF90DF90CF9008952F9250
:10CC20003F924F925F926F927F928F929F92AF92BC
:10CC3000BF92CF92DF92EF92FF921F93CF93DF9339
:10CC4000CDB7DEB728970FB6F894DEBF0FBECDBFC5
:10CC50001C01162F0E943B8F882329F01092700828
:10CC60000E942485DAC020916808309169083E83CB
:10CC70002D83232B09F49DC0E4E01E9FC0011124E5
:10CC800098878F83FC01E459FD4F80809180A280BA
:10CC9000B38020E030E04AE754E4C501B4010F94CA
:10CCA000AB782B013C0120E030E04AE754E4C501B9
:10CCB000B4010F94AC786B017C01809161028823F0
:10CCC000B9F1113029F198F0123091F540905902E4
:10CCD00050905A0260905B0270905C02C0905D02BE
:10CCE000D0905E02E0905F02F090600221C0409020
:10CCF000490250904A0260904B0270904C02C090E2
:10CD00004D02D0904E02E0904F02F090500210C0C1
:10CD10004090510250905202609053027090540221
:10CD2000C0905502D0905602E0905702F090580201
:10CD30002D813E81B901330F880B990B0F94277A0F
:10CD40002091590830915A0840915B0850915C0835
:10CD50000F94C37B9B01AC01C501B4010F94AC7867
:10CD6000EF81F885E459FD4F5F0160837183828311
:10CD700093832D813E8137FF0CC0A30192010F9454
:10CD8000857987FF11C0F5014082518262827382EA
:10CD90000BC0A70196010F94887B18162CF4F5019F
:10CDA000C082D182E282F382812F03DF81E080930F
:10CDB0002702109269081092680880912702882340
:10CDC00061F124E0129FF0011124E459FD4F8081AC
:10CDD0009181A281B38189839A83AB83BC832DEC3B
:10CDE0003CEC4CEC5DE36091590870915A088091DD
:10CDF0005B0890915C080F94887B87FD05C0CE018D
:10CE000001960E9403AE05C060E2CE0101960E9429
:10CE10007BAEBC01C1010E94985128960FB6F894D0
:10CE2000DEBF0FBECDBFDF91CF911F91FF90EF907E
:10CE3000DF90CF90BF90AF909F908F907F906F903A
:10CE40005F904F903F902F90089560E08BE390E3C8
:10CE5000E6CE61E084E390E3E2CE62E08DE290E32F
:10CE6000DECECF93DF9300D01F92CDB7DEB70E9406
:10CE70003B8F882329F0109270080E94248557C0A8
:10CE800060916808709169086115710569F1072E54
:10CE9000000C880B990B0F94277A20915908309138
:10CEA0005A0840915B0850915C080F94C37B9B012A
:10CEB000AC01609178027091790280917A02909130
:10CEC0007B020F94AC786093780270937902809320
:10CED0007A0290937B0283E06CDE81E080932702EC
:10CEE0001092690810926808809127028823F9F04F
:10CEF00020912707309128074091290750912A0750
:10CF0000609178027091790280917A0290917B020F
:10CF10000F94AB7869837A838B839C83CE010196CF
:10CF20000E9403AEBC018CEC9FE20E9498510F90CE
:10CF30000F900F900F90DF91CF91089521E02093F3
:10CF400070086093590870935A0880935B08909317
:10CF50005C0820E040E060E070E08091250790915F
:10CF600026070C94F88460E070E080E291E4E6CF5C
:10CF700060E070E080E89FE3E1CF6DEC7CEC8CEC4E
:10CF80009DE3DCCFFF920F931F93CF93DF93F82E97
:10CF9000709326076093250761E081E00E94AC85CD
:10CFA000D0914208C0E091E081E0F81659F1F816FE
:10CFB00028F082E0F81609F449C06CC0D111D3C042
:10CFC000992389F08091410818166CF02091680827
:10CFD000309169082F5F3F4F3093690820936808AC
:10CFE0008F5F8093410880912702882309F42CC128
:10CFF00000E010E021E041E066E270E38C2F0E9447
:10D00000AE5022C1D111AFC0992389F0809141085F
:10D0100018166CF020916808309169082F5F3F4F17
:10D0200030936908209368088F5F8093410880914E
:10D030002702882309F408C100E010E021E041E064
:10D040006FE170E38C2F0E94AE50FEC0D1118BC0F7
:10D05000992389F08091410818166CF02091680896
:10D06000309169082F5F3F4F30936908209368081B
:10D070008F5F8093410880912702882309F4E4C0E0
:10D0800000E010E021E041E068E170E38C2F0E94B5
:10D09000AE50DAC0409178025091790260917A02E4
:10D0A00070917B02409327075093280760932907CC
:10D0B00070932A07D11122C0992389F080914108E9
:10D0C00018166CF020916808309169082F5F3F4F67
:10D0D00030936908209368088F5F8093410880919E
:10D0E0002702882309F4E8C000E010E021E041E0D5
:10D0F0006EE070E38C2F0E94AE50DEC083E0F81229
:10D1000032C060914E0E70914F0E8091500E9091F2
:10D11000510E2091180E211126C00F94F479209100
:10D1200036023091370262177307ECF4D130C9F43C
:10D1300080914108813021F40E943B8F81118EC083
:10D1400080912702882369F081E090914108913015
:10D1500009F080E004E024E04EEF5FE26C2F0E94D3
:10D160000D5182E072C0D130D9F4809141088130F4
:10D1700021F40E943B8F811179C08091270288237E
:10D1800009F462C081E090914108913009F080E09B
:10D1900004E024E044EF5FE26C2F0E940D5154C084
:10D1A000D230D9F480914108823021F40E943B8F23
:10D1B000811164C080912702882309F445C081E071
:10D1C00090914108923009F080E003E02EE34AEEAE
:10D1D0005FE26C2F0E940D5137C0D330D1F48091A3
:10D1E0004108833021F40E943B8F811151C080910E
:10D1F0002702882349F181E090914108933009F09A
:10D2000080E003E02EE341EE5FE26C2F0E940D51BF
:10D210001BC0D430C9F480914108843021F40E94AD
:10D220003B8F81113FC080912702882369F081E004
:10D2300090914108943009F080E003E02EE346ED40
:10D240005FE26C2F0E940D5185E0CF5FDF5F90E0C1
:10D25000C53009F0A9CE8093400832C00E942485D1
:10D2600080910E08882309F46BCF2AC00E94248580
:10D2700080910E08882309F480CF22C083EB97E6C3
:10D280000E94175580910E08882309F493CF18C087
:10D2900088EB97E60E94175580910E08882309F4C1
:10D2A000A6CF0EC08DEB97E60E94175580910E0811
:10D2B000882309F4B8CF04C083E0F812C5CF21CF8A
:10D2C000DF91CF911F910F91FF9008954FEF65E28D
:10D2D00077E680E057CE4FEF69E277E681E052CE05
:10D2E0004FEF6DE277E682E04DCE4FEF61E377E6F8
:10D2F00083E048CE0F93CF93DF9361E081E00E94FB
:10D30000AC85D0914208C0E0D1111AC0809141088B
:10D31000811104C00E943B8F8111A9C08091270216
:10D32000882309F49BC081E090914108911180E02D
:10D3300004E024E041E95FE26C2F0E940D518EC0B1
:10D34000D130D9F480914108813021F40E943B8F83
:10D35000811195C080912702882309F47FC081E064
:10D3600090914108913009F080E003E02EE347E816
:10D370005FE26C2F0E940D5171C0D230D9F48091C0
:10D380004108823021F40E943B8F811182C080913C
:10D390002702882309F462C081E09091410892300D
:10D3A00009F080E000E22EE349E75FE26C2F0E9483
:10D3B0000D5154C0D330D9F480914108833021F409
:10D3C0000E943B8F81116FC080912702882309F44E
:10D3D00045C081E090914108933009F080E000E27F
:10D3E0002EE342ED5EE26C2F0E940D5137C0D43027
:10D3F000D1F480914108843021F40E943B8F811147
:10D400005CC080912702882349F181E09091410816
:10D41000943009F080E000E22EE343EC5EE26C2FF2
:10D420000E940D511BC0D530C9F480914108853050
:10D4300021F40E943B8F81114AC0809127028823EA
:10D4400069F081E090914108953009F080E000E2B8
:10D450002EE34EEA5EE26C2F0E940D51CF5FDF5F3C
:10D46000C53009F051CF86E08093400839C00E9452
:10D47000248580910E08882309F450CF31C08FECA9
:10D4800094E60E94175580910E08882309F462CF14
:10D4900027C083E89FE20E940B8480910E088823B6
:10D4A00009F475CF1DC08FED9EE20E940B84809120
:10D4B0000E08882309F488CF13C08CE993E00E94FA
:10D4C0000B8480910E08882309F49BCF09C08FEB51
:10D4D0009EE20E940B8480910E08882309F4ADCF50
:10D4E000DF91CF910F910895FC01718360830895BE
:10D4F00064E77AE681E09BE60C9439850F931F93ED
:10D50000CF93DF9361E081E00E94AC85C091420837
:10D51000D0E081E0C11122C0882389F080914108C8
:10D5200018166CF020916808309169082F5F3F4F02
:10D5300030936908209368088F5F80934108809139
:10D540002702882309F441C000E010E020E041E018
:10D5500065EA71E38D2F0E94AE5037C0C130D1F41F
:10D5600080914108813021F40E943B8F811137C0A6
:10D5700080912702882349F181E090914108913000
:10D5800009F080E000E22EE34AE951E36D2F0E94AA
:10D590000D511BC0C230C9F480914108823021F482
:10D5A0000E943B8F811122C080912702882369F05D
:10D5B00081E090914108923009F080E000E22EE392
:10D5C00046E851E36D2F0E940D51DF5FCF5F80E091
:10D5D000D53009F09FCF83E0809340080DC0C09301
:10D5E000B70D80910E08882319F206C0C093B70DBD
:10D5F00080910E088823C1F2DF91CF911F910F9186
:10D6000008950C9403ADEF92FF920F931F93CF9365
:10D61000DF93CDB7DEB72B970FB6F894DEBF0FBE02
:10D62000CDBF7C0140912C07842F042E000C990B58
:10D6300020912D07223051F0233019F024ED31E3F1
:10D640000AC047FF06C020EE31E305C022EF31E3F8
:10D6500002C029EE31E39F934F933F932F938E01A6
:10D660000F5F1F4F1F930F930F9427824091340237
:10D67000509135024F50510997010F900F900F9024
:10D680000F900F900F904E155F050CF49A01309398
:10D69000530E2093520E80E00E94C5D8C8010E940C
:10D6A000A2862B960FB6F894DEBF0FBECDBFDF91DA
:10D6B000CF911F910F91FF90EF900895E0912C076B
:10D6C00087E1E802F0011124E65BF14F8085918546
:10D6D0009ACFAF92BF92CF92DF92EF92FF920F93C9
:10D6E0001F93CF93DF93B82E80932D0760932C0761
:10D6F00061E081E00E94AC85D0914208C0E081E009
:10D70000D1112EC0882389F08091410818166CF041
:10D7100020916808309169082F5F3F4F3093690866
:10D72000209368088F5F80934108809127028823A7
:10D7300009F494C022E0B21649F033E0B31203C0FA
:10D7400066EB71E305C066EA71E302C066EC71E363
:10D7500000E010E021E041E08C2F0E94AE507EC03E
:10D76000D130D9F480914108813021F40E943B8F5F
:10D7700081117DC080912702882309F46FC081E068
:10D7800090914108913009F080E004E024E041E309
:10D7900052E36C2F0E940D5161C0D230D9F48091B8
:10D7A0004108823021F40E943B8F811168C0809132
:10D7B0002702882309F452C081E0909141089230F9
:10D7C00009F080E000E22EE345E252E36C2F0E9474
:10D7D0000D5144C0D330D1F480914108833021F4FD
:10D7E0000E943B8F811156C0809127028823B1F19E
:10D7F00081E090914108933009F080E000E22EE34F
:10D8000049E152E36C2F0E940D5128C0D43031F50C
:10D8100080914108843021F40E943B8F811145C0E2
:10D82000809127028823D1F011E080914108843053
:10D8300009F010E020912C0737E12303F0011124B7
:10D84000E65BF14F808591850E9403AD00E09C016D
:10D850004BEF51E36C2F812F0E943C51CF5FDF5F74
:10D8600080E0C53009F04CCFC093400846C00E940C
:10D87000248580910E08882309F47CCF3EC08091D6
:10D88000340790913507BFDE80910E08882309F494
:10D890008ECF33C08091360790913707B4DE8091E8
:10D8A0000E08882309F4A0CF28C081E00E94308FA1
:10D8B00060912C0727E16203B0011124FB01E65BB4
:10D8C000F14F00851185085711096E5A714FA12C2F
:10D8D0008EE5C82E8BE6D82E98E7E92E9AE6F92E2B
:10D8E0002AEA30E048E750E08AE092E30E940D84A3
:10D8F00080910E08882309F493CFDF91CF911F9177
:10D900000F91FF90EF90DF90CF90BF90AF90089570
:10D9100060E081E0DECE8F929F92AF92BF92CF9275
:10D92000DF92EF92FF920F931F93CF93DF934C01FF
:10D930005B016A0160E085E00E94AC85D0914208FD
:10D94000F12C82E0E82ED1111AC0809127028823A1
:10D9500021F180912A02823041F0833019F46BE585
:10D9600071E305C069E471E302C06BE671E300E0B6
:10D9700010E021E041E08F2D0E94AE500EC0D1306A
:10D9800061F480912702882341F000E010E020E05C
:10D9900041E0B4018F2D0E94AE50A114B10481F07A
:10D9A000D23081F480912702882309F46EC000E010
:10D9B00010E020E041E0B5018F2D0E94AE5065C01F
:10D9C000C2E001C0C3E0C114D10491F0DC130FC068
:10D9D00080912702882351F000E010E020E041E030
:10D9E000B6018F2D0E94AE50CD2F01C0CD2FCF5F3D
:10D9F00021E030E0A114B10411F420E030E081E036
:10DA000090E0C114D10411F480E090E0820F931FE4
:10DA1000029781F0DC130DC080912702882349F022
:10DA200000E010E020E041E064E871E38F2D0E9407
:10DA3000AE50CF5FDC1314C080912702882371F0B1
:10DA400000E010E021E040E069E771E38F2D0E94E3
:10DA5000AE5060912B078F2D0E944F50E09227020D
:10DA6000F394DF5F85E0F8126ECFCF5FC09340087C
:10DA7000DF91CF911F910F91FF90EF90DF90CF90AA
:10DA8000BF90AF909F908F900895C3E0C114D104D0
:10DA900009F0ADCFADCF40E050E060E070E08EE344
:10DAA00091E339CF45E351E365E271E38CE191E322
:10DAB00032CF40E050E06CE071E383E091E32BCFA4
:10DAC00040E050E064EF70E385EE90E324CF40E067
:10DAD00050E066ED70E389EC90E31DCF4DEB50E331
:10DAE0006CEA70E38CE990E316CF40E050E06EE81A
:10DAF00070E385E890E30FCF40E050E065E770E326
:10DB000088E690E308CF40E050E06BE570E38AE5FB
:10DB100090E301CF40E050E06BE470E382E490E3F7
:10DB2000FACE611160932A0240932B07082E000C55
:10DB3000990BAA0BBB0B8C309105A0F5FC01882733
:10DB4000EA56FF4F8F4F0D940D7D82E59DE61FC075
:10DB500089E59DE61CC08CE79DE619C08EE69DE632
:10DB600016C085E79DE613C08AE89DE610C083E8ED
:10DB70009DE60DC087E69DE60AC080E69DE607C0EB
:10DB80001092B70D8EE79AE602C08BE49DE60097EF
:10DB900049F021E02093700820E040E060E070E070
:10DBA0000C94F8840C941D8580915D08882321F0E5
:10DBB000109270080E9424850C94DD4F9091D90A30
:10DBC00093FB882780F993FF06C081E090910909B3
:10DBD000911101C080E00895F1DF882339F0809130
:10DBE000D90A82FB882780F991E0892708950F934D
:10DBF000CF93DF9361E081E00E94AC85D091420831
:10DC0000C0E0D1111AC080914108811104C00E9466
:10DC10003B8F81116FC080912702882309F461C076
:10DC200081E090914108911180E004E024E042E01D
:10DC300053E36C2F0E940D5154C0D130D9F4809120
:10DC40004108813021F40E943B8F81115BC080919B
:10DC50002702882309F445C081E090914108913062
:10DC600009F080E003E02EE341EF52E36C2F0E94C5
:10DC70000D5137C0D230D1F480914108823021F467
:10DC80000E943B8F811148C080912702882349F16F
:10DC900081E090914108923009F080E003E02EE3AA
:10DCA00043EE52E36C2F0E940D511BC0D530C9F4D6
:10DCB00080914108853021F40E943B8F811136C04C
:10DCC00080912702882369F081E090914108953086
:10DCD00009F080E003E02EE34DED52E36C2F0E944B
:10DCE0000D51CF5FDF5FC53009F08BCF86E08093A9
:10DCF000400824C00E94248580910E08882309F4DE
:10DD00008ACF1CC084ED9DE60E94175580910E08B5
:10DD1000882309F49CCF12C082EB94E70E94175528
:10DD200080910E08882309F4AFCF08C08DE295E5F5
:10DD30000E94175580910E08882311F2DF91CF9130
:10DD40000F91089540E061E080E0EBDE89E293E32B
:10DD50000F9438680D942F1B3FDF882321F085E254
:10DD600093E30F9438680C9492D31092811A109216
:10DD700092028091D90A80628093D90A0E949AD334
:10DD80006FEF87E193E30E9429910C941D850F9317
:10DD9000CF93DF9361E081E00E94AC85D09142088F
:10DDA000C0E08C2F8D0FC9F480914108811104C00F
:10DDB0000E943B8F811133C080912702882341F15B
:10DDC00081E090914108911180E004E024E042E17B
:10DDD00053E36C2F0E940D511BC08130C9F4809118
:10DDE0004108813021F40E943B8F81111FC0809136
:10DDF0002702882369F081E090914108913009F071
:10DE000080E000E22EE347E053E36C2F0E940D51C7
:10DE1000CF5FC53031F682E0809340080CC00E948D
:10DE2000248580910E08882339F205C09EDF8091F9
:10DE30000E088823E1F2DF91CF910F910895EF92C0
:10DE4000FF920F931F93CF93DF9361E081E00E94D5
:10DE5000AC85C091420810E0C11118C08091410802
:10DE6000811104C00E943B8F81118BC180912702D8
:10DE7000882361F081E090914108911180E004E0F5
:10DE800024E041ED52E3612F0E940D518091D90AA7
:10DE900082FBDD27D0F982FD06C0D1E09091741A93
:10DEA000913009F0D0E083FBEE24E0F883FF03C05B
:10DEB00085DEF82E01C0F12CDD2309F458C0C130F5
:10DEC000D9F480914108813021F40E943B8F811167
:10DED00060C180912702882309F46CC181E0909190
:10DEE0004108913009F080E000E22EE345EC52E376
:10DEF000612F0E940D515EC1C230D9F4809141085A
:10DF0000823021F40E943B8F81114AC18091270207
:10DF1000882309F44FC181E090914108923009F0C3
:10DF200080E003E02EE34AEB52E3612F0E940D51A3
:10DF300041C1C33009F047C080914108833021F4CA
:10DF40000E943B8F811138C180912702882309F4F8
:10DF500031C181E090914108933009F080E003E005
:10DF60002EE345EB52E3612F0E940D5123C18091B6
:10DF7000741A823029F030DE811102C0D1E004C071
:10DF8000C13009F423C1D2E0CD131BC080914108F8
:10DF90008C1304C00E943B8F81113AC180912702EB
:10DFA000882371F081E0909141089C1380E003E0A8
:10DFB0002EE34FE952E3612F0E940D51DC2F01C087
:10DFC000DC2FDF5F01C0D4E0CD131BC0809141087E
:10DFD0008C1304C00E943B8F811124C180912702C1
:10DFE000882371F081E0909141089C1380E003E068
:10DFF0002EE343E952E3612F0E940D51DC2F01C053
:10E00000DC2F81E08D0FC81318C0809141088C135C
:10E0100004C00E943B8F81110FC180912702882389
:10E0200061F081E0909141089C1380E003E02EE3D1
:10E0300045E852E3612F0E940D5182E08D0F40911F
:10E04000520E5091530E9091180E911107C02091CD
:10E0500036023091370242175307DCF0C81333C041
:10E06000809141088C1304C00E943B8F8111EEC047
:10E0700080912702882339F181E0909141089C1317
:10E0800080E000E22EE34DE652E3612F0E940D5145
:10E090001AC0C81318C0809141088C1304C00E9494
:10E0A0003B8F8111DDC080912702882361F081E0E0
:10E0B000909141089C1380E003E02EE34DE552E38C
:10E0C000612F0E940D51DD5FCD1318C08091410872
:10E0D0008C1304C00E943B8F8111CCC08091270219
:10E0E000882361F081E0909141089C1380E003E077
:10E0F0002EE34FE452E3612F0E940D5191E09D0FFA
:10E10000EE20E9F0F11035C0C91331C0809141080B
:10E110008C1304C00E943B8F8111B6C080912702EE
:10E12000882329F181E0909141089C1380E003E06D
:10E130002EE341E452E3612F0E940D5118C0C91330
:10E1400016C0809141088C1302C00E943B8F8091C1
:10E150002702882361F081E0909141089C1380E0C0
:10E1600000E22EE346E352E3612F0E940D5192E05C
:10E170009D0F1F5FCF5F153009F06ECE9093400862
:10E180008CC00E94248580910E08882309F46ECEED
:10E1900084C0D8DD80910E08882309F49ACE7DC012
:10E1A00087EC9EE60E94175580910E08882309F49B
:10E1B000ADCE73C0D4E025CF8BE192E70E94175516
:10E1C00080910E08882309F4BFCE67C08091410872
:10E1D000813021F40E943B8F811112C0809127026F
:10E1E0008823A1F081E090914108913009F080E00E
:10E1F00000E22EE348EA52E3612F0E940D5106C06F
:10E20000ABDD80910E08882349F347C0D2E0D9CE18
:10E210008AE799E60E94175580910E08882309F431
:10E22000BDCE3BC086EE95E70E94175580910E0843
:10E23000882309F4D3CE31C088EC92E80E941755A8
:10E2400080910E08882309F4E8CE27C08DE792E379
:10E250000E940B8480910E08882309F409CF1DC009
:10E2600088E89CE60E94175580910E08882309F4DF
:10E270001ACF13C087EF9DE60E94175580910E08B4
:10E28000882309F42BCF09C08EE196E50E9417552B
:10E2900080910E08882309F441CFDF91CF911F911F
:10E2A0000F91FF90EF9008956091480E70E080E02C
:10E2B0000C9415D46091800270918102072E000C9D
:10E2C000880B990B0F94277A2AE037ED43E25CE341
:10E2D0000F94C37B60937C0270937D0280937E02D7
:10E2E00090937F020895FC016083089580E00C9470
:10E2F000C5D863E771E78FE791E70C9439850C94F3
:10E300006BACEF92FF920F931F93CF93DF9300D0EC
:10E310001F92CDB7DEB7082F7B010E943B8F882369
:10E3200029F0109270080E9424853FC0409168082F
:10E33000509169084115510571F0109269081092C9
:10E34000680881E080932702052E000C660B770B8E
:10E35000802F0E940CB980912702882331F184E03C
:10E36000089F800111240B551F4E6091A10D7091E3
:10E37000A20D072E000C880B990B0F94277A9B0196
:10E38000AC01F80160817181828193810F94C37B1C
:10E3900069837A838B839C8360E2CE0101960E941D
:10E3A00013AFBC01C7010E9498510F900F900F90BE
:10E3B0000F90DF91CF911F910F91FF90EF900895F3
:10E3C00068EA73E380E09DCF6DE973E381E099CF64
:10E3D00020E040E060E070E00E94F88481E08093FB
:10E3E00070081092A20D1092A10D089580EE91E791
:10E3F000EFCF84EE91E7ECCFAF92CF92DF92EF9226
:10E40000FF920F931F936801DB01ED91FC918F0147
:10E41000041B150B241B350BAE2CE8E7EE2EEAE6A9
:10E42000FE2E0E940D841F910F91FF90EF90DF90C0
:10E43000CF90AF900895AF92CF92DF92EF92FF927C
:10E440000F931F93CF93DF9361E081E00E94AC852F
:10E45000D0914208C0E0D1111AC0809141088111C9
:10E4600004C00E943B8F811121C180912702882323
:10E4700009F413C181E090914108911180E004E01A
:10E4800024E048E953E36C2F0E940D5106C1D130BE
:10E4900011F580914108813021F40E943B8F811158
:10E4A0000DC180912702882309F4F7C011E0809103
:10E4B0004108813009F010E0809166029091670276
:10E4C0000E9403AD00E09C014CE853E36C2F812FC8
:10E4D0000E943C51E2C0D23011F580914108823057
:10E4E00021F40E943B8F8111FBC080912702882379
:10E4F00009F4D3C011E080914108823009F010E0A6
:10E500008091520E9091530E0E9403AD00E09C0149
:10E510004EE753E36C2F812F0E943C51BEC0D33095
:10E5200011F580914108833021F40E943B8F8111C5
:10E53000ECC080912702882309F4AFC011E08091DC
:10E540004108833009F010E080912E0E90912F0E3B
:10E550000E9403AD00E09C0146E753E36C2F812F3E
:10E560000E943C519AC0D43001F58091410884301A
:10E5700021F40E943B8F8111DDC080912702882306
:10E5800009F48BC011E080914108843009F010E05B
:10E590008091480E0E946BAC00E09C0142E653E380
:10E5A0006C2F812F0E943C5178C0D53011F580919D
:10E5B0004108853021F40E943B8F8111DAC080919F
:10E5C0002702882309F469C011E080914108853051
:10E5D00009F010E080918002909181020E9403ADC9
:10E5E00000E09C0148E553E36C2F812F0E943C51D1
:10E5F00054C0D630D9F480914108863021F40E946D
:10E600003B8F8111C8C080912702882309F445C03F
:10E6100081E090914108963009F080E003E02EE31C
:10E620004DE453E36C2F0E940D5137C0D730D1F425
:10E6300080914108873021F40E943B8F8111B5C041
:10E6400080912702882349F181E090914108973019
:10E6500009F080E003E02EE342E453E36C2F0E94D4
:10E660000D511BC0D830C9F480914108883021F485
:10E670000E943B8F8111A3C080912702882369F0FB
:10E6800081E090914108983009F080E003E02EE3AA
:10E6900043E353E36C2F0E940D51CF5FDF5FC53022
:10E6A00009F0D9CE89E08093400892C00E94248569
:10E6B00080910E08882309F4D8CE8AC0E12C00E0AE
:10E6C00010E027EE33E04AE050E066E672E082E9CF
:10E6D00093E392DE80910E08882309F4E2CE78C09D
:10E6E00081E00E94308FE12C06E711E722E231E061
:10E6F00040E050E062E57EE085E893E37DDE8091D6
:10E700000E08882309F4F1CE63C081E00E94308FA7
:10E71000E12C02E119ED2CE830E040E050E06EE23F
:10E720007EE08AE793E368DE80910E08882309F48F
:10E7300000CF4EC081E00E94308F0091480E10E063
:10E74000A12C84E5C82E81E7D82E99E7E92E91E720
:10E75000F92E2FEF30E040E050E068E47EE08CE6F8
:10E7600093E30E940D8480910E08882309F405CF5D
:10E770002FC0E12C0AE511E727EE33E04AE050E034
:10E7800060E872E08DE593E337DE80910E08882320
:10E7900009F415CF1DC086EF91E70E9417558091AF
:10E7A0000E08882309F42FCF13C089EF91E70E9448
:10E7B000175580910E08882309F442CF09C082E1E1
:10E7C00096E80E94175580910E08882309F454CFCB
:10E7D000DF91CF911F910F91FF90EF90DF90CF903D
:10E7E000AF9008954F925F926F927F92AF92BF92D7
:10E7F000CF92DF92EF92FF92CF93DF93EB01FC0178
:10E8000060817181828193812CE3C22ED12CE12C15
:10E81000F12CA70196010F94CF7CB62EA72ECA012A
:10E82000B901A70196010F94CF7C6B017C01CA014D
:10E83000B90128E130E040E050E00F94CF7C2B019B
:10E840003C01C9016DE671E00F94A87C611571056A
:10E85000D9F0AF92BF92DF92CF925F924F929F9387
:10E860008F937F936F938BED93E39F938F93DF93BE
:10E87000CF930F9427828DB79EB70E960FB6F8945C
:10E880009EBF0FBE8DBF61C00097C9F0AF92BF920F
:10E89000DF92CF925F924F929F938F938BEC93E393
:10E8A0009F938F93DF93CF930F942782EDB7FEB79B
:10E8B0003C960FB6F894FEBF0FBEEDBF46C04114A4
:10E8C000510461047104B9F0AF92BF92DF92CF920C
:10E8D0005F924F928FEB93E39F938F93DF93CF934E
:10E8E0000F9427828DB79EB70A960FB6F8949EBFF5
:10E8F0000FBE8DBF2AC0C114D104E104F104A9F0F8
:10E90000AF92BF92DF92CF9287EB93E39F938F9367
:10E91000DF93CF930F942782EDB7FEB738960FB6EB
:10E92000F894FEBF0FBEEDBF10C0AF92BF9283EB55
:10E9300093E39F938F93DF93CF930F9427820F904E
:10E940000F900F900F900F900F90DF91CF91FF904D
:10E95000EF90DF90CF90BF90AF907F906F905F90DF
:10E960004F9008952F923F924F925F926F927F92B5
:10E970008F929F92AF92BF92CF92DF92EF92FF92CF
:10E980000F931F93CF93DF93CDB7DEB76F970FB67B
:10E99000F894DEBF0FBECDBF0E943B8F882319F0D5
:10E9A0000E942485F1C02090750E3090760E8091E3
:10E9B000770E9091780E9F8F8E8F8091790E909127
:10E9C0007A0EA0917B0EB0917C0E8A8F9B8FAC8FBC
:10E9D000BD8F40907D0E50907E0E60907F0E7090A7
:10E9E000800E8090810E9090820EA090830EB09049
:10E9F000840E60E085E00E94AC85E0904208F12C36
:10EA0000DE0111966D01E1100DC08091270288236F
:10EA1000E1F0C1010E9439AD8C0120E040E060E4EA
:10EA200074E310C0B1E0EB1210C08091270288237C
:10EA300061F08E8D9F8D0E9439AD8C0120E040E009
:10EA400064E374E38F2D0E94AE508A8D9B8DAC8D54
:10EA5000BD8D8E8B9F8BA88FB98FB601CE01469648
:10EA6000C1DE92E0E9120BC0809127028823B1F049
:10EA700000E010E020E040E062E274E30CC0A3E0BC
:10EA8000EA120CC080912702882341F0860120E021
:10EA900040E06FE174E38F2D0E94AE504E8A5F8A92
:10EAA000688E798EB601CE0146969CDEB4E0EB12FC
:10EAB0000BC0809127028823B1F000E010E020E035
:10EAC00040E06DE074E30CC085E0E8120CC080917A
:10EAD0002702882341F0860120E040E06AE074E3E9
:10EAE0008F2D0E94AE5020E030E048EC52E4C5018A
:10EAF000B4010F948C790F94F479CB016AE070E043
:10EB00000F94BC7C9F938F9320E030E04AE754E45D
:10EB1000C501B4010F948C790F94F4799F938F936E
:10EB20007F936F93A2E0B4E3BF93AF93DF92CF9252
:10EB30000F9427820FB6F894DEBF0FBECDBFB6E0AC
:10EB4000EB120BC0809127028823B1F000E010E0A7
:10EB500020E040E062EF73E30CC087E0E8120CC0F5
:10EB600080912702882341F0860120E040E06FEE8B
:10EB700073E38F2D0E94AE50F394E39495E0F91265
:10EB800042CF88E0809340086F960FB6F894DEBFBE
:10EB90000FBECDBFDF91CF911F910F91FF90EF90EE
:10EBA000DF90CF90BF90AF909F908F907F906F90AD
:10EBB0005F904F903F902F90089560E070E080E06C
:10EBC0000E9415D40E945FD90C941D85AF92CF92FC
:10EBD000DF92EF92FF920F931F93CF93DF9361E049
:10EBE00081E00E94AC85D0914208C0E0D1111AC0EA
:10EBF00080914108811104C00E943B8F8111ABC0FC
:10EC000080912702882309F474C081E09091410823
:10EC1000911180E004E024E041E854E36C2F0E946D
:10EC20000D5167C0D13011F580914108813021F438
:10EC30000E943B8F811197C080912702882309F49D
:10EC400058C011E080914108813009F010E08091B6
:10EC5000520E9091530E0E9403AD00E09C0143E7D9
:10EC600054E36C2F812F0E943C5143C0D23009F5F0
:10EC700080914108823021F40E943B8F811193C022
:10EC8000809127028823A9F111E080914108823008
:10EC900009F010E080912E0E90912F0E0E9403AD8E
:10ECA00000E09C014BE654E36C2F812F0E943C5105
:10ECB00020C0D330F1F480914108833021F40E94C8
:10ECC0003B8F811190C080912702882391F011E041
:10ECD00080914108833009F010E08091480E0E9435
:10ECE0003CAC00E09C0147E554E36C2F812F0E946F
:10ECF0003C518091520E9091530E20912E0E3091E6
:10ED00002F0E232B11F4892BE9F0D430C9F4809114
:10ED10004108843021F40E943B8F811183C080918F
:10ED20002702882369F081E090914108943009F02E
:10ED300080E000E22EE34EE454E36C2F0E940D517C
:10ED400085E001C084E0CF5FDF5FC53009F04ECFC2
:10ED5000809340086DC00E94248580910E0888230E
:10ED600009F44ECF65C081E00E94308F0091520EB1
:10ED70001091530EA12C46E7C42E41E7D42E58E73C
:10ED8000E52E5AE6F52E22E231E040E050E062E561
:10ED90007EE08AE794E30E940D8480910E08882328
:10EDA00009F44ACF45C081E00E94308F00912E0EB9
:10EDB00010912F0EA12C22E1C22E29EDD22E38E780
:10EDC000E32E3AE6F32E2CE830E040E050E06EE22D
:10EDD0007EE08FE694E30E940D8480910E088823E4
:10EDE00009F44ECF25C081E00E94308F0091480E7B
:10EDF00010E0A12C84E5C82E81E7D82E93E2E92EFD
:10EE000097E5F92E2FEF30E040E050E068E47EE037
:10EE100081E694E30E940D8480910E08882309F412
:10EE200052CF06C0CADE80910E08882309F477CF3E
:10EE3000DF91CF911F910F91FF90EF90DF90CF90D6
:10EE4000AF90089580E095E290933D0780933C0752
:10EE50008CE491E0909339078093380780EC9EEF23
:10EE600090933B0780933A079091410780E2890F86
:10EE7000863740F080EF890F20E431E030933B0784
:10EE800020933A0710923E0780933F078FEF8093BD
:10EE9000400708956F927F929F92AF92BF92CF9258
:10EEA000DF92EF92FF920F931F93CF93DF931F9206
:10EEB000CDB7DEB7B9D7882309F4D2C180916808ED
:10EEC000863214F085E202C087FD80E0282F082EEC
:10EED000000C330B3093690820936808982F990F22
:10EEE000890F8093410780919107882309F4B8C165
:10EEF00020913A0730913B0700913E0710913F0760
:10EF0000020F131FE0903C07F0903D0780913807F7
:10EF100090913907E80EF91E01304FE7140768F0A9
:10EF200031952195310930933B0720933A076CEDD9
:10EF300070E085E090E00F948573F7FE15C0809136
:10EF400038079091390791958195910990933907E8
:10EF50008093380768E171E085E090E00F94857355
:10EF600081E08093400717C081E0E81680E4F8064E
:10EF700094F06BE470E084EF91E00F9485738091DE
:10EF80004B07815080934B07882311F05BDF68C1EA
:10EF90001092910765C12091380730913907C70158
:10EFA0009A508130934108F094C08F2D992787FDA6
:10EFB0009A950A9765E070E00F94BC7C812F17FF4B
:10EFC00002C087E0810F482F45954595459581E022
:10EFD00090E002C0880F991F4A95E2F7FB01EE0FFF
:10EFE000FF1FEE5BF84F40815181DC01A423B52364
:10EFF000AB2B09F419C180959095842395239183B7
:10F00000808384E090E0861B970B4091920750919B
:10F010009307840F951F9093930780939207809195
:10F020004A07815080934A07811103C082E0809390
:10F030009107932F9095991F9927991F80914007C9
:10F04000881F8827881F9817F1F03195219531097D
:10F05000309339072093380720E130E040E050E05A
:10F0600060EF7FEF8FEF9FEF0E94CD3C20913A073A
:10F0700030913B07620F731F70933B0760933A0711
:10F0800060E773E021C080913A0790913B0791952A
:10F090008195910990933B0780933A0720E130E0F6
:10F0A00040E050E060EF7FEF8FEF9FEF0E94CD3C9C
:10F0B0002091380730913907620F731F7093390719
:10F0C0006093380760E872E085E090E00F94857304
:10F0D000ABC0121613060CF0A7C0FDE3FF1A41E007
:10F0E000E41642E0F40608F09FC080914107181B27
:10F0F000103108F099C031952195310930933907C5
:10F100002093380760E773E083E090E00F94857305
:10F110008FEF8093400721E012300CF020E08EEF5B
:10F12000810F8C30A0F080913A0790913B0741E02D
:10F1300050E01816190614F040E050E030E0421795
:10F14000530709F055C091958195910927C0143056
:10F1500050F520E030E0A90160EC7FEF8FEF9FEFEA
:10F160000E94CD3C20913A0730913B07620F731FFC
:10F1700070933B0760933A0761157E4F34F480E04B
:10F180009EEF90933B0780933A0780913A079091C6
:10F190003B078130924064F180E092E090933B071E
:10F1A00080933A0725C01C301CF120E430E040E099
:10F1B00050E060E070E0CB010E94CD3C20913A0726
:10F1C00030913B07620F731F70933B0760933A07C0
:10F1D00061157E4F34F480E09EEF90933B0780935F
:10F1E0003A0780913A0790913B0781309240A4F60C
:10F1F000809191078230C1F480E480934A078FEFB9
:10F200009FEF909343078093420790934507809325
:10F21000440790934707809346079093490780934C
:10F22000480781E08093910720913E0730913F0786
:10F2300080913A0790913B07820F931F90933F076D
:10F2400080933E0720913C0730913D07809138071D
:10F2500090913907820F931F90933D0780933C074D
:10F2600061E08AEE95E00E94643780911E068E313F
:10F2700030F080911E068E3308F458C05CC0809137
:10F2800020068A30B0F382E4E82E87E0F82E9AE078
:10F29000692E712CAA24A394B12C962C80911E0661
:10F2A00090E093012C5F3F4F281739075CF442E050
:10F2B000E40EF11C85E0680E711CEEE16E1671041F
:10F2C00061F7D7CF80912006861588F330E0C12CF6
:10F2D000D12CF70180819181A5010C2C02C0440F33
:10F2E000551F0A94E2F784239523892B39F4FFEF05
:10F2F000CF1ADF0A385F303861F7D9CF00E010E06D
:10F30000A801460D571D80911E0690E04817590729
:10F310003CF08091200690E0841795070CF057C0D0
:10F320000F5F1F4F0430110559F7E1CF8091200680
:10F330008C3308F057C0809191078823B1F08091F9
:10F340003D07482F582F550F550B9A0133272F5F34
:10F350003F4F80911E0690E0281739073CF08091BE
:10F360002006841708F04FC001C077D580911E0693
:10F370008B30D0F469E080E00E94114C80919207BC
:10F38000909193070E94164C69E08EE60E94114C02
:10F3900020914B0783E090E0821B91096FEF7FEF94
:10F3A0008A579B4C0E946E4C0E943B8F8823A1F190
:10F3B0000F90DF91CF911F910F91FF90EF90DF9011
:10F3C000CF90BF90AF909F907F906F9083C527E0C4
:10F3D000492D400F632F8AEE95E039830E947539DD
:10F3E00039819ECF20E14DE3609141078AEE95E09F
:10F3F0000E94753920E14CE3609141078AEE95E067
:10F400000E94753998CF60913F0702E022E08AEEB2
:10F4100095E00E94B639AACF0F90DF91CF911F914E
:10F420000F91FF90EF90DF90CF90BF90AF909F90A3
:10F430007F906F9008956AE477E782E03AD588E399
:10F440008093410783E080934B0780E480934A07D1
:10F45000E2E4F7E011821082138212821582148294
:10F4600017821682EFDC82E190E090936908809326
:10F47000680808951F93CF93DF93F0916407CFE559
:10F48000D7E020E030E090E080E0E22F69912F5F4C
:10F490003F4F6111F22F862BE295E07F40E050E074
:10F4A00070E0DB01042E02C0B595A7950A94E2F73F
:10F4B000A0FF08C0A92FB0E0A05BB84F1E2F142BEF
:10F4C0001C939F5F4F5F5F4F4530510551F72330CD
:10F4D0003105D9F6F093640740E050E020E090E079
:10F4E000BC01042E02C0759567950A94E2F760FF8F
:10F4F00005C0209366072AE335E007C02E504F5F12
:10F500005F4F4530510561F7F4CF422F315088F0FD
:10F51000225FBC01032E02C0759567950A94E2F73D
:10F5200060FFF3CF4093650780916307823069F4F1
:10F5300003C020936507F8CF80916707181614F071
:10F540008CEF01C084E080936707DF91CF911F911A
:10F55000089580E090E0FC01E659F84F128203968E
:10F560008E319105C1F70895109269078AE0809362
:10F57000680783E0809367078FE080936307EFE578
:10F58000F7E08FE180838183828374DFE2CF1F9372
:10F59000CF93DF93EC01162FDCDF80918E078093F1
:10F5A0008B0787E380938C0786E080938D076AE062
:10F5B00070E088EE93E00F94857390918F079150DF
:10F5C00090938F07992351F010928A071883109215
:10F5D0008E07109269081092680801C01882DF91A6
:10F5E000CF911F9108955F926F927F928F929F9219
:10F5F000AF92BF92CF92DF92EF92FF920F931F9341
:10F60000CF93DF9384E08093270280916A08882358
:10F6100009F45AC280916808909169088E31910569
:10F6200014F08DE190E097FF02C080E090E09093AD
:10F63000690880936808880F991F880F991F209187
:10F640008E07422F022E000C550B4817590774F4F1
:10F650002D5FAC01421B510927FD539542305105E6
:10F660001CF020938E0702C080938E0720918E0796
:10F67000422F022E000C550B841795077CF4235063
:10F68000422F022E000C550B481B590B42305105DE
:10F690001CF020938E0702C080938E078091910703
:10F6A000882309F411C220914E07222349F090913A
:10F6B0004F07920F90934F07933F14F410924E0709
:10F6C000823070F0815080939107823011F44CDFCA
:10F6D000FBC1843609F0F8C181E080939107F4C141
:10F6E00080914D078F5F80934D074091630790E0B5
:10F6F000242F30E035952795281739070CF0ACC03A
:10F7000090914C0781E0892780934C0710924D0718
:10F71000442309F4A1C09091670780916907890F7C
:10F7200020916607821724F0209165072817D4F4EA
:10F73000919590936707209168072B5F2093680746
:10F7400080936907809164073AE08302C001112425
:10F75000820F911D27FD9A95C99724F064E181E9F4
:10F7600097E015DF9091690780916707890F809373
:10F77000690780916307882309F46EC024E130E0B3
:10F7800040E050E060E070E0CB010E94CD3C672B90
:10F79000682B692B09F060C0ECE6F7E0C0E0D0E030
:10F7A0008081811153C0CE01880F991FC80FD91FC6
:10F7B000C659D84F209709F44FC02091630730E015
:10F7C0002F5F3F4F032E000C440B550B60E070E0A1
:10F7D000CB010E94CD3CFB01E05BF84F4081242F20
:10F7E00030E0A4E035952795AA95E1F7F901EF54AB
:10F7F000FB4F808190E04F70509169076EE0469F0B
:10F80000500D1124452FFC01E255FB4F5081450F4F
:10F81000FC01E555FB4F90819695842F890F8883D5
:10F820008091680782502F5F3F4F7AE0279F800DBD
:10F830001124898322E030E040E050E060E070E095
:10F84000CB010E94CD3C6E5F6A8306C02196339641
:10F85000CA30D10509F0A4CF90918A07992341F0CD
:10F8600080918907890F8093890787FD10928A0705
:10F8700080918A07882309F495C020918907E09137
:10F8800068072E170CF48EC0022E000C330B0E2EC0
:10F89000000CFF0BCF014D96821793070CF482C02A
:10F8A000D0908807ED2C0D2C000CFF08C091690743
:10F8B000C7018C1B9109C7FD93956EE070E00F9412
:10F8C000BC7CD62F653008F06DC0C9018E1B9F0B24
:10F8D00002966AE070E00F94BC7C162F633008F04B
:10F8E00061C081E090E00D2E01C0880F0A94EAF714
:10F8F000462F660F550BFA01E15AF84F6081262F0B
:10F90000282309F44FC0DA01AF54BB4F2C9130E0EB
:10F910007EE0D79FC00D1124D901A255BB4FDC91C9
:10F92000DC0FDD160CF43EC0D901A555BB4FCC91C0
:10F930002C2F30E02D0F311DD7FD3A95E216F3063E
:10F940008CF510928A0780958623808383E090E06F
:10F95000841B950B2091920730919307820F931F80
:10F9600090939307809392076AE070E088E290E0BA
:10F970000F948573809168079AE0199F800D112478
:10F98000C695CD0FC550C0938B0780938C0784E03C
:10F9900080938D078091630781508093630788234C
:10F9A00021F068DDCCE6D7E011C084E180939107B7
:10F9B000D0DDF8CFFE018291890F8083803454F02E
:10F9C00018822396E7E0CA38DE07E1F09881992390
:10F9D000C1F3F0CF8733ACF3FE01329720818091E1
:10F9E0008E07281774F3022E000C330B082E000C20
:10F9F000990B0A968217930724F368E781E997E049
:10FA0000C6DDDFCF80914E07811124C024EF31E0A5
:10FA100040E050E060E070E0CB010E94CD3C672BFD
:10FA2000682B692BB9F422E030E040E050E060E060
:10FA300070E0CB010E94CD3C672B682B692B09F04D
:10FA40008DC18FEF80934E07813009F489C18FE714
:10FA500080934F0780918A078823B1F180914E07E8
:10FA6000882391F180918907873074F52091880768
:10FA700080914F07281744F1022E000C330B082EFB
:10FA8000000C990B0C9682179307F4F010924E0716
:10FA900010928A0780919207909193070A9690930B
:10FAA0009307809392076AE070E088E290E00F94F9
:10FAB000857380914F078F5F80938B0781E08093E0
:10FAC0008C0784E080938D078091720882FF04C0C8
:10FAD00080916207815001C08AE0809362070E9492
:10FAE0003B8F8823C1F080919107811103C0109250
:10FAF000620711C0813079F480918A0781110BC0AF
:10FB000080918E078B5F8093880784E380938907B9
:10FB10008CEF80938A0780916207811101C0DAD14E
:10FB200061E08AEE95E00E946437C09168074C2F2F
:10FB30000C2E000C550B809164079A01FAE08F029D
:10FB4000200D311D11242250310980911E0690E0B4
:10FB5000821793072CF080914E07811161C065C018
:10FB60008091200690E084179507ACF371EB672E27
:10FB700074E0772EEFE58E2EE7E09E2EFEE15F2EFD
:10FB80005C0EF301C1903F012C2F0C2E000C330BA7
:10FB9000A901495F5F4F80911E0690E04817590701
:10FBA0003CF4C65FFFEF8F1A9F0AC511EACFD3CF8F
:10FBB0008091200690E0821793079CF3D09169070B
:10FBC00016E41D0FA12CB12CD12CCC0CDD1CF401A2
:10FBD000808190E00A2C02C0959587950A94E2F7FF
:10FBE00080FF17C080914C077601E80EF11CC70119
:10FBF00064E0880F991F6A95E1F79C0127543B4CFC
:10FC0000790108E022E04C2F6D2F8AEE95E00E94EA
:10FC10008E37D25F3FEFA31AB30AD113D8CFC1CF2B
:10FC200080911E06883008F49DC08091910788233A
:10FC300069F090911E069F3348F490912006973307
:10FC400028F0823008F49CC081FD9AC080918A0718
:10FC50008823B1F040918907242F042E000C330B28
:10FC6000B9016D5F7F4F80911E0690E0681779079C
:10FC70003CF08091200690E0821793070CF08EC034
:10FC8000C0E0D0E0FE01E659F84F8281882399F068
:10FC90004181842F042E000C990B20911E0630E028
:10FCA0008217930744F002972091200630E028172E
:10FCB00039070CF07BC02396CE31D10519F780911E
:10FCC0008D078823B1F040918C07242F042E000C5F
:10FCD000330BB9016A5F7F4F80911E0690E0681771
:10FCE00079073CF08091200690E0821793070CF092
:10FCF00065C080919107811101C0AFD080911E062F
:10FD00008A3008F06DC069E080E00E94114C80915B
:10FD10009207909193070E94164C80918F07882339
:10FD200009F45EC0C1E040E1C42ED12C80918F0760
:10FD30008C1708F455C0B6016C1B7109660F660F6D
:10FD4000660F54EAE52E54E3F52E05E021E041E08C
:10FD50008AEE95E00E948E37CF5FE8CF81E072CEC9
:10FD600083EF76CE2CE8E22E24E3F22E05E022E0AB
:10FD700042E060914F078AEE95E00E948E3755CFA2
:10FD800099EAE92E94E3F92E08E022E047E3609136
:10FD90008E078AEE95E00E948E3758CF24E060915E
:10FDA00088078AEE95E00E9495396ACF425023E099
:10FDB00060818AEE95E00E9495397DCF86E9E82E34
:10FDC00084E3F82E07E022E060918B078AEE95E04D
:10FDD0000E948E3780918D07815080938D0789CF47
:10FDE000DF91CF911F910F91FF90EF90DF90CF9017
:10FDF000BF90AF909F908F907F906F905F9008958D
:10FE000063EF7AE784E155D083E080938F078AE03F
:10FE10008093620710928A07A7DB10928E071092D8
:10FE2000690810926808089580916A08882319F07B
:10FE300082E08093900784E080932702809191076D
:10FE4000882349F0909190078FEF890F8093900756
:10FE500081E019160CF080E008950F9380911E0642
:10FE6000853228F5809120068B3108F160E08AEE1A
:10FE700095E00E94643709E028E34BE164E28AEEF2
:10FE800095E00E94063A61E08AEE95E00E946437B0
:10FE90000E94868F882359F063E285E20E94114C0C
:10FEA0006FEF7FEF89E195E30F910C946E4C0F910A
:10FEB0000895FB0110929307109292078093910787
:10FEC00020E040E060E070E0CF0192D581E08093D7
:10FED0007008089510927008B7C5809194079091AA
:10FEE000960789130DC08091950790919707891700
:10FEF00014F02FEF01C021E0820F8093950708C016
:10FF0000891714F02FEF01C021E0820F809394072E
:10FF1000891319C02091F80721502093F80730E089
:10FF2000832F90E0DC01AA0FBB1FAC56B84F880F9F
:10FF3000991FFC01EA56F84F808191818D939C9323
:10FF40003F5F231768F70895EF92FF921F93CF93B7
:10FF5000DF931091F8072091FF07E22E022E000C8C
:10FF6000FF0830910008C32F032E000CDD0BE7E9DA
:10FF7000F7E040E0411709F446C0CF010397DC01E8
:10FF80009C91BF0161507109DB018C9198131DC0D8
:10FF9000692F092E000C770B61507109C617D7071E
:10FFA00011F039132DC09081BF0162507109DB013E
:10FFB0008C91582F98170CF4592F25170CF189178D
:10FFC0000CF4892F8217E4F020C0BF016250710940
:10FFD000DB015C91652F052E000C770B61507109D8
:10FFE000E616F70611F025130BC0582F98170CF4DE
:10FFF000592F35172CF089170CF4892F83172CF4FF
:020000021000EC
:100000004F5F3296B7CF80E001C081E0DF91CF91A2
:100010001F91FF90EF90089528E130E040E050E01C
:1000200060E070E0CB010E94CD3C609300082AE0C4
:1000300030E040E050E060E070E0CB010E94CD3C59
:100040006093FF0781DF8111E7CF08959091010848
:10005000811102C08FEF01C081E0980F93709093DF
:100060000108E091F807EF5FE093F807F0E0EE0F8A
:10007000FF1FEC56F84F8091FC0780838091FA07B0
:1000800081830895CF9380E091E09093FC07809363
:10009000FB0780E095E09093FA078093F9071092B0
:1000A00001081092F807E4E9F7E01082C5E0C18387
:1000B00081E0CCDFC093FE071092690810926808B7
:1000C0001092FD07CF910895EF92FF920F931F9327
:1000D000CF93DF938091F807843008F4B1C090E0AB
:1000E000FC01EE0FFF1FEE56F84F2081EC01CC0F04
:1000F000DD1FCC56D84F68810297261719F0F12CD6
:1001000031966BC0E12C219631964E2D50E0481768
:1001100059070CF095C0BA01660F771F8B010C567A
:10012000184FD801FC90DB01AA56B84F3C91F3164A
:10013000E9F0432FF3160CF44F2D24179CF13F15D3
:100140000CF43F2D321774F1DB01AC56B84F119609
:100150005C9141E0308153170CF040E031E0688160
:1001600065170CF430E04317E9F06CC02F111AC08A
:100170006881408111965C91D80111963C91A42F21
:1001800064170CF4A62F732F35170CF4752F7A17FC
:100190004CF046170CF4462F53170CF4352F431729
:1001A0000CF050C0E394B1CFEA01CC0FDD1F8E01FB
:1001B0000C56184FD80111967C91DE01AA56B84F03
:1001C00011963C911197731709F14081532F7317C2
:1001D0000CF4572F45173CF4F3944F2D50E048177B
:1001E000590714F32DC037170CF4372F3417A4F325
:1001F000CC56D84F588141E052170CF040E031E026
:1002000065170CF430E0431739F31CC03081371305
:10021000E3CF4C91D8013C91762F26170CF4722F26
:10022000532F34170CF4542F5717B4F2562F62176C
:100230000CF4522F43170CF4342F53176CF202C0F6
:1002400080E001C081E0DF91CF911F910F91FF907D
:10025000EF900895CF92DF92EF92FF920F931F934A
:10026000CF93DF931F92CDB7DEB7DEDD882309F48D
:1002700080C08091FB079091FC07392F4091F907CE
:100280005091FA0720910108213061F02CF42111DE
:1002900016C0CA01C3970AC0223031F0233079F466
:1002A000C39709C0C39607C0CA01C3969093FA07C3
:1002B0008093F90704C09093FC078093FB0710918B
:1002C000FC070091FA07311303C0051709F451C068
:1002D000183110F40A3048F01092910768E270E08B
:1002E00080E991E00F94857344C0E091F807F0E055
:1002F000EE0FFF1FEC56F84F1083018380916808C2
:100300009091FD07282F291B39F08093FD0781E08C
:1003100012160CF080E09ADE8091FE07882321F00F
:1003200081508093FE0701C0D8DDCEDE8111D4CF8D
:100330008091000818131DC08091FF07081319C091
:100340006CED70E085E090E00F94857368E171E0FA
:1003500085E090E00F9485738091920790919307C8
:100360000196909393078093920782E08093FE0713
:1003700053DE61E08AEE95E00E94643780911E06AC
:10038000893050F467E080E00E94114C8091920720
:10039000909193070E94164C06E32CE749E062E037
:1003A0008AEE95E00E94B639F12C8091F8072091F1
:1003B0001E06F81608F071C0EF2DF0E0AF01440FF3
:1003C000551FDA01AC56B84F9C91FA01EA56F84F26
:1003D0008081981345C091811196EC901E2DE916ED
:1003E0000CF4192F85E01802B0011124625F7F4FD1
:1003F00030E0621773070CF44EC09E150CF4E92E22
:100400009E2DE5E09E0290011124265F3F4F8091D2
:10041000200690E028173907F4F58E2D880F880FF5
:100420008E0D7BE0780FCA018C56984F6C011E151B
:1004300094F1272F072E000C330BA9014D5F5F4F5E
:1004400080911E0690E0481759073CF080912006E5
:1004500090E0821793070CF04DC0E3947B5FE7CFE9
:1004600011963C91432F440F440F340F4BE0D42E90
:10047000D30E4D2D0D2C000C550BBA016D5F7F4F27
:1004800030E0621773073CF02091200630E024171B
:1004900035070CF040C0F39488CF4091FF07842FBC
:1004A000880F880F480F455F642F042E000C770BD0
:1004B000FB013396822F90E0E817F9073CF080911A
:1004C000200690E0861797070CF044C080919107B2
:1004D000811101C0C2DC0E943B8F882309F448C00F
:1004E0000F90DF91CF911F910F91FF90EF90DF90D0
:1004F000CF90F0CCF6016081862F880F880F680FAF
:100500006C5F04E024E0472F8AEE95E079830E9437
:10051000063A7981A2CFE82E98170CF4E92EC82E5E
:1005200089170CF4C92E1E2D110F110F1E0D50E04E
:100530001C5FCE140CF4AFCF612F650F04E024E0F4
:100540004D2D8AEE95E059830E94063AE394598135
:100550005B5FEFCF60910008862F880F880F680FD0
:100560006C5F04E024E08AEE95E00E94B639AECFDD
:100570000F90DF91CF911F910F91FF90EF90DF903F
:10058000CF9008956AE271E881E093DC7BDD44CD91
:100590000F931F93CF93DF9361E081E0DDD2D09181
:1005A0004208C0E0D11117C080914108811104C0F8
:1005B0000E943B8F81119EC080912702882309F4FD
:1005C0003EC081E090914108911180E004E024E078
:1005D00042E755E331C0D130B9F480914108813010
:1005E00021F40E943B8F81118CC0809127028823C7
:1005F00031F181E090914108913009F080E003E011
:100600002EE340E655E318C0D230C9F4809141088A
:10061000823021F40E943B8F81117DC0809127029E
:10062000882369F081E090914108923009F080E0E0
:1006300003E02EE341E555E36C2F0E940D51C1D13B
:10064000182FD330D9F480914108833021F40E94CF
:100650003B8F81116AC080912702882309F478C0FA
:1006600081E090914108933009F080E000E22EE3B0
:1006700042E455E36C2F0E940D516AC081116AC09B
:10068000D430B9F480914108843021F40E943B8F2A
:10069000811152C080912702882319F181E0909145
:1006A0004108943009F080E000E22EE344E355E392
:1006B00015C0D530B1F480914108853009F443C0AC
:1006C00080912702882369F081E09091410895305C
:1006D00009F080E000E22EE343E255E36C2F0E9434
:1006E0000D5186E0CF5FDF5FC53009F05BCF8093AF
:1006F00040083BC0A9D180910E08882309F45CCF43
:1007000034C088E69AE50E94175580910E08882328
:1007100009F46BCF2AC082E196E80E9417558091B8
:100720000E08882309F47ACF20C014D380910E08D4
:10073000882309F490CF19C010D380910E08882324
:1007400009F4A8CF12C00E943B8F811105C0B8CF19
:10075000112339F284E0C6CF0E94F6FD81E04ED22B
:1007600080910E08882309F4ABCFDF91CF911F91C0
:100770000F910895FC0160830895CF93DF93EC01FE
:10078000072E000C880B990B0F94277A20E030E09D
:1007900040E251E40F94C37B0F94F9797983688325
:1007A000DF91CF9108950C9491ACBC01990F880B07
:1007B000990B0F94277A20E030E040E251E40F9447
:1007C000C37B0F94F979CB010C94C0ACE0910F0876
:1007D000E63000F581E08E0F80930F088091680865
:1007E00090916908A0E0B0E0309142082091400863
:1007F00048E0E49FF0011124E05FF74F4091630867
:10080000509164085183408382839383A483B5838A
:100810003683278308950D9438684F925F926F92C4
:100820007F928F929F92AF92CF92DF92EF92FF9240
:100830000F931F93CF93DF933C014B01EA012901F2
:10084000C5DF83E08093270270920D0860920C0848
:1008500090920B0880920A08D0930908C093080868
:1008600050920708409206081093690800936808A0
:10087000F0926408E0926308D0920508C0920408E0
:10088000A0920308DF91CF911F910F91FF90EF90FD
:10089000DF90CF90AF909F908F907F906F905F9000
:1008A0004F900895AF92CF92DF92EF92FF920F9305
:1008B0001F93680150E0DB01EC91F0E08F01041B15
:1008C000150B30E0241B350BAE2CE9E7EE2EE1E7EB
:1008D000FE2EA3DF1F910F91FF90EF90DF90CF903E
:1008E000AF9008952F923F924F925F926F927F92B6
:1008F0008F929F92AF92CF92DF92EF92FF920F93DF
:100900001F93CF93DF934C01EB016901BA0180E0A3
:1009100090E00F94257A2DEC3CEC4CEC5DE30F94C9
:10092000C37B0F94F4792B013C016881798180E0CD
:1009300090E00F94257A2DEC3CEC4CEC5DE30F94A9
:10094000C37B0F94F4791B0124183508B60180E0AD
:1009500090E00F94257A2DEC3CEC4CEC5DE30F9489
:10096000C37B0F94F4799B0124193509AE2C6801DF
:1009700087EAE82E85E8F82E8101A201BE01C401B4
:100980004CDFDF91CF911F910F91FF90EF90DF909F
:10099000CF90AF909F908F907F906F905F904F908F
:1009A0003F902F900895FB01908181E089278083FB
:1009B00083E0809327024115510511F0FA01199443
:1009C00008958091131190911011891B8F7071F40B
:1009D0009091D90A92FB882780F992FD08C081E0A6
:1009E0009091741A913019F080E0089581E0089593
:1009F000E0916308F0916408E817F907E9F0909333
:100A00006408809363087093690860936808409352
:100A10004208209340088A599E4821F41092700899
:100A200010920F080E944E5082E08093270281E0CE
:100A300080930E0810926B08089520E040E060E07B
:100A400070E08AE99EE8D4CFE0910F08EE2381F0B0
:100A5000E150E0930F0888E0E89FF0011124E05F87
:100A6000F74F2781468160E070E080819181C0CF9F
:100A7000E4CFCF93DF93FC01EB0180916808909164
:100A8000690897FF04C010926908109268082091C5
:100A90000608309107088091680890916908281726
:100AA000390724F43093690820936808809127025D
:100AB000882391F0209108083091090880916808F6
:100AC00090916908820F931F1995BC0180910C08C1
:100AD00090910D080E94985180915D08811108C085
:100AE00080910308882359F180912702882339F1E6
:100AF00080910A0890910B08009761F060910808B6
:100B0000709109082091680830916908620F731F7D
:100B1000FE011995E0910408F0910508309741F025
:100B200080910308811103C080915D08811119959E
:100B30000E943B8F882319F0DF91CF9185CFDF9101
:100B4000CF9108956AEB73E883ED93E892CF6DEB54
:100B500073E885ED93E88DCF282F1092620880917D
:100B60006808909169088130904820F010926908D7
:100B70001092680880916A08882331F08091680893
:100B80008093410810920E08809140081816BCF41A
:100B9000082E000C990B821B910920914108022E0E
:100BA000000C330B2817390754F097FF02C080E080
:100BB00090E0809341089093690880936808809141
:100BC00041086623C1F090914208891714F480937C
:100BD000420820914208022E000C330B2C5F3F4F3D
:100BE000482F082E000C550B2417350734F4845079
:100BF000809342080895809342080895882361F005
:100C000063E972E084E690E00F9485736AEB72E02A
:100C100084E690E00D94857368EB71E084E190E0E8
:100C20000D9485738F929F92AF92BF92CF92DF9275
:100C3000EF92FF920E943B8F882369F00E942CF96B
:100C400010927008FF90EF90DF90CF90BF90AF9020
:100C50009F908F90F9CE81E080937008C0906808D3
:100C6000D0906908C114D10409F444C010926908F5
:100C7000109268080D2C000CEE08FF08C701B601A1
:100C80000F94277A2091AD103091AE104091AF10A3
:100C90005091B0100F94C37B2091E50F3091E60F77
:100CA0004091E70F5091E80F0F94AC784B015C0135
:100CB00020E030E040E050EC0F94887B87FD1AC0C4
:100CC00020E030E040EA50E4C501B4010F9485799A
:100CD000181684F0B701A60182E00E940CB9809238
:100CE000E50F9092E60FA092E70FB092E80F82E036
:100CF00080932702809127028823D9F085EE9FE018
:100D00000E9465ADBC0187E795E30E949851609110
:100D1000E50F7091E60F8091E70F9091E80FFF903B
:100D2000EF90DF90CF90BF90AF909F908F900C94FA
:100D3000CF52FF90EF90DF90CF90BF90AF909F90F9
:100D40008F90089521E0209302080F943D6810923F
:100D5000020808950E9467F951CF0F94A80A4ECF58
:100D6000EF92FF920F931F93E0916808F09169084A
:100D7000309759F0A1E01E161F060CF0A0E0FA0112
:100D8000A0831092690810926808FA0140810E94BD
:100D900065521F910F91FF90EF9008956091690F38
:100DA00070916A0F86E39FE00C94523E60912E0F83
:100DB00070912F0F8BEF9EE00C94523E6091F30EDA
:100DC0007091F40E80EC9EE00C94523E6091B80E4F
:100DD0007091B90E85E89EE00C94523E8F929F92DE
:100DE000AF92BF92CF92DF92EF92FF92CF9360913A
:100DF000D9107091DA108091DB109091DC100F9473
:100E0000F9794B015C01C0916F0F86E39FE00E946E
:100E1000C73FDC0120E136E041EC50E00F94247D37
:100E20006B017C01AC2FB0E0A50194010F94247DEF
:100E30002227362F472F582FC701B6010F94CF7C9A
:100E4000BA01A9016627772786E39FE0CF91FF903B
:100E5000EF90DF90CF90BF90AF909F908F900C94C9
:100E60001B408F929F92AF92BF92CF92DF92EF92F0
:100E7000FF92CF936091DD107091DE108091DF10B2
:100E80009091E0100F94F9794B015C01C091340FFF
:100E90008BEF9EE00E94C73FDC0120E136E041EC91
:100EA00050E00F94247D6B017C01AC2FB0E0A501D4
:100EB00094010F94247D2227362F472F582FC701E6
:100EC000B6010F94CF7CBA01A901662777278BEF73
:100ED0009EE0CF91FF90EF90DF90CF90BF90AF90CA
:100EE0009F908F900C941B408F929F92AF92BF92D5
:100EF000CF92DF92EF92FF92CF936091E1107091C9
:100F0000E2108091E3109091E4100F94F9794B0175
:100F10005C01C091F90E80EC9EE00E94C73FDC01AD
:100F200020E136E041EC50E00F94247D6B017C0120
:100F3000AC2FB0E0A50194010F94247D2227362F19
:100F4000472F582FC701B6010F94CF7CBA01A901D2
:100F50006627772780EC9EE0CF91FF90EF90DF909F
:100F6000CF90BF90AF909F908F900C941B408F922A
:100F70009F92AF92BF92CF92DF92EF92FF92CF9368
:100F80006091E5107091E6108091E7109091E81063
:100F90000F94F9794B015C01C091BE0E85E89EE08B
:100FA0000E94C73FDC0120E136E041EC50E00F94A5
:100FB000247D6B017C01AC2FB0E0A50194010F945E
:100FC000247D2227362F472F582FC701B6010F94B3
:100FD000CF7CBA01A9016627772785E89EE0CF91EB
:100FE000FF90EF90DF90CF90BF90AF909F908F9049
:100FF0000C941B406091700F86E39FE00C9494402A
:101000006091350F8BEF9EE00C94944060916E0FD1
:1010100086E39FE00C940F436091330F8BEF9EE0CB
:101020000C940F436091F80E80EC9EE00C940F43FB
:101030006091BD0E85E89EE00C940F430F931F93C3
:10104000CF93DF9361E081E087DDD0914208C0E07B
:1010500081E0D11122C0882389F0809141081816BF
:101060006CF020916808309169082F5F3F4F3093F2
:101070006908209368088F5F809341088091270258
:10108000882309F4AAC000E010E020E041E068E015
:1010900076E38C2F0E94AE50A0C0D130D1F4809165
:1010A0004108813019F4E7D68111A1C0809127024F
:1010B000882309F492C081E090914108913009F0B1
:1010C00080E004E024E04CEF55E36C2F0E940D51CA
:1010D00084C0D230F9F480914108823019F4CBD623
:1010E00081118CC080912702882309F476C08091F9
:1010F0006E0F811103C023EF35E302C027EF35E304
:1011000081E090914108923009F080E001E041EFE8
:1011100055E360C0D330F9F480914108833019F46D
:10112000AAD6811178C080912702882309F455C07E
:101130008091330F811103C028EE35E302C02CEEFD
:1011400035E381E090914108933009F080E001E0BF
:1011500046EE55E33FC0D430F1F48091410884302D
:1011600019F489D6811164C0809127028823A9F1DE
:101170008091F80E811103C02DED35E302C021EE00
:1011800035E381E090914108943009F080E001E07E
:101190004BED55E31FC0D53001F5809141088530F6
:1011A00019F469D6811151C0809127028823A9F0D2
:1011B0008091BD0E811103C021ED35E302C025ED04
:1011C00035E381E090914108953009F080E001E03D
:1011D0004EEC55E36C2F0E943C51CF5FDF5F80E007
:1011E000C53009F036CF86E0809340083AC02CDC49
:1011F00080910E08882309F459CF33C046E058E89F
:101200006EE67FE08AEF95E3CEDB80910E088823BF
:1012100009F468CF26C04CE058E863E37FE08FEE26
:1012200095E3C1DB80910E08882309F47CCF19C0B7
:1012300042E158E868EF7EE084EE95E3B4DB80910C
:101240000E08882309F490CF0CC048E158E86DEBF4
:101250007EE088ED95E3A7DB80910E08882309F4F2
:10126000A3CFDF91CF911F910F910895AF92CF92AD
:10127000DF92EF92FF920F931F93CF93DF9361E082
:1012800081E06ADCD0914208C0E0D11119C08091A0
:101290004108811103C0EFD5811156C0809127020A
:1012A000882309F448C081E090914108911180E0C1
:1012B00004E024E044E256E36C2F0E940D513BC051
:1012C000D130D1F480914108813019F4D4D5811105
:1012D00042C080912702882371F111E0809141087A
:1012E000813009F010E08091700F0E9491AC00E015
:1012F0009C0140E256E31BC0D230E9F480914108E2
:10130000823019F4B8D5811145C080912702882315
:1013100091F011E080914108823009F010E0809155
:10132000350F0E9491AC00E09C014CE156E36C2F1C
:10133000812F0E943C51CF5FDF5FC53009F0A5CF00
:1013400083E08093400844C07FDB80910E088823AF
:1013500009F4A4CF3DC00091700F002E000C110BBA
:10136000005C1F4FA12C2AEFC22E27E8D22E32EAB2
:10137000E32E35E8F32E2FE730E040EC5FEF60E737
:101380007FE082E296E349DA80910E08882309F42F
:10139000A0CF1EC00091350F002E000C110B005C79
:1013A0001F4FA12C80E0C82E88E8D82E92EAE92EA3
:1013B00095E8F92E2FE730E040EC5FEF65E37FE042
:1013C0008EE196E32ADA80910E08882309F49DCFF6
:1013D000DF91CF911F910F91FF90EF90DF90CF9011
:1013E000AF9008950F93CF93DF9361E081E0B4DB7A
:1013F000D0914208C0E0D11116C0809141088111FE
:1014000003C039D581117BC080912702882309F45C
:101410006EC081E090914108911180E004E024E0E9
:1014200046EC55E361C0D130B9F480914108813078
:1014300019F421D581116AC080912702882309F40B
:1014400056C081E090914108913009F080E003E0BE
:101450002EE347EB55E348C0D230B9F48091410800
:10146000823019F408D581115BC08091270288234E
:1014700009F43DC081E090914108923009F080E08C
:1014800003E02EE346EA55E32FC0D330B1F4809158
:101490004108833019F4EFD481114CC080912702A8
:1014A000882329F181E090914108933009F080E090
:1014B00003E02EE344E955E317C0D430C1F4809132
:1014C0004108843019F4D7D481113EC0809127029D
:1014D000882369F081E090914108943009F080E020
:1014E00003E02EE346E855E36C2F0E940D51CF5FD9
:1014F000DF5FC53009F07FCFC09340082EC0A4DA6B
:1015000080910E08882309F47FCF27C081EB9AE8E9
:101510000E94175580910E08882309F48DCF1DC0B5
:1015200080EB9BE80E94175580910E08882309F4F0
:101530009CCF13C086E399E80E94175580910E084E
:10154000882309F4ABCF09C08EE198E80E941755B3
:1015500080910E08882309F4B9CFDF91CF910F91C4
:101560000895EF920F931F93CF93DF9361E081E093
:10157000F3DAD0914208C0E0D11119C0809141083E
:10158000811103C078D4811197C0809127028823EC
:1015900009F48AC081E090914108911180E004E053
:1015A00024E040E656E36C2F0E940D517DC0D130FF
:1015B000E9F480914108813019F45DD4811183C030
:1015C00080912702882309F46FC011E080914108BF
:1015D000813009F010E08091690F90916A0F0E94AC
:1015E000C0AC00E09C014CE556E35AC0D230E9F4AF
:1015F00080914108823019F43ED4811176C08091E7
:101600002702882309F450C011E0809141088230FC
:1016100009F010E080912E0F90912F0F0E94C0AC26
:1016200000E09C0148E556E33BC0D330E1F48091F3
:101630004108833019F41FD4811169C080912702B9
:10164000882391F111E080914108833009F010E086
:101650008091F30E9091F40E0E94C0AC00E09C01CA
:1016600044E556E31DC0D430F9F48091410884303C
:1016700019F401D481115DC0809127028823A1F063
:1016800011E080914108843009F010E08091B80E9B
:101690009091B90E0E94C0AC00E09C014EE456E36C
:1016A0006C2F812F0E943C51CF5FDF5FC53009F066
:1016B00063CFC09340084EC0C7D980910E088823DD
:1016C00009F463CF47C0E12C0EEC16E828EB3BE0B1
:1016D00044E650E069E67FE08EE596E303D9809129
:1016E0000E08882309F46CCF35C0E12C06ED16E80E
:1016F00028EB3BE044E650E06EE27FE08AE596E3CB
:10170000F1D880910E08882309F479CF23C0E12C09
:101710000EED16E828EB3BE044E650E063EF7EE098
:1017200086E596E3DFD880910E08882309F486CFFA
:1017300011C0E12C06EE16E828EB3BE044E650E051
:1017400068EB7EE081E596E3CDD880910E08882392
:1017500009F492CFDF91CF911F910F91EF900895EF
:10176000EF920F931F93CF93DF9361E081E0F4D961
:10177000D0914208C0E0D11119C080914108811177
:1017800003C079D381118FC080912702882309F487
:1017900082C081E090914108911180E004E024E052
:1017A00042E456E36C2F0E940D5175C0D130D9F43C
:1017B00080914108813019F45ED381117BC0809102
:1017C0002702882309F467C011E080914108813025
:1017D00009F010E080916F0F0E946BAC00E09C015B
:1017E0004EE356E354C0D230D9F4809141088230A0
:1017F00019F441D381116FC080912702882309F425
:101800004AC011E080914108823009F010E08091D7
:10181000340F0E946BAC00E09C014AE356E337C0F2
:10182000D330D1F480914108833019F424D381114D
:1018300063C080912702882371F111E080914108F3
:10184000833009F010E08091F90E0E946BAC00E04B
:101850009C0146E356E31BC0D430E9F48091410873
:10186000843019F408D3811158C08091270288234D
:1018700091F011E080914108843009F010E08091EE
:10188000BE0E0E946BAC00E09C0140E356E36C2F5F
:10189000812F0E943C51CF5FDF5FC53009F06BCFD5
:1018A000C09340084AC0D0D880910E08882309F41C
:1018B0006BCF43C0E12C0EEE16E82FEF40E06FE651
:1018C0007FE080E496E30E94528480910E08882392
:1018D00009F475CF32C0E12C01E317E82FEF40E0A7
:1018E00064E37FE08CE396E30E94528480910E08CB
:1018F000882309F481CF21C0E12C04E717E82FEFFA
:1019000040E069EF7EE088E396E30E945284809194
:101910000E08882309F48DCF10C0E12C07EB17E8DF
:101920002FEF40E06EEB7EE083E396E30E9452846B
:1019300080910E08882309F498CFDF91CF911F91F1
:101940000F91EF900895FC0180810895FC0184912E
:1019500008954F925F926F927F928F929F92AF9273
:10196000BF92CF92DF92EF92FF920F931F93CF938C
:10197000DF936C017B015A012901672B31F0882428
:101980008394912CC0E0D0E019C0F801118210823C
:1019900027C03701680C791C76946794E30121977E
:1019A000A201BE01C601F50119951816190654F0D9
:1019B000892BC9F04301FFEF8F1A9F0AE814F9043D
:1019C00040F702C07E01FACFCE15DF0530F4CE011C
:1019D00002968816990620F02196F801D183C083DB
:1019E0008FEF9FEF05C0F801D183C08380E090E0C6
:1019F000DF91CF911F910F91FF90EF90DF90CF90EB
:101A0000BF90AF909F908F907F906F905F904F901E
:101A100008958F929F92AF92BF92CF92DF92EF92F2
:101A2000FF920F931F93CF93DF93EC016B017A0129
:101A3000FB01199587FD06C0082F10E020E030E07B
:101A4000219620C1982F907E903CC1F4082F0F71F1
:101A500010E020E030E04801590186E0880C991C34
:101A6000AA1CBB1C8A95D1F7CE010196F6011995E7
:101A70008F7395018401082B229604C1982F907FC3
:101A8000903E19F58F70882E912CA12CB12C16E068
:101A9000880C991CAA1CBB1C1A95D1F7CE01019683
:101AA000F60119958F73882A06E0880C991CAA1CE8
:101AB000BB1C0A95D1F7CE010296F60119958F73DA
:101AC00095018401082B2396DDC0982F987F903FC5
:101AD00081F58770882E912CA12CB12CF6E0880C12
:101AE000991CAA1CBB1CFA95D1F7CE010196F601F0
:101AF00019958F73882AA6E0880C991CAA1CBB1C18
:101B0000AA95D1F7CE010296F60119958F73882A0E
:101B1000B6E0880C991CAA1CBB1CBA95D1F7CE0163
:101B20000396F60119958F7395018401082B24966D
:101B3000A9C0982F9C7F983FE9F58370882E912C3F
:101B4000A12CB12C56E0880C991CAA1CBB1C5A95E0
:101B5000D1F7CE010196F60119958F73882A66E0B8
:101B6000880C991CAA1CBB1C6A95D1F7CE01029661
:101B7000F60119958F73882A76E0880C991CAA1CA7
:101B8000BB1C7A95D1F7CE010396F60119958F7398
:101B9000882AE6E0880C991CAA1CBB1CEA95D1F7A0
:101BA000CE010496F60119958F7395018401082BD7
:101BB000259668C0982F9E7F9C3F09F04AC081708F
:101BC000882E912CA12CB12C86E0880C991CAA1C83
:101BD000BB1C8A95D1F7CE010196F60119958F733A
:101BE000882A96E0880C991CAA1CBB1C9A95D1F7F0
:101BF000CE010296F60119958F73882A26E0880C8B
:101C0000991CAA1CBB1C2A95D1F7CE010396F6019C
